

Microchip MPLAB XC8 Assembler V2.36 build 20220127204148 
                                                                                               Sun May 15 10:03:28 2022

Microchip MPLAB XC8 C Compiler v2.36 (Free license) build 20220127204148 Og1 
     1                           	processor	18F452
     2                           	fnconf	rparam,??,?,0
     3                           	pagewidth 120
     4                           	opt	flic
     5                           	psect	idataCOMRAM,global,class=CODE,delta=1,noexec
     6                           	psect	nvCOMRAM,global,class=COMRAM,space=1,delta=1,lowdata,noexec
     7                           	psect	smallconst,global,reloc=2,class=SMALLCONST,delta=1,noexec
     8                           	psect	cinit,global,reloc=2,class=CODE,delta=1
     9                           	psect	bssCOMRAM,global,class=COMRAM,space=1,delta=1,lowdata,noexec
    10                           	psect	dataCOMRAM,global,class=COMRAM,space=1,delta=1,lowdata,noexec
    11                           	psect	bssBANK0,global,class=BANK0,space=1,delta=1,lowdata,noexec
    12                           	psect	bssBANK1,global,class=BANK1,space=1,delta=1,lowdata,noexec
    13                           	psect	bssBANK2,global,class=BANK2,space=1,delta=1,lowdata,noexec
    14                           	psect	cstackBANK0,global,class=BANK0,space=1,delta=1,lowdata,noexec
    15                           	psect	cstackCOMRAM,global,class=COMRAM,space=1,delta=1,lowdata,noexec
    16                           	psect	text0,global,reloc=2,class=CODE,delta=1
    17                           	psect	text1,global,reloc=2,class=CODE,delta=1
    18                           	psect	text2,global,reloc=2,class=CODE,delta=1
    19                           	psect	text3,global,reloc=2,class=CODE,delta=1
    20                           	psect	text4,global,reloc=2,class=CODE,delta=1
    21                           	psect	text5,global,reloc=2,class=CODE,delta=1
    22                           	psect	text6,global,reloc=2,class=CODE,delta=1
    23                           	psect	text7,global,reloc=2,class=CODE,delta=1
    24                           	psect	text8,global,reloc=2,class=CODE,delta=1
    25                           	psect	text9,global,reloc=2,class=CODE,delta=1
    26                           	psect	text10,global,reloc=2,class=CODE,delta=1,group=1
    27                           	psect	text11,global,reloc=2,class=CODE,delta=1,group=1
    28                           	psect	text12,global,reloc=2,class=CODE,delta=1,group=1
    29                           	psect	text13,global,reloc=2,class=CODE,delta=1,group=1
    30                           	psect	text14,global,reloc=2,class=CODE,delta=1
    31                           	psect	text15,global,reloc=2,class=CODE,delta=1
    32                           	psect	text16,global,reloc=2,class=CODE,delta=1
    33                           	psect	text17,global,reloc=2,class=CODE,delta=1
    34                           	psect	text18,global,reloc=2,class=CODE,delta=1
    35                           	psect	text19,global,reloc=2,class=CODE,delta=1
    36                           	psect	text20,global,reloc=2,class=CODE,delta=1
    37                           	psect	text21,global,reloc=2,class=CODE,delta=1
    38                           	psect	text22,global,reloc=2,class=CODE,delta=1
    39                           	psect	text23,global,reloc=2,class=CODE,delta=1
    40                           	psect	text24,global,reloc=2,class=CODE,delta=1
    41                           	psect	text25,global,reloc=2,class=CODE,delta=1
    42                           	psect	text26,global,reloc=2,class=CODE,delta=1
    43                           	psect	text27,global,reloc=2,class=CODE,delta=1
    44                           	psect	text28,global,reloc=2,class=CODE,delta=1
    45                           	psect	text29,global,reloc=2,class=CODE,delta=1
    46                           	psect	intcode,global,reloc=2,class=CODE,delta=1
    47                           	psect	text31,global,reloc=2,class=CODE,delta=1,group=2
    48                           	psect	intsave_regs,global,class=BIGRAM,space=1,delta=1,noexec
    49                           	psect	rparam,global,class=COMRAM,space=1,delta=1,noexec
    50                           	psect	temp,global,ovrld,common,class=COMRAM,space=1,delta=1
    51                           	psect	idloc,global,abs,ovrld,class=IDLOC,space=5,delta=1,noexec
    52                           	psect	config,global,abs,ovrld,class=CONFIG,space=4,delta=1,noexec
    53  0000                     
    54                           ; Version 2.20
    55                           ; Generated 12/02/2020 GMT
    56                           ; 
    57                           ; Copyright © 2020, Microchip Technology Inc. and its subsidiaries ("Microchip")
    58                           ; All rights reserved.
    59                           ; 
    60                           ; This software is developed by Microchip Technology Inc. and its subsidiaries ("Microch
      +                          ip").
    61                           ; 
    62                           ; Redistribution and use in source and binary forms, with or without modification, are
    63                           ; permitted provided that the following conditions are met:
    64                           ; 
    65                           ;     1. Redistributions of source code must retain the above copyright notice, this lis
      +                          t of
    66                           ;        conditions and the following disclaimer.
    67                           ; 
    68                           ;     2. Redistributions in binary form must reproduce the above copyright notice, this 
      +                          list
    69                           ;        of conditions and the following disclaimer in the documentation and/or other
    70                           ;        materials provided with the distribution.
    71                           ; 
    72                           ;     3. Microchip's name may not be used to endorse or promote products derived from th
      +                          is
    73                           ;        software without specific prior written permission.
    74                           ; 
    75                           ; THIS SOFTWARE IS PROVIDED BY MICROCHIP "AS IS" AND ANY EXPRESS OR IMPLIED WARRANTIES,
    76                           ; INCLUDING, BUT NOT LIMITED TO, THE IMPLIED WARRANTIES OF MERCHANTABILITY AND FITNESS F
      +                          OR
    77                           ; PURPOSE ARE DISCLAIMED.  IN NO EVENT SHALL MICROCHIP BE LIABLE FOR ANY DIRECT, INDIREC
      +                          T,
    78                           ; INCIDENTAL, SPECIAL, EXEMPLARY, OR CONSEQUENTIAL DAMAGES (INCLUDING BUT NOT LIMITED TO
    79                           ; PROCUREMENT OF SUBSTITUTE GOODS OR SERVICES; LOSS OF USE, DATA OR PROFITS; OR BUSINESS
    80                           ; INTERRUPTION) HOWSOEVER CAUSED AND ON ANY THEORY OF LIABILITY, WHETHER IN CONTRACT, ST
      +                          RICT
    81                           ; LIABILITY, OR TORT (INCLUDING NEGLIGENCE OR OTHERWISE) ARISING IN ANY WAY OUT OF THE U
      +                          SE OF
    82                           ; THIS SOFTWARE, EVEN IF ADVISED OF THE POSSIBILITY OF SUCH DAMAGE.
    83                           ; 
    84                           ; 
    85                           ; Code-generator required, PIC18F452 Definitions
    86                           ; 
    87                           ; SFR Addresses
    88  0000                     
    89                           	psect	idataCOMRAM
    90  001F6C                     __pidataCOMRAM:
    91                           	callstack 0
    92                           
    93                           ;initializer for _mask
    94  001F6C  0003               	dw	3
    95                           
    96                           ;initializer for _BackLight_State
    97  001F6E  08                 	db	8
    98  0000                     _SSPBUF	set	4041
    99  0000                     _SSPADD	set	4040
   100  0000                     _SSPSTAT	set	4039
   101  0000                     _RCREG	set	4014
   102  0000                     _TXREG	set	4013
   103  0000                     _SPBRG	set	4015
   104  0000                     _TXSTAbits	set	4012
   105                           
   106                           	psect	nvCOMRAM
   107  000069                     __pnvCOMRAM:
   108                           	callstack 0
   109  000069                     _periodo:
   110                           	callstack 0
   111  000069                     	ds	2
   112  00006B                     _i2c_add:
   113                           	callstack 0
   114  00006B                     	ds	1
   115  0000                     _RCEN	set	32299
   116  0000                     _ACKSTAT	set	32302
   117  0000                     _SSPIF	set	31987
   118  0000                     _ACKEN	set	32300
   119  0000                     _ACKDT	set	32301
   120  0000                     _PEN	set	32298
   121  0000                     _RSEN	set	32297
   122  0000                     _SEN	set	32296
   123  0000                     _TRISC4	set	31908
   124  0000                     _TRISC3	set	31907
   125  0000                     _TRISC7	set	31911
   126  0000                     _TRISC6	set	31910
   127  0000                     _LATAbits	set	3977
   128  0000                     _TRISA	set	3986
   129  0000                     _TRISBbits	set	3987
   130  0000                     _TRISCbits	set	3988
   131  0000                     _CCP1CON	set	4029
   132  0000                     _PR2	set	4043
   133  0000                     _RCONbits	set	4048
   134  0000                     _ADCON1	set	4033
   135  0000                     _T2CON	set	4042
   136  0000                     _CCPR1L	set	4030
   137  0000                     _PIE1bits	set	3997
   138  0000                     _CCP2CON	set	4026
   139  0000                     _CCPR2L	set	4027
   140  0000                     _INTCONbits	set	4082
   141  0000                     _PIR1bits	set	3998
   142  0000                     _RCSTAbits	set	4011
   143  0000                     _SSPCON2	set	4037
   144  0000                     _SSPCON1	set	4038
   145                           
   146                           	psect	smallconst
   147  000600                     __psmallconst:
   148                           	callstack 0
   149  000600  00                 	db	0
   150  000601                     STR_1:
   151  000601  52                 	db	82	;'R'
   152  000602  6F                 	db	111	;'o'
   153  000603  62                 	db	98	;'b'
   154  000604  6F                 	db	111	;'o'
   155  000605  74                 	db	116	;'t'
   156  000606  21                 	db	33
   157  000607  00                 	db	0
   158  000608  00                 	db	0	; dummy byte at the end
   159  0000                     
   160                           ; #config settings
   161                           
   162                           	psect	cinit
   163  001CEE                     __pcinit:
   164                           	callstack 0
   165  001CEE                     start_initialization:
   166                           	callstack 0
   167  001CEE                     __initialization:
   168                           	callstack 0
   169                           
   170                           ; Initialize objects allocated to COMRAM (3 bytes)
   171                           ; load TBLPTR registers with __pidataCOMRAM
   172  001CEE  0E6C               	movlw	low __pidataCOMRAM
   173  001CF0  6EF6               	movwf	tblptrl,c
   174  001CF2  0E1F               	movlw	high __pidataCOMRAM
   175  001CF4  6EF7               	movwf	tblptrh,c
   176  001CF6  0E00               	movlw	low (__pidataCOMRAM shr (0+16))
   177  001CF8  6EF8               	movwf	tblptru,c
   178  001CFA  0009               	tblrd		*+	;fetch initializer
   179  001CFC  CFF5 F06C          	movff	tablat,__pdataCOMRAM
   180  001D00  0009               	tblrd		*+	;fetch initializer
   181  001D02  CFF5 F06D          	movff	tablat,__pdataCOMRAM+1
   182  001D06  0009               	tblrd		*+	;fetch initializer
   183  001D08  CFF5 F06E          	movff	tablat,__pdataCOMRAM+2
   184                           
   185                           ; Clear objects allocated to BANK2 (255 bytes)
   186  001D0C  EE02  F000         	lfsr	0,__pbssBANK2
   187  001D10  EE10 F0FF          	lfsr	1,255
   188  001D14                     clear_0:
   189  001D14  6AEE               	clrf	postinc0,c
   190  001D16  50E5               	movf	postdec1,w,c
   191  001D18  50E1               	movf	fsr1l,w,c
   192  001D1A  E1FC               	bnz	clear_0
   193  001D1C  50E2               	movf	fsr1h,w,c
   194  001D1E  E1FA               	bnz	clear_0
   195                           
   196                           ; Clear objects allocated to BANK1 (100 bytes)
   197  001D20  EE01  F000         	lfsr	0,__pbssBANK1
   198  001D24  0E64               	movlw	100
   199  001D26                     clear_1:
   200  001D26  6AEE               	clrf	postinc0,c
   201  001D28  06E8               	decf	wreg,f,c
   202  001D2A  E1FD               	bnz	clear_1
   203                           
   204                           ; Clear objects allocated to BANK0 (42 bytes)
   205  001D2C  EE00  F080         	lfsr	0,__pbssBANK0
   206  001D30  0E2A               	movlw	42
   207  001D32                     clear_2:
   208  001D32  6AEE               	clrf	postinc0,c
   209  001D34  06E8               	decf	wreg,f,c
   210  001D36  E1FD               	bnz	clear_2
   211                           
   212                           ; Clear objects allocated to COMRAM (8 bytes)
   213  001D38  EE00  F061         	lfsr	0,__pbssCOMRAM
   214  001D3C  0E08               	movlw	8
   215  001D3E                     clear_3:
   216  001D3E  6AEE               	clrf	postinc0,c
   217  001D40  06E8               	decf	wreg,f,c
   218  001D42  E1FD               	bnz	clear_3
   219  001D44                     end_of_initialization:
   220                           	callstack 0
   221  001D44                     __end_of__initialization:
   222                           	callstack 0
   223  001D44  906F               	bcf	int$flags,0,c	;clear compiler interrupt flag (level 1)
   224  001D46  926F               	bcf	int$flags,1,c	;clear compiler interrupt flag (level 2)
   225  001D48  0E00               	movlw	low (__Lmediumconst shr (0+16))
   226  001D4A  6EF8               	movwf	tblptru,c
   227  001D4C  0100               	movlb	0
   228  001D4E  EFF0  F00B         	goto	_main	;jump to C main() function
   229                           
   230                           	psect	bssCOMRAM
   231  000061                     __pbssCOMRAM:
   232                           	callstack 0
   233  000061                     _duty_temp:
   234                           	callstack 0
   235  000061                     	ds	2
   236  000063                     _cont_rc:
   237                           	callstack 0
   238  000063                     	ds	2
   239  000065                     _valor_prueba_debug2:
   240                           	callstack 0
   241  000065                     	ds	1
   242  000066                     _valor_prueba_debug:
   243                           	callstack 0
   244  000066                     	ds	1
   245  000067                     _data:
   246                           	callstack 0
   247  000067                     	ds	1
   248  000068                     _RS:
   249                           	callstack 0
   250  000068                     	ds	1
   251                           
   252                           	psect	dataCOMRAM
   253  00006C                     __pdataCOMRAM:
   254                           	callstack 0
   255  00006C                     _mask:
   256                           	callstack 0
   257  00006C                     	ds	2
   258  00006E                     _BackLight_State:
   259                           	callstack 0
   260  00006E                     	ds	1
   261                           
   262                           	psect	bssBANK0
   263  000080                     __pbssBANK0:
   264                           	callstack 0
   265  000080                     _test_buff:
   266                           	callstack 0
   267  000080                     	ds	30
   268  00009E                     _tmr2_presc:
   269                           	callstack 0
   270  00009E                     	ds	4
   271  0000A2                     _frec_osc:
   272                           	callstack 0
   273  0000A2                     	ds	4
   274  0000A6                     _pwm_p:
   275                           	callstack 0
   276  0000A6                     	ds	4
   277                           
   278                           	psect	bssBANK1
   279  000100                     __pbssBANK1:
   280                           	callstack 0
   281  000100                     _rc_buff:
   282                           	callstack 0
   283  000100                     	ds	100
   284                           
   285                           	psect	bssBANK2
   286  000200                     __pbssBANK2:
   287                           	callstack 0
   288  000200                     _rc_data:
   289                           	callstack 0
   290  000200                     	ds	255
   291                           
   292                           	psect	cstackBANK0
   293  0000AA                     __pcstackBANK0:
   294                           	callstack 0
   295  0000AA                     globalPWM@period_pwm:
   296                           	callstack 0
   297  0000AA                     setPWM@period_pwm:
   298                           	callstack 0
   299                           
   300                           ; 4 bytes @ 0x0
   301  0000AA                     	ds	4
   302  0000AE                     globalPWM@freq_osc:
   303                           	callstack 0
   304  0000AE                     setPWM@pwm_duty:
   305                           	callstack 0
   306                           
   307                           ; 4 bytes @ 0x4
   308  0000AE                     	ds	4
   309  0000B2                     globalPWM@presc:
   310                           	callstack 0
   311  0000B2                     setPWM@freq_osc:
   312                           	callstack 0
   313                           
   314                           ; 4 bytes @ 0x8
   315  0000B2                     	ds	4
   316  0000B6                     setPWM@presc:
   317                           	callstack 0
   318                           
   319                           ; 4 bytes @ 0xC
   320  0000B6                     	ds	4
   321  0000BA                     setPWM@module:
   322                           	callstack 0
   323                           
   324                           ; 2 bytes @ 0x10
   325  0000BA                     	ds	2
   326  0000BC                     _setPWM$1410:
   327                           	callstack 0
   328                           
   329                           ; 4 bytes @ 0x12
   330  0000BC                     	ds	4
   331  0000C0                     _setPWM$1411:
   332                           	callstack 0
   333                           
   334                           ; 4 bytes @ 0x16
   335  0000C0                     	ds	4
   336                           
   337                           	psect	cstackCOMRAM
   338  000001                     __pcstackCOMRAM:
   339                           	callstack 0
   340  000001                     strcpy@dest:
   341                           	callstack 0
   342                           
   343                           ; 2 bytes @ 0x0
   344  000001                     	ds	2
   345  000003                     strcpy@src:
   346                           	callstack 0
   347                           
   348                           ; 2 bytes @ 0x2
   349  000003                     	ds	2
   350  000005                     strcpy@s:
   351                           	callstack 0
   352                           
   353                           ; 2 bytes @ 0x4
   354  000005                     	ds	2
   355  000007                     strcpy@d:
   356                           	callstack 0
   357                           
   358                           ; 2 bytes @ 0x6
   359  000007                     	ds	2
   360  000009                     ??_adint:
   361                           
   362                           ; 1 bytes @ 0x8
   363  000009                     	ds	6
   364  00000F                     ??_I2C_Master_Wait:
   365  00000F                     ?___fldiv:
   366                           	callstack 0
   367  00000F                     ___fldiv@b:
   368                           	callstack 0
   369                           
   370                           ; 4 bytes @ 0xE
   371  00000F                     	ds	1
   372  000010                     I2C_Master_Write@data:
   373                           	callstack 0
   374                           
   375                           ; 1 bytes @ 0xF
   376  000010                     	ds	1
   377  000011                     IO_Expander_Write@Data:
   378                           	callstack 0
   379                           
   380                           ; 1 bytes @ 0x10
   381  000011                     	ds	1
   382  000012                     LCD_Write_4Bit@Nibble:
   383                           	callstack 0
   384                           
   385                           ; 1 bytes @ 0x11
   386  000012                     	ds	1
   387  000013                     LCD_CMD@CMD:
   388                           	callstack 0
   389  000013                     LCD_Write_Char@Data:
   390                           	callstack 0
   391  000013                     ___fldiv@a:
   392                           	callstack 0
   393                           
   394                           ; 4 bytes @ 0x12
   395  000013                     	ds	1
   396  000014                     ??_LCD_Init:
   397  000014                     LCD_Set_Cursor@COL:
   398                           	callstack 0
   399  000014                     LCD_Write_String@Str:
   400                           	callstack 0
   401                           
   402                           ; 2 bytes @ 0x13
   403  000014                     	ds	1
   404  000015                     ??_LCD_Set_Cursor:
   405                           
   406                           ; 1 bytes @ 0x14
   407  000015                     	ds	1
   408  000016                     ??_LCD_Write_String:
   409  000016                     LCD_Init@I2C_Add:
   410                           	callstack 0
   411                           
   412                           ; 1 bytes @ 0x15
   413  000016                     	ds	1
   414  000017                     ??___fldiv:
   415  000017                     LCD_Set_Cursor@ROW:
   416                           	callstack 0
   417                           
   418                           ; 1 bytes @ 0x16
   419  000017                     	ds	1
   420  000018                     LCD_Write_String@i:
   421                           	callstack 0
   422                           
   423                           ; 2 bytes @ 0x17
   424  000018                     	ds	3
   425  00001B                     ___fldiv@rem:
   426                           	callstack 0
   427                           
   428                           ; 4 bytes @ 0x1A
   429  00001B                     	ds	4
   430  00001F                     ___fldiv@sign:
   431                           	callstack 0
   432                           
   433                           ; 1 bytes @ 0x1E
   434  00001F                     	ds	1
   435  000020                     ___fldiv@new_exp:
   436                           	callstack 0
   437                           
   438                           ; 2 bytes @ 0x1F
   439  000020                     	ds	2
   440  000022                     ___fldiv@grs:
   441                           	callstack 0
   442                           
   443                           ; 4 bytes @ 0x21
   444  000022                     	ds	4
   445  000026                     ___fldiv@bexp:
   446                           	callstack 0
   447                           
   448                           ; 1 bytes @ 0x25
   449  000026                     	ds	1
   450  000027                     ___fldiv@aexp:
   451                           	callstack 0
   452                           
   453                           ; 1 bytes @ 0x26
   454  000027                     	ds	1
   455  000028                     ?___flmul:
   456                           	callstack 0
   457  000028                     ___flmul@b:
   458                           	callstack 0
   459                           
   460                           ; 4 bytes @ 0x27
   461  000028                     	ds	4
   462  00002C                     ___flmul@a:
   463                           	callstack 0
   464                           
   465                           ; 4 bytes @ 0x2B
   466  00002C                     	ds	4
   467  000030                     ??___flmul:
   468                           
   469                           ; 1 bytes @ 0x2F
   470  000030                     	ds	4
   471  000034                     ___flmul@sign:
   472                           	callstack 0
   473                           
   474                           ; 1 bytes @ 0x33
   475  000034                     	ds	1
   476  000035                     ___flmul@grs:
   477                           	callstack 0
   478                           
   479                           ; 4 bytes @ 0x34
   480  000035                     	ds	4
   481  000039                     ___flmul@aexp:
   482                           	callstack 0
   483                           
   484                           ; 1 bytes @ 0x38
   485  000039                     	ds	1
   486  00003A                     ___flmul@bexp:
   487                           	callstack 0
   488                           
   489                           ; 1 bytes @ 0x39
   490  00003A                     	ds	1
   491  00003B                     ___flmul@prod:
   492                           	callstack 0
   493                           
   494                           ; 4 bytes @ 0x3A
   495  00003B                     	ds	4
   496  00003F                     ___flmul@temp:
   497                           	callstack 0
   498                           
   499                           ; 2 bytes @ 0x3E
   500  00003F                     	ds	2
   501  000041                     ?___fladd:
   502                           	callstack 0
   503  000041                     ___fladd@b:
   504                           	callstack 0
   505                           
   506                           ; 4 bytes @ 0x40
   507  000041                     	ds	4
   508  000045                     ___fladd@a:
   509                           	callstack 0
   510                           
   511                           ; 4 bytes @ 0x44
   512  000045                     	ds	4
   513  000049                     ??___fladd:
   514                           
   515                           ; 1 bytes @ 0x48
   516  000049                     	ds	4
   517  00004D                     ___fladd@signs:
   518                           	callstack 0
   519                           
   520                           ; 1 bytes @ 0x4C
   521  00004D                     	ds	1
   522  00004E                     ___fladd@aexp:
   523                           	callstack 0
   524                           
   525                           ; 1 bytes @ 0x4D
   526  00004E                     	ds	1
   527  00004F                     ___fladd@bexp:
   528                           	callstack 0
   529                           
   530                           ; 1 bytes @ 0x4E
   531  00004F                     	ds	1
   532  000050                     ___fladd@grs:
   533                           	callstack 0
   534                           
   535                           ; 1 bytes @ 0x4F
   536  000050                     	ds	1
   537  000051                     ?___fltol:
   538                           	callstack 0
   539  000051                     ___fltol@f1:
   540                           	callstack 0
   541                           
   542                           ; 4 bytes @ 0x50
   543  000051                     	ds	4
   544  000055                     ??___fltol:
   545                           
   546                           ; 1 bytes @ 0x54
   547  000055                     	ds	4
   548  000059                     ___fltol@sign1:
   549                           	callstack 0
   550                           
   551                           ; 1 bytes @ 0x58
   552  000059                     	ds	1
   553  00005A                     ___fltol@exp1:
   554                           	callstack 0
   555                           
   556                           ; 1 bytes @ 0x59
   557  00005A                     	ds	1
   558  00005B                     ??_setPWM:
   559  00005B                     _globalPWM$1409:
   560                           	callstack 0
   561                           
   562                           ; 4 bytes @ 0x5A
   563  00005B                     	ds	4
   564  00005F                     ??_main:
   565                           
   566                           ; 1 bytes @ 0x5E
   567  00005F                     	ds	2
   568                           
   569 ;;
   570 ;;Main: autosize = 0, tempsize = 2, incstack = 0, save=0
   571 ;;
   572 ;; *************** function _main *****************
   573 ;; Defined at:
   574 ;;		line 315 in file "mainTx.c"
   575 ;; Parameters:    Size  Location     Type
   576 ;;		None
   577 ;; Auto vars:     Size  Location     Type
   578 ;;		None
   579 ;; Return value:  Size  Location     Type
   580 ;;                  2  158[None  ] int 
   581 ;; Registers used:
   582 ;;		wreg, status,2, status,0, tblptrl, tblptrh, tblptru, prodl, prodh, cstack
   583 ;; Tracked objects:
   584 ;;		On entry : 0/0
   585 ;;		On exit  : 0/0
   586 ;;		Unchanged: 0/0
   587 ;; Data sizes:     COMRAM   BANK0   BANK1   BANK2   BANK3   BANK4   BANK5
   588 ;;      Params:         0       0       0       0       0       0       0
   589 ;;      Locals:         0       0       0       0       0       0       0
   590 ;;      Temps:          2       0       0       0       0       0       0
   591 ;;      Totals:         2       0       0       0       0       0       0
   592 ;;Total ram usage:        2 bytes
   593 ;; Hardware stack levels required when called: 8
   594 ;; This function calls:
   595 ;;		_LCD_Init
   596 ;;		_LCD_Set_Cursor
   597 ;;		_LCD_Write_String
   598 ;;		_adelanteL
   599 ;;		_adelanteR
   600 ;;		_atrasL
   601 ;;		_atrasR
   602 ;;		_boot
   603 ;;		_setPWM
   604 ;;		_stopL
   605 ;;		_stopR
   606 ;; This function is called by:
   607 ;;		Startup code after reset
   608 ;; This function uses a non-reentrant model
   609 ;;
   610                           
   611                           	psect	text0
   612  0017E0                     __ptext0:
   613                           	callstack 0
   614  0017E0                     _main:
   615                           	callstack 23
   616  0017E0  FFFF               	dw	65535	; assembler added errata NOP
   617                           
   618                           ;mainTx.c: 316:     boot();
   619  0017E2  ECA9  F00E         	call	_boot	;wreg free
   620  0017E6                     
   621                           ;mainTx.c: 317:     LCD_Init(0x4E);
   622  0017E6  0E4E               	movlw	78
   623  0017E8  EC26  F00D         	call	_LCD_Init
   624  0017EC                     
   625                           ;mainTx.c: 318:     LCD_Set_Cursor(1,1);
   626  0017EC  0E01               	movlw	1
   627  0017EE  6E14               	movwf	LCD_Set_Cursor@COL^0,c
   628  0017F0  0E01               	movlw	1
   629  0017F2  EC06  F00E         	call	_LCD_Set_Cursor
   630  0017F6                     
   631                           ;mainTx.c: 319:     LCD_Write_String("Robot!");
   632  0017F6  0E01               	movlw	low STR_1
   633  0017F8  6E14               	movwf	LCD_Write_String@Str^0,c
   634  0017FA  0E06               	movlw	high STR_1
   635  0017FC  6E15               	movwf	(LCD_Write_String@Str+1)^0,c
   636  0017FE  EC44  F00E         	call	_LCD_Write_String	;wreg free
   637  001802                     
   638                           ;mainTx.c: 328:     setPWM(1e0/2e3, 100, 16e6, 16e0, 1);
   639  001802  0E6F               	movlw	111
   640  001804  0100               	movlb	0	; () banked
   641  001806  6FAA               	movwf	setPWM@period_pwm& (0+255),b
   642  001808  0E12               	movlw	18
   643  00180A  6FAB               	movwf	(setPWM@period_pwm+1)& (0+255),b
   644  00180C  0E03               	movlw	3
   645  00180E  6FAC               	movwf	(setPWM@period_pwm+2)& (0+255),b
   646  001810  0E3A               	movlw	58
   647  001812  6FAD               	movwf	(setPWM@period_pwm+3)& (0+255),b
   648  001814  0E00               	movlw	0
   649  001816  6FAE               	movwf	setPWM@pwm_duty& (0+255),b
   650  001818  0E00               	movlw	0
   651  00181A  6FAF               	movwf	(setPWM@pwm_duty+1)& (0+255),b
   652  00181C  0EC8               	movlw	200
   653  00181E  6FB0               	movwf	(setPWM@pwm_duty+2)& (0+255),b
   654  001820  0E42               	movlw	66
   655  001822  6FB1               	movwf	(setPWM@pwm_duty+3)& (0+255),b
   656  001824  0E00               	movlw	0
   657  001826  6FB2               	movwf	setPWM@freq_osc& (0+255),b
   658  001828  0E24               	movlw	36
   659  00182A  6FB3               	movwf	(setPWM@freq_osc+1)& (0+255),b
   660  00182C  0E74               	movlw	116
   661  00182E  6FB4               	movwf	(setPWM@freq_osc+2)& (0+255),b
   662  001830  0E4B               	movlw	75
   663  001832  6FB5               	movwf	(setPWM@freq_osc+3)& (0+255),b
   664  001834  0E00               	movlw	0
   665  001836  6FB6               	movwf	setPWM@presc& (0+255),b
   666  001838  0E00               	movlw	0
   667  00183A  6FB7               	movwf	(setPWM@presc+1)& (0+255),b
   668  00183C  0E80               	movlw	128
   669  00183E  6FB8               	movwf	(setPWM@presc+2)& (0+255),b
   670  001840  0E41               	movlw	65
   671  001842  6FB9               	movwf	(setPWM@presc+3)& (0+255),b
   672  001844  0E00               	movlw	0
   673  001846  6FBB               	movwf	(setPWM@module+1)& (0+255),b
   674  001848  0E01               	movlw	1
   675  00184A  6FBA               	movwf	setPWM@module& (0+255),b
   676  00184C  EC44  F00A         	call	_setPWM	;wreg free
   677  001850                     
   678                           ;mainTx.c: 329:     setPWM(1e0/2e3, 100, 16e6, 16e0, 2);
   679  001850  0E6F               	movlw	111
   680  001852  0100               	movlb	0	; () banked
   681  001854  6FAA               	movwf	setPWM@period_pwm& (0+255),b
   682  001856  0E12               	movlw	18
   683  001858  6FAB               	movwf	(setPWM@period_pwm+1)& (0+255),b
   684  00185A  0E03               	movlw	3
   685  00185C  6FAC               	movwf	(setPWM@period_pwm+2)& (0+255),b
   686  00185E  0E3A               	movlw	58
   687  001860  6FAD               	movwf	(setPWM@period_pwm+3)& (0+255),b
   688  001862  0E00               	movlw	0
   689  001864  6FAE               	movwf	setPWM@pwm_duty& (0+255),b
   690  001866  0E00               	movlw	0
   691  001868  6FAF               	movwf	(setPWM@pwm_duty+1)& (0+255),b
   692  00186A  0EC8               	movlw	200
   693  00186C  6FB0               	movwf	(setPWM@pwm_duty+2)& (0+255),b
   694  00186E  0E42               	movlw	66
   695  001870  6FB1               	movwf	(setPWM@pwm_duty+3)& (0+255),b
   696  001872  0E00               	movlw	0
   697  001874  6FB2               	movwf	setPWM@freq_osc& (0+255),b
   698  001876  0E24               	movlw	36
   699  001878  6FB3               	movwf	(setPWM@freq_osc+1)& (0+255),b
   700  00187A  0E74               	movlw	116
   701  00187C  6FB4               	movwf	(setPWM@freq_osc+2)& (0+255),b
   702  00187E  0E4B               	movlw	75
   703  001880  6FB5               	movwf	(setPWM@freq_osc+3)& (0+255),b
   704  001882  0E00               	movlw	0
   705  001884  6FB6               	movwf	setPWM@presc& (0+255),b
   706  001886  0E00               	movlw	0
   707  001888  6FB7               	movwf	(setPWM@presc+1)& (0+255),b
   708  00188A  0E80               	movlw	128
   709  00188C  6FB8               	movwf	(setPWM@presc+2)& (0+255),b
   710  00188E  0E41               	movlw	65
   711  001890  6FB9               	movwf	(setPWM@presc+3)& (0+255),b
   712  001892  0E00               	movlw	0
   713  001894  6FBB               	movwf	(setPWM@module+1)& (0+255),b
   714  001896  0E02               	movlw	2
   715  001898  6FBA               	movwf	setPWM@module& (0+255),b
   716  00189A  EC44  F00A         	call	_setPWM	;wreg free
   717  00189E                     
   718                           ;mainTx.c: 331:     cont_rc = 0;
   719  00189E  0E00               	movlw	0
   720  0018A0  6E64               	movwf	(_cont_rc+1)^0,c
   721  0018A2  0E00               	movlw	0
   722  0018A4  6E63               	movwf	_cont_rc^0,c
   723  0018A6                     l2689:
   724  0018A6  FFFF               	dw	65535	; assembler added errata NOP
   725                           
   726                           ;mainTx.c: 338:         adelanteL();
   727  0018A8  ECA9  F00F         	call	_adelanteL	;wreg free
   728  0018AC                     
   729                           ;mainTx.c: 339:         adelanteR();
   730  0018AC  ECA4  F00F         	call	_adelanteR	;wreg free
   731  0018B0                     
   732                           ;mainTx.c: 340:         _delay((unsigned long)((5000)*(16000000/4000.0)));
   733  0018B0  0E4D               	movlw	77
   734  0018B2  6E60               	movwf	(??_main+1)^0,c
   735  0018B4  0E26               	movlw	38
   736  0018B6  6E5F               	movwf	??_main^0,c
   737  0018B8  0E05               	movlw	5
   738  0018BA                     u1897:
   739  0018BA  FFFF               	dw	65535	; errata NOP
   740  0018BC  2EE8               	decfsz	wreg,f,c
   741  0018BE  D7FD               	bra	u1897
   742  0018C0  2E5F               	decfsz	??_main^0,f,c
   743  0018C2  D7FB               	bra	u1897
   744  0018C4  2E60               	decfsz	(??_main+1)^0,f,c
   745  0018C6  D7F9               	bra	u1897
   746  0018C8  D000               	nop2	
   747  0018CA                     
   748                           ;mainTx.c: 341:         atrasL();
   749  0018CA  EC9F  F00F         	call	_atrasL	;wreg free
   750  0018CE                     
   751                           ;mainTx.c: 342:         atrasR();
   752  0018CE  EC9A  F00F         	call	_atrasR	;wreg free
   753  0018D2                     
   754                           ;mainTx.c: 343:         _delay((unsigned long)((5000)*(16000000/4000.0)));
   755  0018D2  0E4D               	movlw	77
   756  0018D4  6E60               	movwf	(??_main+1)^0,c
   757  0018D6  0E26               	movlw	38
   758  0018D8  6E5F               	movwf	??_main^0,c
   759  0018DA  0E05               	movlw	5
   760  0018DC                     u1907:
   761  0018DC  FFFF               	dw	65535	; errata NOP
   762  0018DE  2EE8               	decfsz	wreg,f,c
   763  0018E0  D7FD               	bra	u1907
   764  0018E2  2E5F               	decfsz	??_main^0,f,c
   765  0018E4  D7FB               	bra	u1907
   766  0018E6  2E60               	decfsz	(??_main+1)^0,f,c
   767  0018E8  D7F9               	bra	u1907
   768  0018EA  D000               	nop2	
   769  0018EC                     
   770                           ;mainTx.c: 344:         stopL();
   771  0018EC  EC95  F00F         	call	_stopL	;wreg free
   772  0018F0                     
   773                           ;mainTx.c: 345:         stopR();
   774  0018F0  EC90  F00F         	call	_stopR	;wreg free
   775  0018F4                     
   776                           ;mainTx.c: 346:         _delay((unsigned long)((5000)*(16000000/4000.0)));
   777  0018F4  0E4D               	movlw	77
   778  0018F6  6E60               	movwf	(??_main+1)^0,c
   779  0018F8  0E26               	movlw	38
   780  0018FA  6E5F               	movwf	??_main^0,c
   781  0018FC  0E05               	movlw	5
   782  0018FE                     u1917:
   783  0018FE  FFFF               	dw	65535	; errata NOP
   784  001900  2EE8               	decfsz	wreg,f,c
   785  001902  D7FD               	bra	u1917
   786  001904  2E5F               	decfsz	??_main^0,f,c
   787  001906  D7FB               	bra	u1917
   788  001908  2E60               	decfsz	(??_main+1)^0,f,c
   789  00190A  D7F9               	bra	u1917
   790  00190C  D000               	nop2	
   791  00190E  EF53  F00C         	goto	l2689
   792  001912  EF59  F000         	goto	start
   793  001916                     __end_of_main:
   794                           	callstack 0
   795                           
   796 ;; *************** function _stopR *****************
   797 ;; Defined at:
   798 ;;		line 89 in file "mainTx.c"
   799 ;; Parameters:    Size  Location     Type
   800 ;;		None
   801 ;; Auto vars:     Size  Location     Type
   802 ;;		None
   803 ;; Return value:  Size  Location     Type
   804 ;;                  1    wreg      void 
   805 ;; Registers used:
   806 ;;		None
   807 ;; Tracked objects:
   808 ;;		On entry : 0/0
   809 ;;		On exit  : 0/0
   810 ;;		Unchanged: 0/0
   811 ;; Data sizes:     COMRAM   BANK0   BANK1   BANK2   BANK3   BANK4   BANK5
   812 ;;      Params:         0       0       0       0       0       0       0
   813 ;;      Locals:         0       0       0       0       0       0       0
   814 ;;      Temps:          0       0       0       0       0       0       0
   815 ;;      Totals:         0       0       0       0       0       0       0
   816 ;;Total ram usage:        0 bytes
   817 ;; Hardware stack levels used: 1
   818 ;; Hardware stack levels required when called: 2
   819 ;; This function calls:
   820 ;;		Nothing
   821 ;; This function is called by:
   822 ;;		_main
   823 ;; This function uses a non-reentrant model
   824 ;;
   825                           
   826                           	psect	text1
   827  001F20                     __ptext1:
   828                           	callstack 0
   829  001F20                     _stopR:
   830                           	callstack 0
   831  001F20  FFFF               	dw	65535	; assembler added errata NOP
   832  001F22                     
   833                           ;mainTx.c: 90:     LATAbits.LATA0 = 1;
   834  001F22  8089               	bsf	137,0,c	;volatile
   835                           
   836                           ;mainTx.c: 91:     LATAbits.LATA1 = 1;
   837  001F24  8289               	bsf	137,1,c	;volatile
   838  001F26  0012               	return		;funcret
   839  001F28  FFFF               	dw	65535	; errata NOP
   840  001F2A                     __end_of_stopR:
   841                           	callstack 0
   842                           
   843 ;; *************** function _stopL *****************
   844 ;; Defined at:
   845 ;;		line 73 in file "mainTx.c"
   846 ;; Parameters:    Size  Location     Type
   847 ;;		None
   848 ;; Auto vars:     Size  Location     Type
   849 ;;		None
   850 ;; Return value:  Size  Location     Type
   851 ;;                  1    wreg      void 
   852 ;; Registers used:
   853 ;;		None
   854 ;; Tracked objects:
   855 ;;		On entry : 0/0
   856 ;;		On exit  : 0/0
   857 ;;		Unchanged: 0/0
   858 ;; Data sizes:     COMRAM   BANK0   BANK1   BANK2   BANK3   BANK4   BANK5
   859 ;;      Params:         0       0       0       0       0       0       0
   860 ;;      Locals:         0       0       0       0       0       0       0
   861 ;;      Temps:          0       0       0       0       0       0       0
   862 ;;      Totals:         0       0       0       0       0       0       0
   863 ;;Total ram usage:        0 bytes
   864 ;; Hardware stack levels used: 1
   865 ;; Hardware stack levels required when called: 2
   866 ;; This function calls:
   867 ;;		Nothing
   868 ;; This function is called by:
   869 ;;		_main
   870 ;; This function uses a non-reentrant model
   871 ;;
   872                           
   873                           	psect	text2
   874  001F2A                     __ptext2:
   875                           	callstack 0
   876  001F2A                     _stopL:
   877                           	callstack 0
   878  001F2A  FFFF               	dw	65535	; assembler added errata NOP
   879  001F2C                     
   880                           ;mainTx.c: 74:     LATAbits.LATA2 = 1;
   881  001F2C  8489               	bsf	137,2,c	;volatile
   882                           
   883                           ;mainTx.c: 75:     LATAbits.LATA3 = 1;
   884  001F2E  8689               	bsf	137,3,c	;volatile
   885  001F30  0012               	return		;funcret
   886  001F32  FFFF               	dw	65535	; errata NOP
   887  001F34                     __end_of_stopL:
   888                           	callstack 0
   889                           
   890 ;; *************** function _setPWM *****************
   891 ;; Defined at:
   892 ;;		line 103 in file "mainTx.c"
   893 ;; Parameters:    Size  Location     Type
   894 ;;  period_pwm      4    0[BANK0 ] float 
   895 ;;  pwm_duty        4    4[BANK0 ] float 
   896 ;;  freq_osc        4    8[BANK0 ] float 
   897 ;;  presc           4   12[BANK0 ] float 
   898 ;;  module          2   16[BANK0 ] int 
   899 ;; Auto vars:     Size  Location     Type
   900 ;;		None
   901 ;; Return value:  Size  Location     Type
   902 ;;                  1    wreg      void 
   903 ;; Registers used:
   904 ;;		wreg, status,2, status,0, prodl, prodh, cstack
   905 ;; Tracked objects:
   906 ;;		On entry : 0/0
   907 ;;		On exit  : 0/0
   908 ;;		Unchanged: 0/0
   909 ;; Data sizes:     COMRAM   BANK0   BANK1   BANK2   BANK3   BANK4   BANK5
   910 ;;      Params:         0      18       0       0       0       0       0
   911 ;;      Locals:         0       8       0       0       0       0       0
   912 ;;      Temps:          2       0       0       0       0       0       0
   913 ;;      Totals:         2      26       0       0       0       0       0
   914 ;;Total ram usage:       28 bytes
   915 ;; Hardware stack levels used: 1
   916 ;; Hardware stack levels required when called: 3
   917 ;; This function calls:
   918 ;;		___fldiv
   919 ;;		___flmul
   920 ;;		___fltol
   921 ;; This function is called by:
   922 ;;		_main
   923 ;; This function uses a non-reentrant model
   924 ;;
   925                           
   926                           	psect	text3
   927  001488                     __ptext3:
   928                           	callstack 0
   929  001488                     _setPWM:
   930                           	callstack 0
   931  001488  FFFF               	dw	65535	; assembler added errata NOP
   932  00148A                     
   933                           ;mainTx.c: 103: void setPWM(float period_pwm, float pwm_duty, float freq_osc, float pres
      +                          c, int module);mainTx.c: 104: {;mainTx.c: 128:     switch(module){
   934  00148A  EFD5  F00B         	goto	l2657
   935  00148E                     l2583:
   936  00148E  FFFF               	dw	65535	; assembler added errata NOP
   937                           
   938                           ;mainTx.c: 131:             mask = 0x03;
   939  001490  0E00               	movlw	0
   940  001492  6E6D               	movwf	(_mask+1)^0,c
   941  001494  0E03               	movlw	3
   942  001496  6E6C               	movwf	_mask^0,c
   943  001498                     
   944                           ;mainTx.c: 132:             pwm_p = period_pwm;
   945  001498  C0AA  F0A6         	movff	setPWM@period_pwm,_pwm_p
   946  00149C  C0AB  F0A7         	movff	setPWM@period_pwm+1,_pwm_p+1
   947  0014A0  C0AC  F0A8         	movff	setPWM@period_pwm+2,_pwm_p+2
   948  0014A4  C0AD  F0A9         	movff	setPWM@period_pwm+3,_pwm_p+3
   949  0014A8                     
   950                           ;mainTx.c: 133:             frec_osc = freq_osc;
   951  0014A8  C0B2  F0A2         	movff	setPWM@freq_osc,_frec_osc
   952  0014AC  C0B3  F0A3         	movff	setPWM@freq_osc+1,_frec_osc+1
   953  0014B0  C0B4  F0A4         	movff	setPWM@freq_osc+2,_frec_osc+2
   954  0014B4  C0B5  F0A5         	movff	setPWM@freq_osc+3,_frec_osc+3
   955  0014B8                     
   956                           ;mainTx.c: 134:             tmr2_presc = presc;
   957  0014B8  C0B6  F09E         	movff	setPWM@presc,_tmr2_presc
   958  0014BC  C0B7  F09F         	movff	setPWM@presc+1,_tmr2_presc+1
   959  0014C0  C0B8  F0A0         	movff	setPWM@presc+2,_tmr2_presc+2
   960  0014C4  C0B9  F0A1         	movff	setPWM@presc+3,_tmr2_presc+3
   961  0014C8                     
   962                           ;mainTx.c: 144:             duty_temp = (unsigned int) (((pwm_duty * period_pwm) / 100) 
      +                          / ((1 / freq_osc) * presc));
   963  0014C8  C0B6  F02C         	movff	setPWM@presc,___flmul@a
   964  0014CC  C0B7  F02D         	movff	setPWM@presc+1,___flmul@a+1
   965  0014D0  C0B8  F02E         	movff	setPWM@presc+2,___flmul@a+2
   966  0014D4  C0B9  F02F         	movff	setPWM@presc+3,___flmul@a+3
   967  0014D8  C0B2  F013         	movff	setPWM@freq_osc,___fldiv@a
   968  0014DC  C0B3  F014         	movff	setPWM@freq_osc+1,___fldiv@a+1
   969  0014E0  C0B4  F015         	movff	setPWM@freq_osc+2,___fldiv@a+2
   970  0014E4  C0B5  F016         	movff	setPWM@freq_osc+3,___fldiv@a+3
   971  0014E8  0E00               	movlw	0
   972  0014EA  6E0F               	movwf	___fldiv@b^0,c
   973  0014EC  0E00               	movlw	0
   974  0014EE  6E10               	movwf	(___fldiv@b+1)^0,c
   975  0014F0  0E80               	movlw	128
   976  0014F2  6E11               	movwf	(___fldiv@b+2)^0,c
   977  0014F4  0E3F               	movlw	63
   978  0014F6  6E12               	movwf	(___fldiv@b+3)^0,c
   979  0014F8  EC2B  F008         	call	___fldiv	;wreg free
   980  0014FC  C00F  F028         	movff	?___fldiv,___flmul@b
   981  001500  C010  F029         	movff	?___fldiv+1,___flmul@b+1
   982  001504  C011  F02A         	movff	?___fldiv+2,___flmul@b+2
   983  001508  C012  F02B         	movff	?___fldiv+3,___flmul@b+3
   984  00150C  ECD9  F005         	call	___flmul	;wreg free
   985  001510  C028  F0BC         	movff	?___flmul,_setPWM$1410
   986  001514  C029  F0BD         	movff	?___flmul+1,_setPWM$1410+1
   987  001518  C02A  F0BE         	movff	?___flmul+2,_setPWM$1410+2
   988  00151C  C02B  F0BF         	movff	?___flmul+3,_setPWM$1410+3
   989  001520                     
   990                           ;mainTx.c: 144:             duty_temp = (unsigned int) (((pwm_duty * period_pwm) / 100) 
      +                          / ((1 / freq_osc) * presc));
   991  001520  0E00               	movlw	0
   992  001522  6E13               	movwf	___fldiv@a^0,c
   993  001524  0E00               	movlw	0
   994  001526  6E14               	movwf	(___fldiv@a+1)^0,c
   995  001528  0EC8               	movlw	200
   996  00152A  6E15               	movwf	(___fldiv@a+2)^0,c
   997  00152C  0E42               	movlw	66
   998  00152E  6E16               	movwf	(___fldiv@a+3)^0,c
   999  001530  C0AA  F02C         	movff	setPWM@period_pwm,___flmul@a
  1000  001534  C0AB  F02D         	movff	setPWM@period_pwm+1,___flmul@a+1
  1001  001538  C0AC  F02E         	movff	setPWM@period_pwm+2,___flmul@a+2
  1002  00153C  C0AD  F02F         	movff	setPWM@period_pwm+3,___flmul@a+3
  1003  001540  C0AE  F028         	movff	setPWM@pwm_duty,___flmul@b
  1004  001544  C0AF  F029         	movff	setPWM@pwm_duty+1,___flmul@b+1
  1005  001548  C0B0  F02A         	movff	setPWM@pwm_duty+2,___flmul@b+2
  1006  00154C  C0B1  F02B         	movff	setPWM@pwm_duty+3,___flmul@b+3
  1007  001550  ECD9  F005         	call	___flmul	;wreg free
  1008  001554  C028  F00F         	movff	?___flmul,___fldiv@b
  1009  001558  C029  F010         	movff	?___flmul+1,___fldiv@b+1
  1010  00155C  C02A  F011         	movff	?___flmul+2,___fldiv@b+2
  1011  001560  C02B  F012         	movff	?___flmul+3,___fldiv@b+3
  1012  001564  EC2B  F008         	call	___fldiv	;wreg free
  1013  001568  C00F  F0C0         	movff	?___fldiv,_setPWM$1411
  1014  00156C  C010  F0C1         	movff	?___fldiv+1,_setPWM$1411+1
  1015  001570  C011  F0C2         	movff	?___fldiv+2,_setPWM$1411+2
  1016  001574  C012  F0C3         	movff	?___fldiv+3,_setPWM$1411+3
  1017  001578                     
  1018                           ;mainTx.c: 144:             duty_temp = (unsigned int) (((pwm_duty * period_pwm) / 100) 
      +                          / ((1 / freq_osc) * presc));
  1019  001578  C0BC  F013         	movff	_setPWM$1410,___fldiv@a
  1020  00157C  C0BD  F014         	movff	_setPWM$1410+1,___fldiv@a+1
  1021  001580  C0BE  F015         	movff	_setPWM$1410+2,___fldiv@a+2
  1022  001584  C0BF  F016         	movff	_setPWM$1410+3,___fldiv@a+3
  1023  001588  C0C0  F00F         	movff	_setPWM$1411,___fldiv@b
  1024  00158C  C0C1  F010         	movff	_setPWM$1411+1,___fldiv@b+1
  1025  001590  C0C2  F011         	movff	_setPWM$1411+2,___fldiv@b+2
  1026  001594  C0C3  F012         	movff	_setPWM$1411+3,___fldiv@b+3
  1027  001598  EC2B  F008         	call	___fldiv	;wreg free
  1028  00159C  C00F  F051         	movff	?___fldiv,___fltol@f1
  1029  0015A0  C010  F052         	movff	?___fldiv+1,___fltol@f1+1
  1030  0015A4  C011  F053         	movff	?___fldiv+2,___fltol@f1+2
  1031  0015A8  C012  F054         	movff	?___fldiv+3,___fltol@f1+3
  1032  0015AC  EC8B  F00C         	call	___fltol	;wreg free
  1033  0015B0  C051  F061         	movff	?___fltol,_duty_temp
  1034  0015B4  C052  F062         	movff	?___fltol+1,_duty_temp+1
  1035  0015B8                     
  1036                           ;mainTx.c: 145:             mask &= duty_temp;
  1037  0015B8  5061               	movf	_duty_temp^0,w,c
  1038  0015BA  166C               	andwf	_mask^0,f,c
  1039  0015BC  5062               	movf	(_duty_temp+1)^0,w,c
  1040  0015BE  166D               	andwf	(_mask+1)^0,f,c
  1041  0015C0                     
  1042                           ;mainTx.c: 146:             mask = mask << 4;
  1043  0015C0  C06C  F05B         	movff	_mask,??_setPWM
  1044  0015C4  C06D  F05C         	movff	_mask+1,??_setPWM+1
  1045  0015C8  3A5B               	swapf	??_setPWM^0,f,c
  1046  0015CA  3A5C               	swapf	(??_setPWM+1)^0,f,c
  1047  0015CC  0EF0               	movlw	240
  1048  0015CE  165C               	andwf	(??_setPWM+1)^0,f,c
  1049  0015D0  505B               	movf	??_setPWM^0,w,c
  1050  0015D2  0B0F               	andlw	15
  1051  0015D4  125C               	iorwf	(??_setPWM+1)^0,f,c
  1052  0015D6  0EF0               	movlw	240
  1053  0015D8  165B               	andwf	??_setPWM^0,f,c
  1054  0015DA  C05B  F06C         	movff	??_setPWM,_mask
  1055  0015DE  C05C  F06D         	movff	??_setPWM+1,_mask+1
  1056  0015E2                     
  1057                           ;mainTx.c: 147:             CCP1CON |= mask;
  1058  0015E2  506C               	movf	_mask^0,w,c	;volatile
  1059  0015E4  12BD               	iorwf	189,f,c	;volatile
  1060  0015E6                     
  1061                           ;mainTx.c: 149:             CCPR1L = duty_temp >> 2;
  1062  0015E6  C061  F05B         	movff	_duty_temp,??_setPWM
  1063  0015EA  C062  F05C         	movff	_duty_temp+1,??_setPWM+1
  1064  0015EE  90D8               	bcf	status,0,c
  1065  0015F0  325C               	rrcf	(??_setPWM+1)^0,f,c
  1066  0015F2  325B               	rrcf	??_setPWM^0,f,c
  1067  0015F4  90D8               	bcf	status,0,c
  1068  0015F6  325C               	rrcf	(??_setPWM+1)^0,f,c
  1069  0015F8  325B               	rrcf	??_setPWM^0,f,c
  1070  0015FA  505B               	movf	??_setPWM^0,w,c
  1071  0015FC  6EBE               	movwf	190,c	;volatile
  1072  0015FE                     
  1073                           ;mainTx.c: 151:             valor_prueba_debug = 0x00;
  1074  0015FE  0E00               	movlw	0
  1075  001600  6E66               	movwf	_valor_prueba_debug^0,c
  1076  001602                     
  1077                           ;mainTx.c: 152:             valor_prueba_debug2 = 0x00;
  1078  001602  0E00               	movlw	0
  1079  001604  6E65               	movwf	_valor_prueba_debug2^0,c
  1080  001606                     
  1081                           ;mainTx.c: 154:             valor_prueba_debug |= CCP1CON;
  1082  001606  50BD               	movf	189,w,c	;volatile
  1083  001608  1266               	iorwf	_valor_prueba_debug^0,f,c
  1084  00160A                     
  1085                           ;mainTx.c: 155:             valor_prueba_debug2 |= CCPR1L;
  1086  00160A  50BE               	movf	190,w,c	;volatile
  1087  00160C  1265               	iorwf	_valor_prueba_debug2^0,f,c
  1088  00160E                     
  1089                           ;mainTx.c: 158:             TRISCbits.RC2 = 0;
  1090  00160E  9494               	bcf	148,2,c	;volatile
  1091  001610                     
  1092                           ;mainTx.c: 163:             T2CON = 0x07;
  1093  001610  0E07               	movlw	7
  1094  001612  6ECA               	movwf	202,c	;volatile
  1095  001614                     
  1096                           ;mainTx.c: 166:             CCP1CON |= 0x0F;
  1097  001614  0E0F               	movlw	15
  1098  001616  12BD               	iorwf	189,f,c	;volatile
  1099                           
  1100                           ;mainTx.c: 167:             break;
  1101  001618  EFED  F00B         	goto	l118
  1102  00161C                     l2619:
  1103  00161C  FFFF               	dw	65535	; assembler added errata NOP
  1104                           
  1105                           ;mainTx.c: 169:             mask = 0x03;
  1106  00161E  0E00               	movlw	0
  1107  001620  6E6D               	movwf	(_mask+1)^0,c
  1108  001622  0E03               	movlw	3
  1109  001624  6E6C               	movwf	_mask^0,c
  1110  001626                     
  1111                           ;mainTx.c: 170:             pwm_p = period_pwm;
  1112  001626  C0AA  F0A6         	movff	setPWM@period_pwm,_pwm_p
  1113  00162A  C0AB  F0A7         	movff	setPWM@period_pwm+1,_pwm_p+1
  1114  00162E  C0AC  F0A8         	movff	setPWM@period_pwm+2,_pwm_p+2
  1115  001632  C0AD  F0A9         	movff	setPWM@period_pwm+3,_pwm_p+3
  1116  001636                     
  1117                           ;mainTx.c: 171:             frec_osc = freq_osc;
  1118  001636  C0B2  F0A2         	movff	setPWM@freq_osc,_frec_osc
  1119  00163A  C0B3  F0A3         	movff	setPWM@freq_osc+1,_frec_osc+1
  1120  00163E  C0B4  F0A4         	movff	setPWM@freq_osc+2,_frec_osc+2
  1121  001642  C0B5  F0A5         	movff	setPWM@freq_osc+3,_frec_osc+3
  1122  001646                     
  1123                           ;mainTx.c: 172:             tmr2_presc = presc;
  1124  001646  C0B6  F09E         	movff	setPWM@presc,_tmr2_presc
  1125  00164A  C0B7  F09F         	movff	setPWM@presc+1,_tmr2_presc+1
  1126  00164E  C0B8  F0A0         	movff	setPWM@presc+2,_tmr2_presc+2
  1127  001652  C0B9  F0A1         	movff	setPWM@presc+3,_tmr2_presc+3
  1128  001656                     
  1129                           ;mainTx.c: 182:             duty_temp = (unsigned int) (((pwm_duty * period_pwm) / 100) 
      +                          / ((1 / freq_osc) * presc));
  1130  001656  C0B6  F02C         	movff	setPWM@presc,___flmul@a
  1131  00165A  C0B7  F02D         	movff	setPWM@presc+1,___flmul@a+1
  1132  00165E  C0B8  F02E         	movff	setPWM@presc+2,___flmul@a+2
  1133  001662  C0B9  F02F         	movff	setPWM@presc+3,___flmul@a+3
  1134  001666  C0B2  F013         	movff	setPWM@freq_osc,___fldiv@a
  1135  00166A  C0B3  F014         	movff	setPWM@freq_osc+1,___fldiv@a+1
  1136  00166E  C0B4  F015         	movff	setPWM@freq_osc+2,___fldiv@a+2
  1137  001672  C0B5  F016         	movff	setPWM@freq_osc+3,___fldiv@a+3
  1138  001676  0E00               	movlw	0
  1139  001678  6E0F               	movwf	___fldiv@b^0,c
  1140  00167A  0E00               	movlw	0
  1141  00167C  6E10               	movwf	(___fldiv@b+1)^0,c
  1142  00167E  0E80               	movlw	128
  1143  001680  6E11               	movwf	(___fldiv@b+2)^0,c
  1144  001682  0E3F               	movlw	63
  1145  001684  6E12               	movwf	(___fldiv@b+3)^0,c
  1146  001686  EC2B  F008         	call	___fldiv	;wreg free
  1147  00168A  C00F  F028         	movff	?___fldiv,___flmul@b
  1148  00168E  C010  F029         	movff	?___fldiv+1,___flmul@b+1
  1149  001692  C011  F02A         	movff	?___fldiv+2,___flmul@b+2
  1150  001696  C012  F02B         	movff	?___fldiv+3,___flmul@b+3
  1151  00169A  ECD9  F005         	call	___flmul	;wreg free
  1152  00169E  C028  F0BC         	movff	?___flmul,_setPWM$1410
  1153  0016A2  C029  F0BD         	movff	?___flmul+1,_setPWM$1410+1
  1154  0016A6  C02A  F0BE         	movff	?___flmul+2,_setPWM$1410+2
  1155  0016AA  C02B  F0BF         	movff	?___flmul+3,_setPWM$1410+3
  1156  0016AE                     
  1157                           ;mainTx.c: 182:             duty_temp = (unsigned int) (((pwm_duty * period_pwm) / 100) 
      +                          / ((1 / freq_osc) * presc));
  1158  0016AE  0E00               	movlw	0
  1159  0016B0  6E13               	movwf	___fldiv@a^0,c
  1160  0016B2  0E00               	movlw	0
  1161  0016B4  6E14               	movwf	(___fldiv@a+1)^0,c
  1162  0016B6  0EC8               	movlw	200
  1163  0016B8  6E15               	movwf	(___fldiv@a+2)^0,c
  1164  0016BA  0E42               	movlw	66
  1165  0016BC  6E16               	movwf	(___fldiv@a+3)^0,c
  1166  0016BE  C0AA  F02C         	movff	setPWM@period_pwm,___flmul@a
  1167  0016C2  C0AB  F02D         	movff	setPWM@period_pwm+1,___flmul@a+1
  1168  0016C6  C0AC  F02E         	movff	setPWM@period_pwm+2,___flmul@a+2
  1169  0016CA  C0AD  F02F         	movff	setPWM@period_pwm+3,___flmul@a+3
  1170  0016CE  C0AE  F028         	movff	setPWM@pwm_duty,___flmul@b
  1171  0016D2  C0AF  F029         	movff	setPWM@pwm_duty+1,___flmul@b+1
  1172  0016D6  C0B0  F02A         	movff	setPWM@pwm_duty+2,___flmul@b+2
  1173  0016DA  C0B1  F02B         	movff	setPWM@pwm_duty+3,___flmul@b+3
  1174  0016DE  ECD9  F005         	call	___flmul	;wreg free
  1175  0016E2  C028  F00F         	movff	?___flmul,___fldiv@b
  1176  0016E6  C029  F010         	movff	?___flmul+1,___fldiv@b+1
  1177  0016EA  C02A  F011         	movff	?___flmul+2,___fldiv@b+2
  1178  0016EE  C02B  F012         	movff	?___flmul+3,___fldiv@b+3
  1179  0016F2  EC2B  F008         	call	___fldiv	;wreg free
  1180  0016F6  C00F  F0C0         	movff	?___fldiv,_setPWM$1411
  1181  0016FA  C010  F0C1         	movff	?___fldiv+1,_setPWM$1411+1
  1182  0016FE  C011  F0C2         	movff	?___fldiv+2,_setPWM$1411+2
  1183  001702  C012  F0C3         	movff	?___fldiv+3,_setPWM$1411+3
  1184  001706                     
  1185                           ;mainTx.c: 182:             duty_temp = (unsigned int) (((pwm_duty * period_pwm) / 100) 
      +                          / ((1 / freq_osc) * presc));
  1186  001706  C0BC  F013         	movff	_setPWM$1410,___fldiv@a
  1187  00170A  C0BD  F014         	movff	_setPWM$1410+1,___fldiv@a+1
  1188  00170E  C0BE  F015         	movff	_setPWM$1410+2,___fldiv@a+2
  1189  001712  C0BF  F016         	movff	_setPWM$1410+3,___fldiv@a+3
  1190  001716  C0C0  F00F         	movff	_setPWM$1411,___fldiv@b
  1191  00171A  C0C1  F010         	movff	_setPWM$1411+1,___fldiv@b+1
  1192  00171E  C0C2  F011         	movff	_setPWM$1411+2,___fldiv@b+2
  1193  001722  C0C3  F012         	movff	_setPWM$1411+3,___fldiv@b+3
  1194  001726  EC2B  F008         	call	___fldiv	;wreg free
  1195  00172A  C00F  F051         	movff	?___fldiv,___fltol@f1
  1196  00172E  C010  F052         	movff	?___fldiv+1,___fltol@f1+1
  1197  001732  C011  F053         	movff	?___fldiv+2,___fltol@f1+2
  1198  001736  C012  F054         	movff	?___fldiv+3,___fltol@f1+3
  1199  00173A  EC8B  F00C         	call	___fltol	;wreg free
  1200  00173E  C051  F061         	movff	?___fltol,_duty_temp
  1201  001742  C052  F062         	movff	?___fltol+1,_duty_temp+1
  1202  001746                     
  1203                           ;mainTx.c: 183:             mask &= duty_temp;
  1204  001746  5061               	movf	_duty_temp^0,w,c
  1205  001748  166C               	andwf	_mask^0,f,c
  1206  00174A  5062               	movf	(_duty_temp+1)^0,w,c
  1207  00174C  166D               	andwf	(_mask+1)^0,f,c
  1208  00174E                     
  1209                           ;mainTx.c: 184:             mask = mask << 4;
  1210  00174E  C06C  F05B         	movff	_mask,??_setPWM
  1211  001752  C06D  F05C         	movff	_mask+1,??_setPWM+1
  1212  001756  3A5B               	swapf	??_setPWM^0,f,c
  1213  001758  3A5C               	swapf	(??_setPWM+1)^0,f,c
  1214  00175A  0EF0               	movlw	240
  1215  00175C  165C               	andwf	(??_setPWM+1)^0,f,c
  1216  00175E  505B               	movf	??_setPWM^0,w,c
  1217  001760  0B0F               	andlw	15
  1218  001762  125C               	iorwf	(??_setPWM+1)^0,f,c
  1219  001764  0EF0               	movlw	240
  1220  001766  165B               	andwf	??_setPWM^0,f,c
  1221  001768  C05B  F06C         	movff	??_setPWM,_mask
  1222  00176C  C05C  F06D         	movff	??_setPWM+1,_mask+1
  1223  001770                     
  1224                           ;mainTx.c: 185:             CCP2CON |= mask;
  1225  001770  506C               	movf	_mask^0,w,c	;volatile
  1226  001772  12BA               	iorwf	186,f,c	;volatile
  1227  001774                     
  1228                           ;mainTx.c: 187:             CCPR2L = duty_temp >> 2;
  1229  001774  C061  F05B         	movff	_duty_temp,??_setPWM
  1230  001778  C062  F05C         	movff	_duty_temp+1,??_setPWM+1
  1231  00177C  90D8               	bcf	status,0,c
  1232  00177E  325C               	rrcf	(??_setPWM+1)^0,f,c
  1233  001780  325B               	rrcf	??_setPWM^0,f,c
  1234  001782  90D8               	bcf	status,0,c
  1235  001784  325C               	rrcf	(??_setPWM+1)^0,f,c
  1236  001786  325B               	rrcf	??_setPWM^0,f,c
  1237  001788  505B               	movf	??_setPWM^0,w,c
  1238  00178A  6EBB               	movwf	187,c	;volatile
  1239  00178C                     
  1240                           ;mainTx.c: 191:             valor_prueba_debug = 0x00;
  1241  00178C  0E00               	movlw	0
  1242  00178E  6E66               	movwf	_valor_prueba_debug^0,c
  1243  001790                     
  1244                           ;mainTx.c: 192:             valor_prueba_debug2 = 0x00;
  1245  001790  0E00               	movlw	0
  1246  001792  6E65               	movwf	_valor_prueba_debug2^0,c
  1247  001794                     
  1248                           ;mainTx.c: 194:             valor_prueba_debug |= CCP2CON;
  1249  001794  50BA               	movf	186,w,c	;volatile
  1250  001796  1266               	iorwf	_valor_prueba_debug^0,f,c
  1251  001798                     
  1252                           ;mainTx.c: 195:             valor_prueba_debug2 |= CCPR2L;
  1253  001798  50BB               	movf	187,w,c	;volatile
  1254  00179A  1265               	iorwf	_valor_prueba_debug2^0,f,c
  1255  00179C                     
  1256                           ;mainTx.c: 199:             TRISBbits.RB3 = 0;
  1257  00179C  9693               	bcf	147,3,c	;volatile
  1258  00179E                     
  1259                           ;mainTx.c: 204:             T2CON = 0x07;
  1260  00179E  0E07               	movlw	7
  1261  0017A0  6ECA               	movwf	202,c	;volatile
  1262  0017A2                     
  1263                           ;mainTx.c: 207:             CCP2CON |= 0x0F;
  1264  0017A2  0E0F               	movlw	15
  1265  0017A4  12BA               	iorwf	186,f,c	;volatile
  1266                           
  1267                           ;mainTx.c: 208:             break;
  1268  0017A6  EFED  F00B         	goto	l118
  1269  0017AA                     l2657:
  1270  0017AA  FFFF               	dw	65535	; assembler added errata NOP
  1271  0017AC  C0BA  F05B         	movff	setPWM@module,??_setPWM
  1272  0017B0  C0BB  F05C         	movff	setPWM@module+1,??_setPWM+1
  1273                           
  1274                           ; Switch on 2 bytes has been partitioned into a top level switch of size 1, and 1 sub-sw
      +                          itches
  1275                           ; Switch size 1, requested type "simple"
  1276                           ; Number of cases is 1, Range of values is 0 to 0
  1277                           ; switch strategies available:
  1278                           ; Name         Instructions Cycles
  1279                           ; simple_byte            4     3 (average)
  1280                           ;	Chosen strategy is simple_byte
  1281  0017B4  505C               	movf	(??_setPWM+1)^0,w,c
  1282  0017B6  0A00               	xorlw	0	; case 0
  1283  0017B8  B4D8               	btfsc	status,2,c
  1284  0017BA  EFE1  F00B         	goto	l2719
  1285  0017BE  EFED  F00B         	goto	l118
  1286  0017C2                     l2719:
  1287  0017C2  FFFF               	dw	65535	; assembler added errata NOP
  1288                           
  1289                           ; Switch size 1, requested type "simple"
  1290                           ; Number of cases is 2, Range of values is 1 to 2
  1291                           ; switch strategies available:
  1292                           ; Name         Instructions Cycles
  1293                           ; simple_byte            7     4 (average)
  1294                           ;	Chosen strategy is simple_byte
  1295  0017C4  505B               	movf	??_setPWM^0,w,c
  1296  0017C6  0A01               	xorlw	1	; case 1
  1297  0017C8  B4D8               	btfsc	status,2,c
  1298  0017CA  EF47  F00A         	goto	l2583
  1299  0017CE  0A03               	xorlw	3	; case 2
  1300  0017D0  B4D8               	btfsc	status,2,c
  1301  0017D2  EF0E  F00B         	goto	l2619
  1302  0017D6  EFED  F00B         	goto	l118
  1303  0017DA                     l118:
  1304  0017DA  FFFF               	dw	65535	; assembler added errata NOP
  1305  0017DC  0012               	return		;funcret
  1306  0017DE  FFFF               	dw	65535	; errata NOP
  1307  0017E0                     __end_of_setPWM:
  1308                           	callstack 0
  1309                           
  1310 ;; *************** function _boot *****************
  1311 ;; Defined at:
  1312 ;;		line 303 in file "mainTx.c"
  1313 ;; Parameters:    Size  Location     Type
  1314 ;;		None
  1315 ;; Auto vars:     Size  Location     Type
  1316 ;;		None
  1317 ;; Return value:  Size  Location     Type
  1318 ;;                  1    wreg      void 
  1319 ;; Registers used:
  1320 ;;		wreg, status,2, status,0, prodl, prodh, cstack
  1321 ;; Tracked objects:
  1322 ;;		On entry : 0/0
  1323 ;;		On exit  : 0/0
  1324 ;;		Unchanged: 0/0
  1325 ;; Data sizes:     COMRAM   BANK0   BANK1   BANK2   BANK3   BANK4   BANK5
  1326 ;;      Params:         0       0       0       0       0       0       0
  1327 ;;      Locals:         0       0       0       0       0       0       0
  1328 ;;      Temps:          0       0       0       0       0       0       0
  1329 ;;      Totals:         0       0       0       0       0       0       0
  1330 ;;Total ram usage:        0 bytes
  1331 ;; Hardware stack levels used: 1
  1332 ;; Hardware stack levels required when called: 4
  1333 ;; This function calls:
  1334 ;;		_I2C_Master_Init
  1335 ;;		_globalPWM
  1336 ;;		_init_interrupts
  1337 ;;		_init_uart
  1338 ;; This function is called by:
  1339 ;;		_main
  1340 ;; This function uses a non-reentrant model
  1341 ;;
  1342                           
  1343                           	psect	text4
  1344  001D52                     __ptext4:
  1345                           	callstack 0
  1346  001D52                     _boot:
  1347                           	callstack 0
  1348  001D52  FFFF               	dw	65535	; assembler added errata NOP
  1349  001D54                     
  1350                           ;mainTx.c: 304:     init_interrupts();
  1351  001D54  EC7C  F00F         	call	_init_interrupts	;wreg free
  1352  001D58                     
  1353                           ;mainTx.c: 305:     init_uart();
  1354  001D58  EC61  F00F         	call	_init_uart	;wreg free
  1355  001D5C                     
  1356                           ;mainTx.c: 306:     I2C_Master_Init();
  1357  001D5C  EC6F  F00F         	call	_I2C_Master_Init	;wreg free
  1358  001D60                     
  1359                           ;mainTx.c: 307:     globalPWM(1e0/2e3, 16e6, 16e0);
  1360  001D60  0E6F               	movlw	111
  1361  001D62  0100               	movlb	0	; () banked
  1362  001D64  6FAA               	movwf	globalPWM@period_pwm& (0+255),b
  1363  001D66  0E12               	movlw	18
  1364  001D68  6FAB               	movwf	(globalPWM@period_pwm+1)& (0+255),b
  1365  001D6A  0E03               	movlw	3
  1366  001D6C  6FAC               	movwf	(globalPWM@period_pwm+2)& (0+255),b
  1367  001D6E  0E3A               	movlw	58
  1368  001D70  6FAD               	movwf	(globalPWM@period_pwm+3)& (0+255),b
  1369  001D72  0E00               	movlw	0
  1370  001D74  6FAE               	movwf	globalPWM@freq_osc& (0+255),b
  1371  001D76  0E24               	movlw	36
  1372  001D78  6FAF               	movwf	(globalPWM@freq_osc+1)& (0+255),b
  1373  001D7A  0E74               	movlw	116
  1374  001D7C  6FB0               	movwf	(globalPWM@freq_osc+2)& (0+255),b
  1375  001D7E  0E4B               	movlw	75
  1376  001D80  6FB1               	movwf	(globalPWM@freq_osc+3)& (0+255),b
  1377  001D82  0E00               	movlw	0
  1378  001D84  6FB2               	movwf	globalPWM@presc& (0+255),b
  1379  001D86  0E00               	movlw	0
  1380  001D88  6FB3               	movwf	(globalPWM@presc+1)& (0+255),b
  1381  001D8A  0E80               	movlw	128
  1382  001D8C  6FB4               	movwf	(globalPWM@presc+2)& (0+255),b
  1383  001D8E  0E41               	movlw	65
  1384  001D90  6FB5               	movwf	(globalPWM@presc+3)& (0+255),b
  1385  001D92  ECA3  F00D         	call	_globalPWM	;wreg free
  1386  001D96                     
  1387                           ;mainTx.c: 310:     ADCON1 = 0x06;
  1388  001D96  0E06               	movlw	6
  1389  001D98  6EC1               	movwf	193,c	;volatile
  1390  001D9A                     
  1391                           ;mainTx.c: 311:     TRISA = 0x00;
  1392  001D9A  0E00               	movlw	0
  1393  001D9C  6E92               	movwf	146,c	;volatile
  1394  001D9E  0012               	return		;funcret
  1395  001DA0  FFFF               	dw	65535	; errata NOP
  1396  001DA2                     __end_of_boot:
  1397                           	callstack 0
  1398                           
  1399 ;; *************** function _init_uart *****************
  1400 ;; Defined at:
  1401 ;;		line 254 in file "mainTx.c"
  1402 ;; Parameters:    Size  Location     Type
  1403 ;;		None
  1404 ;; Auto vars:     Size  Location     Type
  1405 ;;		None
  1406 ;; Return value:  Size  Location     Type
  1407 ;;                  1    wreg      void 
  1408 ;; Registers used:
  1409 ;;		wreg, status,2, cstack
  1410 ;; Tracked objects:
  1411 ;;		On entry : 0/0
  1412 ;;		On exit  : 0/0
  1413 ;;		Unchanged: 0/0
  1414 ;; Data sizes:     COMRAM   BANK0   BANK1   BANK2   BANK3   BANK4   BANK5
  1415 ;;      Params:         0       0       0       0       0       0       0
  1416 ;;      Locals:         0       0       0       0       0       0       0
  1417 ;;      Temps:          0       0       0       0       0       0       0
  1418 ;;      Totals:         0       0       0       0       0       0       0
  1419 ;;Total ram usage:        0 bytes
  1420 ;; Hardware stack levels used: 1
  1421 ;; Hardware stack levels required when called: 3
  1422 ;; This function calls:
  1423 ;;		_rx_start
  1424 ;;		_tx_start
  1425 ;; This function is called by:
  1426 ;;		_boot
  1427 ;; This function uses a non-reentrant model
  1428 ;;
  1429                           
  1430                           	psect	text5
  1431  001EC2                     __ptext5:
  1432                           	callstack 0
  1433  001EC2                     _init_uart:
  1434                           	callstack 0
  1435  001EC2  FFFF               	dw	65535	; assembler added errata NOP
  1436  001EC4                     
  1437                           ;mainTx.c: 255:     TXSTAbits.BRGH = 1;
  1438  001EC4  84AC               	bsf	172,2,c	;volatile
  1439  001EC6                     
  1440                           ;mainTx.c: 256:     SPBRG = 103;
  1441  001EC6  0E67               	movlw	103
  1442  001EC8  6EAF               	movwf	175,c	;volatile
  1443  001ECA                     
  1444                           ;mainTx.c: 258:     TXSTAbits.SYNC = 0;
  1445  001ECA  98AC               	bcf	172,4,c	;volatile
  1446  001ECC                     
  1447                           ;mainTx.c: 259:     RCSTAbits.SPEN = 1;
  1448  001ECC  8EAB               	bsf	171,7,c	;volatile
  1449  001ECE                     
  1450                           ;mainTx.c: 261:     TRISC6 = 1;
  1451  001ECE  8C94               	bsf	3988,6,c	;volatile
  1452  001ED0                     
  1453                           ;mainTx.c: 262:     TRISC7 = 1;
  1454  001ED0  8E94               	bsf	3988,7,c	;volatile
  1455  001ED2                     
  1456                           ;mainTx.c: 263:     tx_start();
  1457  001ED2  ECAE  F00F         	call	_tx_start	;wreg free
  1458  001ED6                     
  1459                           ;mainTx.c: 264:     rx_start();
  1460  001ED6  ECB2  F00F         	call	_rx_start	;wreg free
  1461  001EDA  0012               	return		;funcret
  1462  001EDC  FFFF               	dw	65535	; errata NOP
  1463  001EDE                     __end_of_init_uart:
  1464                           	callstack 0
  1465                           
  1466 ;; *************** function _tx_start *****************
  1467 ;; Defined at:
  1468 ;;		line 267 in file "mainTx.c"
  1469 ;; Parameters:    Size  Location     Type
  1470 ;;		None
  1471 ;; Auto vars:     Size  Location     Type
  1472 ;;		None
  1473 ;; Return value:  Size  Location     Type
  1474 ;;                  1    wreg      void 
  1475 ;; Registers used:
  1476 ;;		None
  1477 ;; Tracked objects:
  1478 ;;		On entry : 0/0
  1479 ;;		On exit  : 0/0
  1480 ;;		Unchanged: 0/0
  1481 ;; Data sizes:     COMRAM   BANK0   BANK1   BANK2   BANK3   BANK4   BANK5
  1482 ;;      Params:         0       0       0       0       0       0       0
  1483 ;;      Locals:         0       0       0       0       0       0       0
  1484 ;;      Temps:          0       0       0       0       0       0       0
  1485 ;;      Totals:         0       0       0       0       0       0       0
  1486 ;;Total ram usage:        0 bytes
  1487 ;; Hardware stack levels used: 1
  1488 ;; Hardware stack levels required when called: 2
  1489 ;; This function calls:
  1490 ;;		Nothing
  1491 ;; This function is called by:
  1492 ;;		_init_uart
  1493 ;; This function uses a non-reentrant model
  1494 ;;
  1495                           
  1496                           	psect	text6
  1497  001F5C                     __ptext6:
  1498                           	callstack 0
  1499  001F5C                     _tx_start:
  1500                           	callstack 0
  1501  001F5C  FFFF               	dw	65535	; assembler added errata NOP
  1502  001F5E                     
  1503                           ;mainTx.c: 268:     TXSTAbits.TXEN = 1;
  1504  001F5E  8AAC               	bsf	172,5,c	;volatile
  1505  001F60  0012               	return		;funcret
  1506  001F62  FFFF               	dw	65535	; errata NOP
  1507  001F64                     __end_of_tx_start:
  1508                           	callstack 0
  1509                           
  1510 ;; *************** function _rx_start *****************
  1511 ;; Defined at:
  1512 ;;		line 246 in file "mainTx.c"
  1513 ;; Parameters:    Size  Location     Type
  1514 ;;		None
  1515 ;; Auto vars:     Size  Location     Type
  1516 ;;		None
  1517 ;; Return value:  Size  Location     Type
  1518 ;;                  1    wreg      void 
  1519 ;; Registers used:
  1520 ;;		None
  1521 ;; Tracked objects:
  1522 ;;		On entry : 0/0
  1523 ;;		On exit  : 0/0
  1524 ;;		Unchanged: 0/0
  1525 ;; Data sizes:     COMRAM   BANK0   BANK1   BANK2   BANK3   BANK4   BANK5
  1526 ;;      Params:         0       0       0       0       0       0       0
  1527 ;;      Locals:         0       0       0       0       0       0       0
  1528 ;;      Temps:          0       0       0       0       0       0       0
  1529 ;;      Totals:         0       0       0       0       0       0       0
  1530 ;;Total ram usage:        0 bytes
  1531 ;; Hardware stack levels used: 1
  1532 ;; Hardware stack levels required when called: 2
  1533 ;; This function calls:
  1534 ;;		Nothing
  1535 ;; This function is called by:
  1536 ;;		_init_uart
  1537 ;; This function uses a non-reentrant model
  1538 ;;
  1539                           
  1540                           	psect	text7
  1541  001F64                     __ptext7:
  1542                           	callstack 0
  1543  001F64                     _rx_start:
  1544                           	callstack 0
  1545  001F64  FFFF               	dw	65535	; assembler added errata NOP
  1546  001F66                     
  1547                           ;mainTx.c: 247:     RCSTAbits.CREN = 1;
  1548  001F66  88AB               	bsf	171,4,c	;volatile
  1549  001F68  0012               	return		;funcret
  1550  001F6A  FFFF               	dw	65535	; errata NOP
  1551  001F6C                     __end_of_rx_start:
  1552                           	callstack 0
  1553                           
  1554 ;; *************** function _init_interrupts *****************
  1555 ;; Defined at:
  1556 ;;		line 221 in file "mainTx.c"
  1557 ;; Parameters:    Size  Location     Type
  1558 ;;		None
  1559 ;; Auto vars:     Size  Location     Type
  1560 ;;		None
  1561 ;; Return value:  Size  Location     Type
  1562 ;;                  1    wreg      void 
  1563 ;; Registers used:
  1564 ;;		None
  1565 ;; Tracked objects:
  1566 ;;		On entry : 0/0
  1567 ;;		On exit  : 0/0
  1568 ;;		Unchanged: 0/0
  1569 ;; Data sizes:     COMRAM   BANK0   BANK1   BANK2   BANK3   BANK4   BANK5
  1570 ;;      Params:         0       0       0       0       0       0       0
  1571 ;;      Locals:         0       0       0       0       0       0       0
  1572 ;;      Temps:          0       0       0       0       0       0       0
  1573 ;;      Totals:         0       0       0       0       0       0       0
  1574 ;;Total ram usage:        0 bytes
  1575 ;; Hardware stack levels used: 1
  1576 ;; Hardware stack levels required when called: 2
  1577 ;; This function calls:
  1578 ;;		Nothing
  1579 ;; This function is called by:
  1580 ;;		_boot
  1581 ;; This function uses a non-reentrant model
  1582 ;;
  1583                           
  1584                           	psect	text8
  1585  001EF8                     __ptext8:
  1586                           	callstack 0
  1587  001EF8                     _init_interrupts:
  1588                           	callstack 0
  1589  001EF8  FFFF               	dw	65535	; assembler added errata NOP
  1590  001EFA                     
  1591                           ;mainTx.c: 222:     RCONbits.IPEN = 0;
  1592  001EFA  9ED0               	bcf	208,7,c	;volatile
  1593                           
  1594                           ;mainTx.c: 223:     INTCONbits.GIE = 1;
  1595  001EFC  8EF2               	bsf	242,7,c	;volatile
  1596                           
  1597                           ;mainTx.c: 224:     INTCONbits.PEIE = 1;
  1598  001EFE  8CF2               	bsf	242,6,c	;volatile
  1599                           
  1600                           ;mainTx.c: 227:     PIE1bits.TXIE = 0;
  1601  001F00  989D               	bcf	157,4,c	;volatile
  1602                           
  1603                           ;mainTx.c: 228:     PIE1bits.RCIE = 1;
  1604  001F02  8A9D               	bsf	157,5,c	;volatile
  1605  001F04  0012               	return		;funcret
  1606  001F06  FFFF               	dw	65535	; errata NOP
  1607  001F08                     __end_of_init_interrupts:
  1608                           	callstack 0
  1609                           
  1610 ;; *************** function _globalPWM *****************
  1611 ;; Defined at:
  1612 ;;		line 96 in file "mainTx.c"
  1613 ;; Parameters:    Size  Location     Type
  1614 ;;  period_pwm      4    0[BANK0 ] float 
  1615 ;;  freq_osc        4    4[BANK0 ] float 
  1616 ;;  presc           4    8[BANK0 ] float 
  1617 ;; Auto vars:     Size  Location     Type
  1618 ;;		None
  1619 ;; Return value:  Size  Location     Type
  1620 ;;                  1    wreg      void 
  1621 ;; Registers used:
  1622 ;;		wreg, status,2, status,0, prodl, prodh, cstack
  1623 ;; Tracked objects:
  1624 ;;		On entry : 0/0
  1625 ;;		On exit  : 0/0
  1626 ;;		Unchanged: 0/0
  1627 ;; Data sizes:     COMRAM   BANK0   BANK1   BANK2   BANK3   BANK4   BANK5
  1628 ;;      Params:         0      12       0       0       0       0       0
  1629 ;;      Locals:         4       0       0       0       0       0       0
  1630 ;;      Temps:          0       0       0       0       0       0       0
  1631 ;;      Totals:         4      12       0       0       0       0       0
  1632 ;;Total ram usage:       16 bytes
  1633 ;; Hardware stack levels used: 1
  1634 ;; Hardware stack levels required when called: 3
  1635 ;; This function calls:
  1636 ;;		___fladd
  1637 ;;		___fldiv
  1638 ;;		___flmul
  1639 ;;		___fltol
  1640 ;; This function is called by:
  1641 ;;		_boot
  1642 ;; This function uses a non-reentrant model
  1643 ;;
  1644                           
  1645                           	psect	text9
  1646  001B46                     __ptext9:
  1647                           	callstack 0
  1648  001B46                     _globalPWM:
  1649                           	callstack 0
  1650  001B46  FFFF               	dw	65535	; assembler added errata NOP
  1651  001B48                     
  1652                           ;mainTx.c: 98:     periodo = (unsigned int) ((period_pwm / ((4 / freq_osc) * presc))-1);
  1653  001B48  C0B2  F02C         	movff	globalPWM@presc,___flmul@a
  1654  001B4C  C0B3  F02D         	movff	globalPWM@presc+1,___flmul@a+1
  1655  001B50  C0B4  F02E         	movff	globalPWM@presc+2,___flmul@a+2
  1656  001B54  C0B5  F02F         	movff	globalPWM@presc+3,___flmul@a+3
  1657  001B58  C0AE  F013         	movff	globalPWM@freq_osc,___fldiv@a
  1658  001B5C  C0AF  F014         	movff	globalPWM@freq_osc+1,___fldiv@a+1
  1659  001B60  C0B0  F015         	movff	globalPWM@freq_osc+2,___fldiv@a+2
  1660  001B64  C0B1  F016         	movff	globalPWM@freq_osc+3,___fldiv@a+3
  1661  001B68  0E00               	movlw	0
  1662  001B6A  6E0F               	movwf	___fldiv@b^0,c
  1663  001B6C  0E00               	movlw	0
  1664  001B6E  6E10               	movwf	(___fldiv@b+1)^0,c
  1665  001B70  0E80               	movlw	128
  1666  001B72  6E11               	movwf	(___fldiv@b+2)^0,c
  1667  001B74  0E40               	movlw	64
  1668  001B76  6E12               	movwf	(___fldiv@b+3)^0,c
  1669  001B78  EC2B  F008         	call	___fldiv	;wreg free
  1670  001B7C  C00F  F028         	movff	?___fldiv,___flmul@b
  1671  001B80  C010  F029         	movff	?___fldiv+1,___flmul@b+1
  1672  001B84  C011  F02A         	movff	?___fldiv+2,___flmul@b+2
  1673  001B88  C012  F02B         	movff	?___fldiv+3,___flmul@b+3
  1674  001B8C  ECD9  F005         	call	___flmul	;wreg free
  1675  001B90  C028  F05B         	movff	?___flmul,_globalPWM$1409
  1676  001B94  C029  F05C         	movff	?___flmul+1,_globalPWM$1409+1
  1677  001B98  C02A  F05D         	movff	?___flmul+2,_globalPWM$1409+2
  1678  001B9C  C02B  F05E         	movff	?___flmul+3,_globalPWM$1409+3
  1679  001BA0                     
  1680                           ;mainTx.c: 98:     periodo = (unsigned int) ((period_pwm / ((4 / freq_osc) * presc))-1);
  1681  001BA0  0E00               	movlw	0
  1682  001BA2  6E45               	movwf	___fladd@a^0,c
  1683  001BA4  0E00               	movlw	0
  1684  001BA6  6E46               	movwf	(___fladd@a+1)^0,c
  1685  001BA8  0E80               	movlw	128
  1686  001BAA  6E47               	movwf	(___fladd@a+2)^0,c
  1687  001BAC  0EBF               	movlw	191
  1688  001BAE  6E48               	movwf	(___fladd@a+3)^0,c
  1689  001BB0  C05B  F013         	movff	_globalPWM$1409,___fldiv@a
  1690  001BB4  C05C  F014         	movff	_globalPWM$1409+1,___fldiv@a+1
  1691  001BB8  C05D  F015         	movff	_globalPWM$1409+2,___fldiv@a+2
  1692  001BBC  C05E  F016         	movff	_globalPWM$1409+3,___fldiv@a+3
  1693  001BC0  C0AA  F00F         	movff	globalPWM@period_pwm,___fldiv@b
  1694  001BC4  C0AB  F010         	movff	globalPWM@period_pwm+1,___fldiv@b+1
  1695  001BC8  C0AC  F011         	movff	globalPWM@period_pwm+2,___fldiv@b+2
  1696  001BCC  C0AD  F012         	movff	globalPWM@period_pwm+3,___fldiv@b+3
  1697  001BD0  EC2B  F008         	call	___fldiv	;wreg free
  1698  001BD4  C00F  F041         	movff	?___fldiv,___fladd@b
  1699  001BD8  C010  F042         	movff	?___fldiv+1,___fladd@b+1
  1700  001BDC  C011  F043         	movff	?___fldiv+2,___fladd@b+2
  1701  001BE0  C012  F044         	movff	?___fldiv+3,___fladd@b+3
  1702  001BE4  EC05  F003         	call	___fladd	;wreg free
  1703  001BE8  C041  F051         	movff	?___fladd,___fltol@f1
  1704  001BEC  C042  F052         	movff	?___fladd+1,___fltol@f1+1
  1705  001BF0  C043  F053         	movff	?___fladd+2,___fltol@f1+2
  1706  001BF4  C044  F054         	movff	?___fladd+3,___fltol@f1+3
  1707  001BF8  EC8B  F00C         	call	___fltol	;wreg free
  1708  001BFC  C051  F069         	movff	?___fltol,_periodo
  1709  001C00  C052  F06A         	movff	?___fltol+1,_periodo+1
  1710  001C04                     
  1711                           ;mainTx.c: 99:     PR2 = periodo;
  1712  001C04  C069  FFCB         	movff	_periodo,4043	;volatile
  1713  001C08  0012               	return		;funcret
  1714  001C0A  FFFF               	dw	65535	; errata NOP
  1715  001C0C                     __end_of_globalPWM:
  1716                           	callstack 0
  1717                           
  1718 ;; *************** function ___fltol *****************
  1719 ;; Defined at:
  1720 ;;		line 43 in file "/opt/microchip/xc8/v2.36/pic/sources/c99/common/fltol.c"
  1721 ;; Parameters:    Size  Location     Type
  1722 ;;  f1              4   80[COMRAM] void 
  1723 ;; Auto vars:     Size  Location     Type
  1724 ;;  exp1            1   89[COMRAM] unsigned char 
  1725 ;;  sign1           1   88[COMRAM] unsigned char 
  1726 ;; Return value:  Size  Location     Type
  1727 ;;                  4   80[COMRAM] long 
  1728 ;; Registers used:
  1729 ;;		wreg, status,2, status,0
  1730 ;; Tracked objects:
  1731 ;;		On entry : 0/0
  1732 ;;		On exit  : 0/0
  1733 ;;		Unchanged: 0/0
  1734 ;; Data sizes:     COMRAM   BANK0   BANK1   BANK2   BANK3   BANK4   BANK5
  1735 ;;      Params:         4       0       0       0       0       0       0
  1736 ;;      Locals:         2       0       0       0       0       0       0
  1737 ;;      Temps:          4       0       0       0       0       0       0
  1738 ;;      Totals:        10       0       0       0       0       0       0
  1739 ;;Total ram usage:       10 bytes
  1740 ;; Hardware stack levels used: 1
  1741 ;; Hardware stack levels required when called: 2
  1742 ;; This function calls:
  1743 ;;		Nothing
  1744 ;; This function is called by:
  1745 ;;		_globalPWM
  1746 ;;		_setPWM
  1747 ;;		_change_duty
  1748 ;; This function uses a non-reentrant model
  1749 ;;
  1750                           
  1751                           	psect	text10
  1752  001916                     __ptext10:
  1753                           	callstack 0
  1754  001916                     ___fltol:
  1755                           	callstack 0
  1756  001916  FFFF               	dw	65535	; assembler added errata NOP
  1757  001918  3453               	rlcf	(___fltol@f1+2)^0,w,c
  1758  00191A  3454               	rlcf	(___fltol@f1+3)^0,w,c
  1759  00191C  6E5A               	movwf	___fltol@exp1^0,c
  1760  00191E  505A               	movf	___fltol@exp1^0,w,c
  1761  001920  A4D8               	btfss	status,2,c
  1762  001922  EF95  F00C         	goto	u1791
  1763  001926  EF98  F00C         	goto	u1790
  1764  00192A                     u1791:
  1765  00192A  FFFF               	dw	65535	; assembler added errata NOP
  1766  00192C  EFA4  F00C         	goto	l2335
  1767  001930                     u1790:
  1768  001930  FFFF               	dw	65535	; assembler added errata NOP
  1769  001932                     l2331:
  1770  001932  FFFF               	dw	65535	; assembler added errata NOP
  1771  001934  0E00               	movlw	0
  1772  001936  6E51               	movwf	?___fltol^0,c
  1773  001938  0E00               	movlw	0
  1774  00193A  6E52               	movwf	(?___fltol+1)^0,c
  1775  00193C  0E00               	movlw	0
  1776  00193E  6E53               	movwf	(?___fltol+2)^0,c
  1777  001940  0E00               	movlw	0
  1778  001942  6E54               	movwf	(?___fltol+3)^0,c
  1779  001944  EF23  F00D         	goto	l595
  1780  001948                     l2335:
  1781  001948  FFFF               	dw	65535	; assembler added errata NOP
  1782  00194A  C051  F055         	movff	___fltol@f1,??___fltol
  1783  00194E  C052  F056         	movff	___fltol@f1+1,??___fltol+1
  1784  001952  C053  F057         	movff	___fltol@f1+2,??___fltol+2
  1785  001956  C054  F058         	movff	___fltol@f1+3,??___fltol+3
  1786  00195A  0E20               	movlw	32
  1787  00195C  EFB6  F00C         	goto	u1800
  1788  001960                     u1805:
  1789  001960  FFFF               	dw	65535	; assembler added errata NOP
  1790  001962  90D8               	bcf	status,0,c
  1791  001964  3258               	rrcf	(??___fltol+3)^0,f,c
  1792  001966  3257               	rrcf	(??___fltol+2)^0,f,c
  1793  001968  3256               	rrcf	(??___fltol+1)^0,f,c
  1794  00196A  3255               	rrcf	??___fltol^0,f,c
  1795  00196C                     u1800:
  1796  00196C  FFFF               	dw	65535	; assembler added errata NOP
  1797  00196E  2EE8               	decfsz	wreg,f,c
  1798  001970  EFB0  F00C         	goto	u1805
  1799  001974  5055               	movf	??___fltol^0,w,c
  1800  001976  6E59               	movwf	___fltol@sign1^0,c
  1801  001978  8E53               	bsf	(___fltol@f1+2)^0,7,c
  1802  00197A  0EFF               	movlw	255
  1803  00197C  1651               	andwf	___fltol@f1^0,f,c
  1804  00197E  0EFF               	movlw	255
  1805  001980  1652               	andwf	(___fltol@f1+1)^0,f,c
  1806  001982  0EFF               	movlw	255
  1807  001984  1653               	andwf	(___fltol@f1+2)^0,f,c
  1808  001986  0E00               	movlw	0
  1809  001988  1654               	andwf	(___fltol@f1+3)^0,f,c
  1810  00198A  0E96               	movlw	150
  1811  00198C  5E5A               	subwf	___fltol@exp1^0,f,c
  1812  00198E  BE5A               	btfsc	___fltol@exp1^0,7,c
  1813  001990  EFCF  F00C         	goto	u1810
  1814  001994  EFCC  F00C         	goto	u1811
  1815  001998                     u1811:
  1816  001998  FFFF               	dw	65535	; assembler added errata NOP
  1817  00199A  EFE9  F00C         	goto	l2355
  1818  00199E                     u1810:
  1819  00199E  FFFF               	dw	65535	; assembler added errata NOP
  1820  0019A0  505A               	movf	___fltol@exp1^0,w,c
  1821  0019A2  0A80               	xorlw	128
  1822  0019A4  0F97               	addlw	151
  1823  0019A6  B0D8               	btfsc	status,0,c
  1824  0019A8  EFD8  F00C         	goto	u1821
  1825  0019AC  EFDB  F00C         	goto	u1820
  1826  0019B0                     u1821:
  1827  0019B0  FFFF               	dw	65535	; assembler added errata NOP
  1828  0019B2  EFDE  F00C         	goto	l2351
  1829  0019B6                     u1820:
  1830  0019B6  FFFF               	dw	65535	; assembler added errata NOP
  1831  0019B8  EF99  F00C         	goto	l2331
  1832  0019BC                     l2351:
  1833  0019BC  FFFF               	dw	65535	; assembler added errata NOP
  1834  0019BE  90D8               	bcf	status,0,c
  1835  0019C0  3254               	rrcf	(___fltol@f1+3)^0,f,c
  1836  0019C2  3253               	rrcf	(___fltol@f1+2)^0,f,c
  1837  0019C4  3252               	rrcf	(___fltol@f1+1)^0,f,c
  1838  0019C6  3251               	rrcf	___fltol@f1^0,f,c
  1839  0019C8  3E5A               	incfsz	___fltol@exp1^0,f,c
  1840  0019CA  EFDE  F00C         	goto	l2351
  1841  0019CE  EF07  F00D         	goto	l2365
  1842  0019D2                     l2355:
  1843  0019D2  FFFF               	dw	65535	; assembler added errata NOP
  1844  0019D4  0E1F               	movlw	31
  1845  0019D6  645A               	cpfsgt	___fltol@exp1^0,c
  1846  0019D8  EFF0  F00C         	goto	u1831
  1847  0019DC  EFF3  F00C         	goto	u1830
  1848  0019E0                     u1831:
  1849  0019E0  FFFF               	dw	65535	; assembler added errata NOP
  1850  0019E2  EFFD  F00C         	goto	l2363
  1851  0019E6                     u1830:
  1852  0019E6  FFFF               	dw	65535	; assembler added errata NOP
  1853  0019E8  EF99  F00C         	goto	l2331
  1854  0019EC                     l2361:
  1855  0019EC  FFFF               	dw	65535	; assembler added errata NOP
  1856  0019EE  90D8               	bcf	status,0,c
  1857  0019F0  3651               	rlcf	___fltol@f1^0,f,c
  1858  0019F2  3652               	rlcf	(___fltol@f1+1)^0,f,c
  1859  0019F4  3653               	rlcf	(___fltol@f1+2)^0,f,c
  1860  0019F6  3654               	rlcf	(___fltol@f1+3)^0,f,c
  1861  0019F8  065A               	decf	___fltol@exp1^0,f,c
  1862  0019FA                     l2363:
  1863  0019FA  FFFF               	dw	65535	; assembler added errata NOP
  1864  0019FC  505A               	movf	___fltol@exp1^0,w,c
  1865  0019FE  A4D8               	btfss	status,2,c
  1866  001A00  EF04  F00D         	goto	u1841
  1867  001A04  EF07  F00D         	goto	u1840
  1868  001A08                     u1841:
  1869  001A08  FFFF               	dw	65535	; assembler added errata NOP
  1870  001A0A  EFF6  F00C         	goto	l2361
  1871  001A0E                     u1840:
  1872  001A0E                     l2365:
  1873  001A0E  FFFF               	dw	65535	; assembler added errata NOP
  1874  001A10  5059               	movf	___fltol@sign1^0,w,c
  1875  001A12  B4D8               	btfsc	status,2,c
  1876  001A14  EF0E  F00D         	goto	u1851
  1877  001A18  EF11  F00D         	goto	u1850
  1878  001A1C                     u1851:
  1879  001A1C  FFFF               	dw	65535	; assembler added errata NOP
  1880  001A1E  EF1A  F00D         	goto	l2369
  1881  001A22                     u1850:
  1882  001A22  FFFF               	dw	65535	; assembler added errata NOP
  1883  001A24  1E54               	comf	(___fltol@f1+3)^0,f,c
  1884  001A26  1E53               	comf	(___fltol@f1+2)^0,f,c
  1885  001A28  1E52               	comf	(___fltol@f1+1)^0,f,c
  1886  001A2A  6C51               	negf	___fltol@f1^0,c
  1887  001A2C  0E00               	movlw	0
  1888  001A2E  2252               	addwfc	(___fltol@f1+1)^0,f,c
  1889  001A30  2253               	addwfc	(___fltol@f1+2)^0,f,c
  1890  001A32  2254               	addwfc	(___fltol@f1+3)^0,f,c
  1891  001A34                     l2369:
  1892  001A34  FFFF               	dw	65535	; assembler added errata NOP
  1893  001A36  C051  F051         	movff	___fltol@f1,?___fltol
  1894  001A3A  C052  F052         	movff	___fltol@f1+1,?___fltol+1
  1895  001A3E  C053  F053         	movff	___fltol@f1+2,?___fltol+2
  1896  001A42  C054  F054         	movff	___fltol@f1+3,?___fltol+3
  1897  001A46                     l595:
  1898  001A46  FFFF               	dw	65535	; assembler added errata NOP
  1899  001A48  0012               	return		;funcret
  1900  001A4A  FFFF               	dw	65535	; errata NOP
  1901  001A4C                     __end_of___fltol:
  1902                           	callstack 0
  1903                           
  1904 ;; *************** function ___flmul *****************
  1905 ;; Defined at:
  1906 ;;		line 8 in file "/opt/microchip/xc8/v2.36/pic/sources/c99/common/sprcmul.c"
  1907 ;; Parameters:    Size  Location     Type
  1908 ;;  b               4   39[COMRAM] long 
  1909 ;;  a               4   43[COMRAM] long 
  1910 ;; Auto vars:     Size  Location     Type
  1911 ;;  prod            4   58[COMRAM] struct .
  1912 ;;  grs             4   52[COMRAM] unsigned long 
  1913 ;;  temp            2   62[COMRAM] struct .
  1914 ;;  bexp            1   57[COMRAM] unsigned char 
  1915 ;;  aexp            1   56[COMRAM] unsigned char 
  1916 ;;  sign            1   51[COMRAM] unsigned char 
  1917 ;; Return value:  Size  Location     Type
  1918 ;;                  4   39[COMRAM] unsigned char 
  1919 ;; Registers used:
  1920 ;;		wreg, status,2, status,0, prodl, prodh
  1921 ;; Tracked objects:
  1922 ;;		On entry : 0/0
  1923 ;;		On exit  : 0/0
  1924 ;;		Unchanged: 0/0
  1925 ;; Data sizes:     COMRAM   BANK0   BANK1   BANK2   BANK3   BANK4   BANK5
  1926 ;;      Params:         8       0       0       0       0       0       0
  1927 ;;      Locals:        13       0       0       0       0       0       0
  1928 ;;      Temps:          4       0       0       0       0       0       0
  1929 ;;      Totals:        25       0       0       0       0       0       0
  1930 ;;Total ram usage:       25 bytes
  1931 ;; Hardware stack levels used: 1
  1932 ;; Hardware stack levels required when called: 2
  1933 ;; This function calls:
  1934 ;;		Nothing
  1935 ;; This function is called by:
  1936 ;;		_globalPWM
  1937 ;;		_setPWM
  1938 ;;		_change_duty
  1939 ;; This function uses a non-reentrant model
  1940 ;;
  1941                           
  1942                           	psect	text11
  1943  000BB2                     __ptext11:
  1944                           	callstack 0
  1945  000BB2                     ___flmul:
  1946                           	callstack 0
  1947  000BB2  FFFF               	dw	65535	; assembler added errata NOP
  1948  000BB4  502B               	movf	(___flmul@b+3)^0,w,c
  1949  000BB6  0B80               	andlw	128
  1950  000BB8  6E34               	movwf	___flmul@sign^0,c
  1951  000BBA  502B               	movf	(___flmul@b+3)^0,w,c
  1952  000BBC  242B               	addwf	(___flmul@b+3)^0,w,c
  1953  000BBE  6E3A               	movwf	___flmul@bexp^0,c
  1954  000BC0  AE2A               	btfss	(___flmul@b+2)^0,7,c
  1955  000BC2  EFE5  F005         	goto	u1601
  1956  000BC6  EFE8  F005         	goto	u1600
  1957  000BCA                     u1601:
  1958  000BCA  FFFF               	dw	65535	; assembler added errata NOP
  1959  000BCC  EFEA  F005         	goto	l2205
  1960  000BD0                     u1600:
  1961  000BD0  FFFF               	dw	65535	; assembler added errata NOP
  1962  000BD2  803A               	bsf	___flmul@bexp^0,0,c
  1963  000BD4                     l2205:
  1964  000BD4  FFFF               	dw	65535	; assembler added errata NOP
  1965  000BD6  503A               	movf	___flmul@bexp^0,w,c
  1966  000BD8  B4D8               	btfsc	status,2,c
  1967  000BDA  EFF1  F005         	goto	u1611
  1968  000BDE  EFF4  F005         	goto	u1610
  1969  000BE2                     u1611:
  1970  000BE2  FFFF               	dw	65535	; assembler added errata NOP
  1971  000BE4  EF0B  F006         	goto	l2213
  1972  000BE8                     u1610:
  1973  000BE8  FFFF               	dw	65535	; assembler added errata NOP
  1974  000BEA  283A               	incf	___flmul@bexp^0,w,c
  1975  000BEC  A4D8               	btfss	status,2,c
  1976  000BEE  EFFB  F005         	goto	u1621
  1977  000BF2  EFFE  F005         	goto	u1620
  1978  000BF6                     u1621:
  1979  000BF6  FFFF               	dw	65535	; assembler added errata NOP
  1980  000BF8  EF07  F006         	goto	l2211
  1981  000BFC                     u1620:
  1982  000BFC  FFFF               	dw	65535	; assembler added errata NOP
  1983  000BFE  0E00               	movlw	0
  1984  000C00  6E28               	movwf	___flmul@b^0,c
  1985  000C02  0E00               	movlw	0
  1986  000C04  6E29               	movwf	(___flmul@b+1)^0,c
  1987  000C06  0E00               	movlw	0
  1988  000C08  6E2A               	movwf	(___flmul@b+2)^0,c
  1989  000C0A  0E00               	movlw	0
  1990  000C0C  6E2B               	movwf	(___flmul@b+3)^0,c
  1991  000C0E                     l2211:
  1992  000C0E  FFFF               	dw	65535	; assembler added errata NOP
  1993  000C10  8E2A               	bsf	(___flmul@b+2)^0,7,c
  1994  000C12  EF14  F006         	goto	l2215
  1995  000C16                     l2213:
  1996  000C16  FFFF               	dw	65535	; assembler added errata NOP
  1997  000C18  0E00               	movlw	0
  1998  000C1A  6E28               	movwf	___flmul@b^0,c
  1999  000C1C  0E00               	movlw	0
  2000  000C1E  6E29               	movwf	(___flmul@b+1)^0,c
  2001  000C20  0E00               	movlw	0
  2002  000C22  6E2A               	movwf	(___flmul@b+2)^0,c
  2003  000C24  0E00               	movlw	0
  2004  000C26  6E2B               	movwf	(___flmul@b+3)^0,c
  2005  000C28                     l2215:
  2006  000C28  FFFF               	dw	65535	; assembler added errata NOP
  2007  000C2A  502F               	movf	(___flmul@a+3)^0,w,c
  2008  000C2C  0B80               	andlw	128
  2009  000C2E  1A34               	xorwf	___flmul@sign^0,f,c
  2010  000C30  502F               	movf	(___flmul@a+3)^0,w,c
  2011  000C32  242F               	addwf	(___flmul@a+3)^0,w,c
  2012  000C34  6E39               	movwf	___flmul@aexp^0,c
  2013  000C36  AE2E               	btfss	(___flmul@a+2)^0,7,c
  2014  000C38  EF20  F006         	goto	u1631
  2015  000C3C  EF23  F006         	goto	u1630
  2016  000C40                     u1631:
  2017  000C40  FFFF               	dw	65535	; assembler added errata NOP
  2018  000C42  EF25  F006         	goto	l2223
  2019  000C46                     u1630:
  2020  000C46  FFFF               	dw	65535	; assembler added errata NOP
  2021  000C48  8039               	bsf	___flmul@aexp^0,0,c
  2022  000C4A                     l2223:
  2023  000C4A  FFFF               	dw	65535	; assembler added errata NOP
  2024  000C4C  5039               	movf	___flmul@aexp^0,w,c
  2025  000C4E  B4D8               	btfsc	status,2,c
  2026  000C50  EF2C  F006         	goto	u1641
  2027  000C54  EF2F  F006         	goto	u1640
  2028  000C58                     u1641:
  2029  000C58  FFFF               	dw	65535	; assembler added errata NOP
  2030  000C5A  EF46  F006         	goto	l2231
  2031  000C5E                     u1640:
  2032  000C5E  FFFF               	dw	65535	; assembler added errata NOP
  2033  000C60  2839               	incf	___flmul@aexp^0,w,c
  2034  000C62  A4D8               	btfss	status,2,c
  2035  000C64  EF36  F006         	goto	u1651
  2036  000C68  EF39  F006         	goto	u1650
  2037  000C6C                     u1651:
  2038  000C6C  FFFF               	dw	65535	; assembler added errata NOP
  2039  000C6E  EF42  F006         	goto	l2229
  2040  000C72                     u1650:
  2041  000C72  FFFF               	dw	65535	; assembler added errata NOP
  2042  000C74  0E00               	movlw	0
  2043  000C76  6E2C               	movwf	___flmul@a^0,c
  2044  000C78  0E00               	movlw	0
  2045  000C7A  6E2D               	movwf	(___flmul@a+1)^0,c
  2046  000C7C  0E00               	movlw	0
  2047  000C7E  6E2E               	movwf	(___flmul@a+2)^0,c
  2048  000C80  0E00               	movlw	0
  2049  000C82  6E2F               	movwf	(___flmul@a+3)^0,c
  2050  000C84                     l2229:
  2051  000C84  FFFF               	dw	65535	; assembler added errata NOP
  2052  000C86  8E2E               	bsf	(___flmul@a+2)^0,7,c
  2053  000C88  EF4F  F006         	goto	l912
  2054  000C8C                     l2231:
  2055  000C8C  FFFF               	dw	65535	; assembler added errata NOP
  2056  000C8E  0E00               	movlw	0
  2057  000C90  6E2C               	movwf	___flmul@a^0,c
  2058  000C92  0E00               	movlw	0
  2059  000C94  6E2D               	movwf	(___flmul@a+1)^0,c
  2060  000C96  0E00               	movlw	0
  2061  000C98  6E2E               	movwf	(___flmul@a+2)^0,c
  2062  000C9A  0E00               	movlw	0
  2063  000C9C  6E2F               	movwf	(___flmul@a+3)^0,c
  2064  000C9E                     l912:
  2065  000C9E  FFFF               	dw	65535	; assembler added errata NOP
  2066  000CA0  5039               	movf	___flmul@aexp^0,w,c
  2067  000CA2  B4D8               	btfsc	status,2,c
  2068  000CA4  EF56  F006         	goto	u1661
  2069  000CA8  EF59  F006         	goto	u1660
  2070  000CAC                     u1661:
  2071  000CAC  FFFF               	dw	65535	; assembler added errata NOP
  2072  000CAE  EF63  F006         	goto	l2235
  2073  000CB2                     u1660:
  2074  000CB2  FFFF               	dw	65535	; assembler added errata NOP
  2075  000CB4  503A               	movf	___flmul@bexp^0,w,c
  2076  000CB6  A4D8               	btfss	status,2,c
  2077  000CB8  EF60  F006         	goto	u1671
  2078  000CBC  EF63  F006         	goto	u1670
  2079  000CC0                     u1671:
  2080  000CC0  FFFF               	dw	65535	; assembler added errata NOP
  2081  000CC2  EF6E  F006         	goto	l2239
  2082  000CC6                     u1670:
  2083  000CC6                     l2235:
  2084  000CC6  FFFF               	dw	65535	; assembler added errata NOP
  2085  000CC8  0E00               	movlw	0
  2086  000CCA  6E28               	movwf	?___flmul^0,c
  2087  000CCC  0E00               	movlw	0
  2088  000CCE  6E29               	movwf	(?___flmul+1)^0,c
  2089  000CD0  0E00               	movlw	0
  2090  000CD2  6E2A               	movwf	(?___flmul+2)^0,c
  2091  000CD4  0E00               	movlw	0
  2092  000CD6  6E2B               	movwf	(?___flmul+3)^0,c
  2093  000CD8  EF28  F008         	goto	l916
  2094  000CDC                     l2239:
  2095  000CDC  FFFF               	dw	65535	; assembler added errata NOP
  2096  000CDE  502E               	movf	(___flmul@a+2)^0,w,c
  2097  000CE0  0228               	mulwf	___flmul@b^0,c
  2098  000CE2  CFF3 F03F          	movff	prodl,___flmul@temp
  2099  000CE6  CFF4 F040          	movff	prodh,___flmul@temp+1
  2100  000CEA  503F               	movf	___flmul@temp^0,w,c
  2101  000CEC  6E35               	movwf	___flmul@grs^0,c
  2102  000CEE  6A36               	clrf	(___flmul@grs+1)^0,c
  2103  000CF0  6A37               	clrf	(___flmul@grs+2)^0,c
  2104  000CF2  6A38               	clrf	(___flmul@grs+3)^0,c
  2105  000CF4  5040               	movf	(___flmul@temp+1)^0,w,c
  2106  000CF6  6E3B               	movwf	___flmul@prod^0,c
  2107  000CF8  6A3C               	clrf	(___flmul@prod+1)^0,c
  2108  000CFA  6A3D               	clrf	(___flmul@prod+2)^0,c
  2109  000CFC  6A3E               	clrf	(___flmul@prod+3)^0,c
  2110  000CFE  502D               	movf	(___flmul@a+1)^0,w,c
  2111  000D00  0229               	mulwf	(___flmul@b+1)^0,c
  2112  000D02  CFF3 F03F          	movff	prodl,___flmul@temp
  2113  000D06  CFF4 F040          	movff	prodh,___flmul@temp+1
  2114  000D0A  503F               	movf	___flmul@temp^0,w,c
  2115  000D0C  2635               	addwf	___flmul@grs^0,f,c
  2116  000D0E  0E00               	movlw	0
  2117  000D10  2236               	addwfc	(___flmul@grs+1)^0,f,c
  2118  000D12  2237               	addwfc	(___flmul@grs+2)^0,f,c
  2119  000D14  2238               	addwfc	(___flmul@grs+3)^0,f,c
  2120  000D16  5040               	movf	(___flmul@temp+1)^0,w,c
  2121  000D18  263B               	addwf	___flmul@prod^0,f,c
  2122  000D1A  0E00               	movlw	0
  2123  000D1C  223C               	addwfc	(___flmul@prod+1)^0,f,c
  2124  000D1E  223D               	addwfc	(___flmul@prod+2)^0,f,c
  2125  000D20  223E               	addwfc	(___flmul@prod+3)^0,f,c
  2126  000D22  502C               	movf	___flmul@a^0,w,c
  2127  000D24  022A               	mulwf	(___flmul@b+2)^0,c
  2128  000D26  CFF3 F03F          	movff	prodl,___flmul@temp
  2129  000D2A  CFF4 F040          	movff	prodh,___flmul@temp+1
  2130  000D2E  503F               	movf	___flmul@temp^0,w,c
  2131  000D30  2635               	addwf	___flmul@grs^0,f,c
  2132  000D32  0E00               	movlw	0
  2133  000D34  2236               	addwfc	(___flmul@grs+1)^0,f,c
  2134  000D36  2237               	addwfc	(___flmul@grs+2)^0,f,c
  2135  000D38  2238               	addwfc	(___flmul@grs+3)^0,f,c
  2136  000D3A  5040               	movf	(___flmul@temp+1)^0,w,c
  2137  000D3C  263B               	addwf	___flmul@prod^0,f,c
  2138  000D3E  0E00               	movlw	0
  2139  000D40  223C               	addwfc	(___flmul@prod+1)^0,f,c
  2140  000D42  223D               	addwfc	(___flmul@prod+2)^0,f,c
  2141  000D44  223E               	addwfc	(___flmul@prod+3)^0,f,c
  2142  000D46  C037  F038         	movff	___flmul@grs+2,___flmul@grs+3
  2143  000D4A  C036  F037         	movff	___flmul@grs+1,___flmul@grs+2
  2144  000D4E  C035  F036         	movff	___flmul@grs,___flmul@grs+1
  2145  000D52  6A35               	clrf	___flmul@grs^0,c
  2146  000D54  502C               	movf	___flmul@a^0,w,c
  2147  000D56  0229               	mulwf	(___flmul@b+1)^0,c
  2148  000D58  CFF3 F03F          	movff	prodl,___flmul@temp
  2149  000D5C  CFF4 F040          	movff	prodh,___flmul@temp+1
  2150  000D60  503F               	movf	___flmul@temp^0,w,c
  2151  000D62  2635               	addwf	___flmul@grs^0,f,c
  2152  000D64  5040               	movf	(___flmul@temp+1)^0,w,c
  2153  000D66  2236               	addwfc	(___flmul@grs+1)^0,f,c
  2154  000D68  0E00               	movlw	0
  2155  000D6A  2237               	addwfc	(___flmul@grs+2)^0,f,c
  2156  000D6C  0E00               	movlw	0
  2157  000D6E  2238               	addwfc	(___flmul@grs+3)^0,f,c
  2158  000D70  502D               	movf	(___flmul@a+1)^0,w,c
  2159  000D72  0228               	mulwf	___flmul@b^0,c
  2160  000D74  CFF3 F03F          	movff	prodl,___flmul@temp
  2161  000D78  CFF4 F040          	movff	prodh,___flmul@temp+1
  2162  000D7C  503F               	movf	___flmul@temp^0,w,c
  2163  000D7E  2635               	addwf	___flmul@grs^0,f,c
  2164  000D80  5040               	movf	(___flmul@temp+1)^0,w,c
  2165  000D82  2236               	addwfc	(___flmul@grs+1)^0,f,c
  2166  000D84  0E00               	movlw	0
  2167  000D86  2237               	addwfc	(___flmul@grs+2)^0,f,c
  2168  000D88  0E00               	movlw	0
  2169  000D8A  2238               	addwfc	(___flmul@grs+3)^0,f,c
  2170  000D8C  C037  F038         	movff	___flmul@grs+2,___flmul@grs+3
  2171  000D90  C036  F037         	movff	___flmul@grs+1,___flmul@grs+2
  2172  000D94  C035  F036         	movff	___flmul@grs,___flmul@grs+1
  2173  000D98  6A35               	clrf	___flmul@grs^0,c
  2174  000D9A  502C               	movf	___flmul@a^0,w,c
  2175  000D9C  0228               	mulwf	___flmul@b^0,c
  2176  000D9E  CFF3 F03F          	movff	prodl,___flmul@temp
  2177  000DA2  CFF4 F040          	movff	prodh,___flmul@temp+1
  2178  000DA6  503F               	movf	___flmul@temp^0,w,c
  2179  000DA8  2635               	addwf	___flmul@grs^0,f,c
  2180  000DAA  5040               	movf	(___flmul@temp+1)^0,w,c
  2181  000DAC  2236               	addwfc	(___flmul@grs+1)^0,f,c
  2182  000DAE  0E00               	movlw	0
  2183  000DB0  2237               	addwfc	(___flmul@grs+2)^0,f,c
  2184  000DB2  0E00               	movlw	0
  2185  000DB4  2238               	addwfc	(___flmul@grs+3)^0,f,c
  2186  000DB6  502E               	movf	(___flmul@a+2)^0,w,c
  2187  000DB8  0229               	mulwf	(___flmul@b+1)^0,c
  2188  000DBA  CFF3 F03F          	movff	prodl,___flmul@temp
  2189  000DBE  CFF4 F040          	movff	prodh,___flmul@temp+1
  2190  000DC2  503F               	movf	___flmul@temp^0,w,c
  2191  000DC4  263B               	addwf	___flmul@prod^0,f,c
  2192  000DC6  5040               	movf	(___flmul@temp+1)^0,w,c
  2193  000DC8  223C               	addwfc	(___flmul@prod+1)^0,f,c
  2194  000DCA  0E00               	movlw	0
  2195  000DCC  223D               	addwfc	(___flmul@prod+2)^0,f,c
  2196  000DCE  0E00               	movlw	0
  2197  000DD0  223E               	addwfc	(___flmul@prod+3)^0,f,c
  2198  000DD2  502D               	movf	(___flmul@a+1)^0,w,c
  2199  000DD4  022A               	mulwf	(___flmul@b+2)^0,c
  2200  000DD6  CFF3 F03F          	movff	prodl,___flmul@temp
  2201  000DDA  CFF4 F040          	movff	prodh,___flmul@temp+1
  2202  000DDE  503F               	movf	___flmul@temp^0,w,c
  2203  000DE0  263B               	addwf	___flmul@prod^0,f,c
  2204  000DE2  5040               	movf	(___flmul@temp+1)^0,w,c
  2205  000DE4  223C               	addwfc	(___flmul@prod+1)^0,f,c
  2206  000DE6  0E00               	movlw	0
  2207  000DE8  223D               	addwfc	(___flmul@prod+2)^0,f,c
  2208  000DEA  0E00               	movlw	0
  2209  000DEC  223E               	addwfc	(___flmul@prod+3)^0,f,c
  2210  000DEE  502E               	movf	(___flmul@a+2)^0,w,c
  2211  000DF0  022A               	mulwf	(___flmul@b+2)^0,c
  2212  000DF2  CFF3 F03F          	movff	prodl,___flmul@temp
  2213  000DF6  CFF4 F040          	movff	prodh,___flmul@temp+1
  2214  000DFA  503F               	movf	___flmul@temp^0,w,c
  2215  000DFC  6E30               	movwf	??___flmul^0,c
  2216  000DFE  5040               	movf	(___flmul@temp+1)^0,w,c
  2217  000E00  6E31               	movwf	(??___flmul+1)^0,c
  2218  000E02  6A32               	clrf	(??___flmul+2)^0,c
  2219  000E04  6A33               	clrf	(??___flmul+3)^0,c
  2220  000E06  C032  F033         	movff	??___flmul+2,??___flmul+3
  2221  000E0A  C031  F032         	movff	??___flmul+1,??___flmul+2
  2222  000E0E  C030  F031         	movff	??___flmul,??___flmul+1
  2223  000E12  6A30               	clrf	??___flmul^0,c
  2224  000E14  5030               	movf	??___flmul^0,w,c
  2225  000E16  263B               	addwf	___flmul@prod^0,f,c
  2226  000E18  5031               	movf	(??___flmul+1)^0,w,c
  2227  000E1A  223C               	addwfc	(___flmul@prod+1)^0,f,c
  2228  000E1C  5032               	movf	(??___flmul+2)^0,w,c
  2229  000E1E  223D               	addwfc	(___flmul@prod+2)^0,f,c
  2230  000E20  5033               	movf	(??___flmul+3)^0,w,c
  2231  000E22  223E               	addwfc	(___flmul@prod+3)^0,f,c
  2232  000E24  C035  F030         	movff	___flmul@grs,??___flmul
  2233  000E28  C036  F031         	movff	___flmul@grs+1,??___flmul+1
  2234  000E2C  C037  F032         	movff	___flmul@grs+2,??___flmul+2
  2235  000E30  C038  F033         	movff	___flmul@grs+3,??___flmul+3
  2236  000E34  0E19               	movlw	25
  2237  000E36  EF23  F007         	goto	u1680
  2238  000E3A                     u1685:
  2239  000E3A  FFFF               	dw	65535	; assembler added errata NOP
  2240  000E3C  90D8               	bcf	status,0,c
  2241  000E3E  3233               	rrcf	(??___flmul+3)^0,f,c
  2242  000E40  3232               	rrcf	(??___flmul+2)^0,f,c
  2243  000E42  3231               	rrcf	(??___flmul+1)^0,f,c
  2244  000E44  3230               	rrcf	??___flmul^0,f,c
  2245  000E46                     u1680:
  2246  000E46  FFFF               	dw	65535	; assembler added errata NOP
  2247  000E48  2EE8               	decfsz	wreg,f,c
  2248  000E4A  EF1D  F007         	goto	u1685
  2249  000E4E  5030               	movf	??___flmul^0,w,c
  2250  000E50  263B               	addwf	___flmul@prod^0,f,c
  2251  000E52  5031               	movf	(??___flmul+1)^0,w,c
  2252  000E54  223C               	addwfc	(___flmul@prod+1)^0,f,c
  2253  000E56  5032               	movf	(??___flmul+2)^0,w,c
  2254  000E58  223D               	addwfc	(___flmul@prod+2)^0,f,c
  2255  000E5A  5033               	movf	(??___flmul+3)^0,w,c
  2256  000E5C  223E               	addwfc	(___flmul@prod+3)^0,f,c
  2257  000E5E  C037  F038         	movff	___flmul@grs+2,___flmul@grs+3
  2258  000E62  C036  F037         	movff	___flmul@grs+1,___flmul@grs+2
  2259  000E66  C035  F036         	movff	___flmul@grs,___flmul@grs+1
  2260  000E6A  6A35               	clrf	___flmul@grs^0,c
  2261  000E6C  5039               	movf	___flmul@aexp^0,w,c
  2262  000E6E  C03A  F030         	movff	___flmul@bexp,??___flmul
  2263  000E72  6A31               	clrf	(??___flmul+1)^0,c
  2264  000E74  2630               	addwf	??___flmul^0,f,c
  2265  000E76  0E00               	movlw	0
  2266  000E78  2231               	addwfc	(??___flmul+1)^0,f,c
  2267  000E7A  0E82               	movlw	130
  2268  000E7C  2430               	addwf	??___flmul^0,w,c
  2269  000E7E  6E3F               	movwf	___flmul@temp^0,c
  2270  000E80  0EFF               	movlw	255
  2271  000E82  2031               	addwfc	(??___flmul+1)^0,w,c
  2272  000E84  6E40               	movwf	(___flmul@temp+1)^0,c
  2273  000E86  EF5E  F007         	goto	l2287
  2274  000E8A                     l2281:
  2275  000E8A  FFFF               	dw	65535	; assembler added errata NOP
  2276  000E8C  90D8               	bcf	status,0,c
  2277  000E8E  363B               	rlcf	___flmul@prod^0,f,c
  2278  000E90  363C               	rlcf	(___flmul@prod+1)^0,f,c
  2279  000E92  363D               	rlcf	(___flmul@prod+2)^0,f,c
  2280  000E94  363E               	rlcf	(___flmul@prod+3)^0,f,c
  2281  000E96  AE38               	btfss	(___flmul@grs+3)^0,7,c
  2282  000E98  EF50  F007         	goto	u1691
  2283  000E9C  EF53  F007         	goto	u1690
  2284  000EA0                     u1691:
  2285  000EA0  FFFF               	dw	65535	; assembler added errata NOP
  2286  000EA2  EF55  F007         	goto	l919
  2287  000EA6                     u1690:
  2288  000EA6  FFFF               	dw	65535	; assembler added errata NOP
  2289  000EA8  803B               	bsf	___flmul@prod^0,0,c
  2290  000EAA                     l919:
  2291  000EAA  FFFF               	dw	65535	; assembler added errata NOP
  2292  000EAC  90D8               	bcf	status,0,c
  2293  000EAE  3635               	rlcf	___flmul@grs^0,f,c
  2294  000EB0  3636               	rlcf	(___flmul@grs+1)^0,f,c
  2295  000EB2  3637               	rlcf	(___flmul@grs+2)^0,f,c
  2296  000EB4  3638               	rlcf	(___flmul@grs+3)^0,f,c
  2297  000EB6  063F               	decf	___flmul@temp^0,f,c
  2298  000EB8  A0D8               	btfss	status,0,c
  2299  000EBA  0640               	decf	(___flmul@temp+1)^0,f,c
  2300  000EBC                     l2287:
  2301  000EBC  FFFF               	dw	65535	; assembler added errata NOP
  2302  000EBE  AE3D               	btfss	(___flmul@prod+2)^0,7,c
  2303  000EC0  EF64  F007         	goto	u1701
  2304  000EC4  EF67  F007         	goto	u1700
  2305  000EC8                     u1701:
  2306  000EC8  FFFF               	dw	65535	; assembler added errata NOP
  2307  000ECA  EF45  F007         	goto	l2281
  2308  000ECE                     u1700:
  2309  000ECE  FFFF               	dw	65535	; assembler added errata NOP
  2310  000ED0  0E00               	movlw	0
  2311  000ED2  6E39               	movwf	___flmul@aexp^0,c
  2312  000ED4  AE38               	btfss	(___flmul@grs+3)^0,7,c
  2313  000ED6  EF6F  F007         	goto	u1711
  2314  000EDA  EF72  F007         	goto	u1710
  2315  000EDE                     u1711:
  2316  000EDE  FFFF               	dw	65535	; assembler added errata NOP
  2317  000EE0  EF9D  F007         	goto	l921
  2318  000EE4                     u1710:
  2319  000EE4  FFFF               	dw	65535	; assembler added errata NOP
  2320  000EE6  0EFF               	movlw	255
  2321  000EE8  1435               	andwf	___flmul@grs^0,w,c
  2322  000EEA  6E30               	movwf	??___flmul^0,c
  2323  000EEC  0EFF               	movlw	255
  2324  000EEE  1436               	andwf	(___flmul@grs+1)^0,w,c
  2325  000EF0  6E31               	movwf	(??___flmul+1)^0,c
  2326  000EF2  0EFF               	movlw	255
  2327  000EF4  1437               	andwf	(___flmul@grs+2)^0,w,c
  2328  000EF6  6E32               	movwf	(??___flmul+2)^0,c
  2329  000EF8  0E7F               	movlw	127
  2330  000EFA  1438               	andwf	(___flmul@grs+3)^0,w,c
  2331  000EFC  6E33               	movwf	(??___flmul+3)^0,c
  2332  000EFE  5030               	movf	??___flmul^0,w,c
  2333  000F00  1031               	iorwf	(??___flmul+1)^0,w,c
  2334  000F02  1032               	iorwf	(??___flmul+2)^0,w,c
  2335  000F04  1033               	iorwf	(??___flmul+3)^0,w,c
  2336  000F06  B4D8               	btfsc	status,2,c
  2337  000F08  EF88  F007         	goto	u1721
  2338  000F0C  EF8B  F007         	goto	u1720
  2339  000F10                     u1721:
  2340  000F10  FFFF               	dw	65535	; assembler added errata NOP
  2341  000F12  EF91  F007         	goto	l922
  2342  000F16                     u1720:
  2343  000F16  FFFF               	dw	65535	; assembler added errata NOP
  2344  000F18                     l2295:
  2345  000F18  FFFF               	dw	65535	; assembler added errata NOP
  2346  000F1A  0E01               	movlw	1
  2347  000F1C  6E39               	movwf	___flmul@aexp^0,c
  2348  000F1E  EF9D  F007         	goto	l921
  2349  000F22                     l922:
  2350  000F22  FFFF               	dw	65535	; assembler added errata NOP
  2351  000F24  A03B               	btfss	___flmul@prod^0,0,c
  2352  000F26  EF97  F007         	goto	u1731
  2353  000F2A  EF9A  F007         	goto	u1730
  2354  000F2E                     u1731:
  2355  000F2E  FFFF               	dw	65535	; assembler added errata NOP
  2356  000F30  EF9D  F007         	goto	l921
  2357  000F34                     u1730:
  2358  000F34  FFFF               	dw	65535	; assembler added errata NOP
  2359  000F36  EF8C  F007         	goto	l2295
  2360  000F3A                     l921:
  2361  000F3A  FFFF               	dw	65535	; assembler added errata NOP
  2362  000F3C  5039               	movf	___flmul@aexp^0,w,c
  2363  000F3E  B4D8               	btfsc	status,2,c
  2364  000F40  EFA4  F007         	goto	u1741
  2365  000F44  EFA7  F007         	goto	u1740
  2366  000F48                     u1741:
  2367  000F48  FFFF               	dw	65535	; assembler added errata NOP
  2368  000F4A  EFCE  F007         	goto	l2307
  2369  000F4E                     u1740:
  2370  000F4E  FFFF               	dw	65535	; assembler added errata NOP
  2371  000F50  0E01               	movlw	1
  2372  000F52  263B               	addwf	___flmul@prod^0,f,c
  2373  000F54  0E00               	movlw	0
  2374  000F56  223C               	addwfc	(___flmul@prod+1)^0,f,c
  2375  000F58  223D               	addwfc	(___flmul@prod+2)^0,f,c
  2376  000F5A  223E               	addwfc	(___flmul@prod+3)^0,f,c
  2377  000F5C  A03E               	btfss	(___flmul@prod+3)^0,0,c
  2378  000F5E  EFB3  F007         	goto	u1751
  2379  000F62  EFB6  F007         	goto	u1750
  2380  000F66                     u1751:
  2381  000F66  FFFF               	dw	65535	; assembler added errata NOP
  2382  000F68  EFCE  F007         	goto	l2307
  2383  000F6C                     u1750:
  2384  000F6C  FFFF               	dw	65535	; assembler added errata NOP
  2385  000F6E  C03B  F030         	movff	___flmul@prod,??___flmul
  2386  000F72  C03C  F031         	movff	___flmul@prod+1,??___flmul+1
  2387  000F76  C03D  F032         	movff	___flmul@prod+2,??___flmul+2
  2388  000F7A  C03E  F033         	movff	___flmul@prod+3,??___flmul+3
  2389  000F7E  3433               	rlcf	(??___flmul+3)^0,w,c
  2390  000F80  3233               	rrcf	(??___flmul+3)^0,f,c
  2391  000F82  3232               	rrcf	(??___flmul+2)^0,f,c
  2392  000F84  3231               	rrcf	(??___flmul+1)^0,f,c
  2393  000F86  3230               	rrcf	??___flmul^0,f,c
  2394  000F88  C030  F03B         	movff	??___flmul,___flmul@prod
  2395  000F8C  C031  F03C         	movff	??___flmul+1,___flmul@prod+1
  2396  000F90  C032  F03D         	movff	??___flmul+2,___flmul@prod+2
  2397  000F94  C033  F03E         	movff	??___flmul+3,___flmul@prod+3
  2398  000F98  4A3F               	infsnz	___flmul@temp^0,f,c
  2399  000F9A  2A40               	incf	(___flmul@temp+1)^0,f,c
  2400  000F9C                     l2307:
  2401  000F9C  FFFF               	dw	65535	; assembler added errata NOP
  2402  000F9E  BE40               	btfsc	(___flmul@temp+1)^0,7,c
  2403  000FA0  EFDA  F007         	goto	u1761
  2404  000FA4  5040               	movf	(___flmul@temp+1)^0,w,c
  2405  000FA6  E109               	bnz	u1760
  2406  000FA8  283F               	incf	___flmul@temp^0,w,c
  2407  000FAA  A0D8               	btfss	status,0,c
  2408  000FAC  EFDA  F007         	goto	u1761
  2409  000FB0  EFDD  F007         	goto	u1760
  2410  000FB4                     u1761:
  2411  000FB4  FFFF               	dw	65535	; assembler added errata NOP
  2412  000FB6  EFE8  F007         	goto	l2311
  2413  000FBA                     u1760:
  2414  000FBA  FFFF               	dw	65535	; assembler added errata NOP
  2415  000FBC  0E00               	movlw	0
  2416  000FBE  6E3B               	movwf	___flmul@prod^0,c
  2417  000FC0  0E00               	movlw	0
  2418  000FC2  6E3C               	movwf	(___flmul@prod+1)^0,c
  2419  000FC4  0E80               	movlw	128
  2420  000FC6  6E3D               	movwf	(___flmul@prod+2)^0,c
  2421  000FC8  0E7F               	movlw	127
  2422  000FCA  6E3E               	movwf	(___flmul@prod+3)^0,c
  2423  000FCC  EF1D  F008         	goto	l2323
  2424  000FD0                     l2311:
  2425  000FD0  FFFF               	dw	65535	; assembler added errata NOP
  2426  000FD2  BE40               	btfsc	(___flmul@temp+1)^0,7,c
  2427  000FD4  EFF7  F007         	goto	u1770
  2428  000FD8  5040               	movf	(___flmul@temp+1)^0,w,c
  2429  000FDA  E106               	bnz	u1771
  2430  000FDC  043F               	decf	___flmul@temp^0,w,c
  2431  000FDE  B0D8               	btfsc	status,0,c
  2432  000FE0  EFF4  F007         	goto	u1771
  2433  000FE4  EFF7  F007         	goto	u1770
  2434  000FE8                     u1771:
  2435  000FE8  FFFF               	dw	65535	; assembler added errata NOP
  2436  000FEA  EF04  F008         	goto	l929
  2437  000FEE                     u1770:
  2438  000FEE  FFFF               	dw	65535	; assembler added errata NOP
  2439  000FF0  0E00               	movlw	0
  2440  000FF2  6E3B               	movwf	___flmul@prod^0,c
  2441  000FF4  0E00               	movlw	0
  2442  000FF6  6E3C               	movwf	(___flmul@prod+1)^0,c
  2443  000FF8  0E00               	movlw	0
  2444  000FFA  6E3D               	movwf	(___flmul@prod+2)^0,c
  2445  000FFC  0E00               	movlw	0
  2446  000FFE  6E3E               	movwf	(___flmul@prod+3)^0,c
  2447  001000  0E00               	movlw	0
  2448  001002  6E34               	movwf	___flmul@sign^0,c
  2449  001004  EF1D  F008         	goto	l2323
  2450  001008                     l929:
  2451  001008  FFFF               	dw	65535	; assembler added errata NOP
  2452  00100A  C03F  F03A         	movff	___flmul@temp,___flmul@bexp
  2453  00100E  0EFF               	movlw	255
  2454  001010  163B               	andwf	___flmul@prod^0,f,c
  2455  001012  0EFF               	movlw	255
  2456  001014  163C               	andwf	(___flmul@prod+1)^0,f,c
  2457  001016  0E7F               	movlw	127
  2458  001018  163D               	andwf	(___flmul@prod+2)^0,f,c
  2459  00101A  0E00               	movlw	0
  2460  00101C  163E               	andwf	(___flmul@prod+3)^0,f,c
  2461  00101E  A03A               	btfss	___flmul@bexp^0,0,c
  2462  001020  EF14  F008         	goto	u1781
  2463  001024  EF17  F008         	goto	u1780
  2464  001028                     u1781:
  2465  001028  FFFF               	dw	65535	; assembler added errata NOP
  2466  00102A  EF19  F008         	goto	l2321
  2467  00102E                     u1780:
  2468  00102E  FFFF               	dw	65535	; assembler added errata NOP
  2469  001030  8E3D               	bsf	(___flmul@prod+2)^0,7,c
  2470  001032                     l2321:
  2471  001032  FFFF               	dw	65535	; assembler added errata NOP
  2472  001034  90D8               	bcf	status,0,c
  2473  001036  303A               	rrcf	___flmul@bexp^0,w,c
  2474  001038  6E3E               	movwf	(___flmul@prod+3)^0,c
  2475  00103A                     l2323:
  2476  00103A  FFFF               	dw	65535	; assembler added errata NOP
  2477  00103C  5034               	movf	___flmul@sign^0,w,c
  2478  00103E  123E               	iorwf	(___flmul@prod+3)^0,f,c
  2479  001040  C03B  F028         	movff	___flmul@prod,?___flmul
  2480  001044  C03C  F029         	movff	___flmul@prod+1,?___flmul+1
  2481  001048  C03D  F02A         	movff	___flmul@prod+2,?___flmul+2
  2482  00104C  C03E  F02B         	movff	___flmul@prod+3,?___flmul+3
  2483  001050                     l916:
  2484  001050  FFFF               	dw	65535	; assembler added errata NOP
  2485  001052  0012               	return		;funcret
  2486  001054  FFFF               	dw	65535	; errata NOP
  2487  001056                     __end_of___flmul:
  2488                           	callstack 0
  2489                           
  2490 ;; *************** function ___fldiv *****************
  2491 ;; Defined at:
  2492 ;;		line 11 in file "/opt/microchip/xc8/v2.36/pic/sources/c99/common/sprcdiv.c"
  2493 ;; Parameters:    Size  Location     Type
  2494 ;;  b               4   14[COMRAM] unsigned char 
  2495 ;;  a               4   18[COMRAM] unsigned char 
  2496 ;; Auto vars:     Size  Location     Type
  2497 ;;  grs             4   33[COMRAM] unsigned long 
  2498 ;;  rem             4   26[COMRAM] unsigned long 
  2499 ;;  new_exp         2   31[COMRAM] short 
  2500 ;;  aexp            1   38[COMRAM] unsigned char 
  2501 ;;  bexp            1   37[COMRAM] unsigned char 
  2502 ;;  sign            1   30[COMRAM] unsigned char 
  2503 ;; Return value:  Size  Location     Type
  2504 ;;                  4   14[COMRAM] unsigned char 
  2505 ;; Registers used:
  2506 ;;		wreg, status,2, status,0
  2507 ;; Tracked objects:
  2508 ;;		On entry : 0/0
  2509 ;;		On exit  : 0/0
  2510 ;;		Unchanged: 0/0
  2511 ;; Data sizes:     COMRAM   BANK0   BANK1   BANK2   BANK3   BANK4   BANK5
  2512 ;;      Params:         8       0       0       0       0       0       0
  2513 ;;      Locals:        13       0       0       0       0       0       0
  2514 ;;      Temps:          4       0       0       0       0       0       0
  2515 ;;      Totals:        25       0       0       0       0       0       0
  2516 ;;Total ram usage:       25 bytes
  2517 ;; Hardware stack levels used: 1
  2518 ;; Hardware stack levels required when called: 2
  2519 ;; This function calls:
  2520 ;;		Nothing
  2521 ;; This function is called by:
  2522 ;;		_globalPWM
  2523 ;;		_setPWM
  2524 ;;		_change_duty
  2525 ;; This function uses a non-reentrant model
  2526 ;;
  2527                           
  2528                           	psect	text12
  2529  001056                     __ptext12:
  2530                           	callstack 0
  2531  001056                     ___fldiv:
  2532                           	callstack 0
  2533  001056  FFFF               	dw	65535	; assembler added errata NOP
  2534  001058  5012               	movf	(___fldiv@b+3)^0,w,c
  2535  00105A  0B80               	andlw	128
  2536  00105C  6E1F               	movwf	___fldiv@sign^0,c
  2537  00105E  5012               	movf	(___fldiv@b+3)^0,w,c
  2538  001060  2412               	addwf	(___fldiv@b+3)^0,w,c
  2539  001062  6E26               	movwf	___fldiv@bexp^0,c
  2540  001064  AE11               	btfss	(___fldiv@b+2)^0,7,c
  2541  001066  EF37  F008         	goto	u1371
  2542  00106A  EF3A  F008         	goto	u1370
  2543  00106E                     u1371:
  2544  00106E  FFFF               	dw	65535	; assembler added errata NOP
  2545  001070  EF3C  F008         	goto	l2067
  2546  001074                     u1370:
  2547  001074  FFFF               	dw	65535	; assembler added errata NOP
  2548  001076  8026               	bsf	___fldiv@bexp^0,0,c
  2549  001078                     l2067:
  2550  001078  FFFF               	dw	65535	; assembler added errata NOP
  2551  00107A  5026               	movf	___fldiv@bexp^0,w,c
  2552  00107C  B4D8               	btfsc	status,2,c
  2553  00107E  EF43  F008         	goto	u1381
  2554  001082  EF46  F008         	goto	u1380
  2555  001086                     u1381:
  2556  001086  FFFF               	dw	65535	; assembler added errata NOP
  2557  001088  EF5F  F008         	goto	l2077
  2558  00108C                     u1380:
  2559  00108C  FFFF               	dw	65535	; assembler added errata NOP
  2560  00108E  2826               	incf	___fldiv@bexp^0,w,c
  2561  001090  A4D8               	btfss	status,2,c
  2562  001092  EF4D  F008         	goto	u1391
  2563  001096  EF50  F008         	goto	u1390
  2564  00109A                     u1391:
  2565  00109A  FFFF               	dw	65535	; assembler added errata NOP
  2566  00109C  EF59  F008         	goto	l2073
  2567  0010A0                     u1390:
  2568  0010A0  FFFF               	dw	65535	; assembler added errata NOP
  2569  0010A2  0E00               	movlw	0
  2570  0010A4  6E0F               	movwf	___fldiv@b^0,c
  2571  0010A6  0E00               	movlw	0
  2572  0010A8  6E10               	movwf	(___fldiv@b+1)^0,c
  2573  0010AA  0E00               	movlw	0
  2574  0010AC  6E11               	movwf	(___fldiv@b+2)^0,c
  2575  0010AE  0E00               	movlw	0
  2576  0010B0  6E12               	movwf	(___fldiv@b+3)^0,c
  2577  0010B2                     l2073:
  2578  0010B2  FFFF               	dw	65535	; assembler added errata NOP
  2579  0010B4  8E11               	bsf	(___fldiv@b+2)^0,7,c
  2580  0010B6  0E00               	movlw	0
  2581  0010B8  6E12               	movwf	(___fldiv@b+3)^0,c
  2582  0010BA  EF68  F008         	goto	l2079
  2583  0010BE                     l2077:
  2584  0010BE  FFFF               	dw	65535	; assembler added errata NOP
  2585  0010C0  0E00               	movlw	0
  2586  0010C2  6E0F               	movwf	___fldiv@b^0,c
  2587  0010C4  0E00               	movlw	0
  2588  0010C6  6E10               	movwf	(___fldiv@b+1)^0,c
  2589  0010C8  0E00               	movlw	0
  2590  0010CA  6E11               	movwf	(___fldiv@b+2)^0,c
  2591  0010CC  0E00               	movlw	0
  2592  0010CE  6E12               	movwf	(___fldiv@b+3)^0,c
  2593  0010D0                     l2079:
  2594  0010D0  FFFF               	dw	65535	; assembler added errata NOP
  2595  0010D2  5016               	movf	(___fldiv@a+3)^0,w,c
  2596  0010D4  0B80               	andlw	128
  2597  0010D6  1A1F               	xorwf	___fldiv@sign^0,f,c
  2598  0010D8  5016               	movf	(___fldiv@a+3)^0,w,c
  2599  0010DA  2416               	addwf	(___fldiv@a+3)^0,w,c
  2600  0010DC  6E27               	movwf	___fldiv@aexp^0,c
  2601  0010DE  AE15               	btfss	(___fldiv@a+2)^0,7,c
  2602  0010E0  EF74  F008         	goto	u1401
  2603  0010E4  EF77  F008         	goto	u1400
  2604  0010E8                     u1401:
  2605  0010E8  FFFF               	dw	65535	; assembler added errata NOP
  2606  0010EA  EF79  F008         	goto	l2087
  2607  0010EE                     u1400:
  2608  0010EE  FFFF               	dw	65535	; assembler added errata NOP
  2609  0010F0  8027               	bsf	___fldiv@aexp^0,0,c
  2610  0010F2                     l2087:
  2611  0010F2  FFFF               	dw	65535	; assembler added errata NOP
  2612  0010F4  5027               	movf	___fldiv@aexp^0,w,c
  2613  0010F6  B4D8               	btfsc	status,2,c
  2614  0010F8  EF80  F008         	goto	u1411
  2615  0010FC  EF83  F008         	goto	u1410
  2616  001100                     u1411:
  2617  001100  FFFF               	dw	65535	; assembler added errata NOP
  2618  001102  EF9C  F008         	goto	l2097
  2619  001106                     u1410:
  2620  001106  FFFF               	dw	65535	; assembler added errata NOP
  2621  001108  2827               	incf	___fldiv@aexp^0,w,c
  2622  00110A  A4D8               	btfss	status,2,c
  2623  00110C  EF8A  F008         	goto	u1421
  2624  001110  EF8D  F008         	goto	u1420
  2625  001114                     u1421:
  2626  001114  FFFF               	dw	65535	; assembler added errata NOP
  2627  001116  EF96  F008         	goto	l2093
  2628  00111A                     u1420:
  2629  00111A  FFFF               	dw	65535	; assembler added errata NOP
  2630  00111C  0E00               	movlw	0
  2631  00111E  6E13               	movwf	___fldiv@a^0,c
  2632  001120  0E00               	movlw	0
  2633  001122  6E14               	movwf	(___fldiv@a+1)^0,c
  2634  001124  0E00               	movlw	0
  2635  001126  6E15               	movwf	(___fldiv@a+2)^0,c
  2636  001128  0E00               	movlw	0
  2637  00112A  6E16               	movwf	(___fldiv@a+3)^0,c
  2638  00112C                     l2093:
  2639  00112C  FFFF               	dw	65535	; assembler added errata NOP
  2640  00112E  8E15               	bsf	(___fldiv@a+2)^0,7,c
  2641  001130  0E00               	movlw	0
  2642  001132  6E16               	movwf	(___fldiv@a+3)^0,c
  2643  001134  EFA5  F008         	goto	l2099
  2644  001138                     l2097:
  2645  001138  FFFF               	dw	65535	; assembler added errata NOP
  2646  00113A  0E00               	movlw	0
  2647  00113C  6E13               	movwf	___fldiv@a^0,c
  2648  00113E  0E00               	movlw	0
  2649  001140  6E14               	movwf	(___fldiv@a+1)^0,c
  2650  001142  0E00               	movlw	0
  2651  001144  6E15               	movwf	(___fldiv@a+2)^0,c
  2652  001146  0E00               	movlw	0
  2653  001148  6E16               	movwf	(___fldiv@a+3)^0,c
  2654  00114A                     l2099:
  2655  00114A  FFFF               	dw	65535	; assembler added errata NOP
  2656  00114C  5013               	movf	___fldiv@a^0,w,c
  2657  00114E  1014               	iorwf	(___fldiv@a+1)^0,w,c
  2658  001150  1015               	iorwf	(___fldiv@a+2)^0,w,c
  2659  001152  1016               	iorwf	(___fldiv@a+3)^0,w,c
  2660  001154  A4D8               	btfss	status,2,c
  2661  001156  EFAF  F008         	goto	u1431
  2662  00115A  EFB2  F008         	goto	u1430
  2663  00115E                     u1431:
  2664  00115E  FFFF               	dw	65535	; assembler added errata NOP
  2665  001160  EFCC  F008         	goto	l2111
  2666  001164                     u1430:
  2667  001164  FFFF               	dw	65535	; assembler added errata NOP
  2668  001166  0E00               	movlw	0
  2669  001168  6E0F               	movwf	___fldiv@b^0,c
  2670  00116A  0E00               	movlw	0
  2671  00116C  6E10               	movwf	(___fldiv@b+1)^0,c
  2672  00116E  0E00               	movlw	0
  2673  001170  6E11               	movwf	(___fldiv@b+2)^0,c
  2674  001172  0E00               	movlw	0
  2675  001174  6E12               	movwf	(___fldiv@b+3)^0,c
  2676  001176  0E80               	movlw	128
  2677  001178  1211               	iorwf	(___fldiv@b+2)^0,f,c
  2678  00117A  0E7F               	movlw	127
  2679  00117C  1212               	iorwf	(___fldiv@b+3)^0,f,c
  2680  00117E                     l2105:
  2681  00117E  FFFF               	dw	65535	; assembler added errata NOP
  2682  001180  501F               	movf	___fldiv@sign^0,w,c
  2683  001182  1212               	iorwf	(___fldiv@b+3)^0,f,c
  2684  001184  C00F  F00F         	movff	___fldiv@b,?___fldiv
  2685  001188  C010  F010         	movff	___fldiv@b+1,?___fldiv+1
  2686  00118C  C011  F011         	movff	___fldiv@b+2,?___fldiv+2
  2687  001190  C012  F012         	movff	___fldiv@b+3,?___fldiv+3
  2688  001194  EF41  F00A         	goto	l880
  2689  001198                     l2111:
  2690  001198  FFFF               	dw	65535	; assembler added errata NOP
  2691  00119A  5026               	movf	___fldiv@bexp^0,w,c
  2692  00119C  A4D8               	btfss	status,2,c
  2693  00119E  EFD3  F008         	goto	u1441
  2694  0011A2  EFD6  F008         	goto	u1440
  2695  0011A6                     u1441:
  2696  0011A6  FFFF               	dw	65535	; assembler added errata NOP
  2697  0011A8  EFE1  F008         	goto	l2119
  2698  0011AC                     u1440:
  2699  0011AC  FFFF               	dw	65535	; assembler added errata NOP
  2700  0011AE  0E00               	movlw	0
  2701  0011B0  6E0F               	movwf	?___fldiv^0,c
  2702  0011B2  0E00               	movlw	0
  2703  0011B4  6E10               	movwf	(?___fldiv+1)^0,c
  2704  0011B6  0E00               	movlw	0
  2705  0011B8  6E11               	movwf	(?___fldiv+2)^0,c
  2706  0011BA  0E00               	movlw	0
  2707  0011BC  6E12               	movwf	(?___fldiv+3)^0,c
  2708  0011BE  EF41  F00A         	goto	l880
  2709  0011C2                     l2119:
  2710  0011C2  FFFF               	dw	65535	; assembler added errata NOP
  2711  0011C4  5027               	movf	___fldiv@aexp^0,w,c
  2712  0011C6  C026  F017         	movff	___fldiv@bexp,??___fldiv
  2713  0011CA  6A18               	clrf	(??___fldiv+1)^0,c
  2714  0011CC  5E17               	subwf	??___fldiv^0,f,c
  2715  0011CE  0E00               	movlw	0
  2716  0011D0  5A18               	subwfb	(??___fldiv+1)^0,f,c
  2717  0011D2  0E7F               	movlw	127
  2718  0011D4  2417               	addwf	??___fldiv^0,w,c
  2719  0011D6  6E20               	movwf	___fldiv@new_exp^0,c
  2720  0011D8  0E00               	movlw	0
  2721  0011DA  2018               	addwfc	(??___fldiv+1)^0,w,c
  2722  0011DC  6E21               	movwf	(___fldiv@new_exp+1)^0,c
  2723  0011DE  C00F  F01B         	movff	___fldiv@b,___fldiv@rem
  2724  0011E2  C010  F01C         	movff	___fldiv@b+1,___fldiv@rem+1
  2725  0011E6  C011  F01D         	movff	___fldiv@b+2,___fldiv@rem+2
  2726  0011EA  C012  F01E         	movff	___fldiv@b+3,___fldiv@rem+3
  2727  0011EE  0E00               	movlw	0
  2728  0011F0  6E0F               	movwf	___fldiv@b^0,c
  2729  0011F2  0E00               	movlw	0
  2730  0011F4  6E10               	movwf	(___fldiv@b+1)^0,c
  2731  0011F6  0E00               	movlw	0
  2732  0011F8  6E11               	movwf	(___fldiv@b+2)^0,c
  2733  0011FA  0E00               	movlw	0
  2734  0011FC  6E12               	movwf	(___fldiv@b+3)^0,c
  2735  0011FE  0E00               	movlw	0
  2736  001200  6E22               	movwf	___fldiv@grs^0,c
  2737  001202  0E00               	movlw	0
  2738  001204  6E23               	movwf	(___fldiv@grs+1)^0,c
  2739  001206  0E00               	movlw	0
  2740  001208  6E24               	movwf	(___fldiv@grs+2)^0,c
  2741  00120A  0E00               	movlw	0
  2742  00120C  6E25               	movwf	(___fldiv@grs+3)^0,c
  2743  00120E  0E00               	movlw	0
  2744  001210  6E27               	movwf	___fldiv@aexp^0,c
  2745  001212  EF4D  F009         	goto	l882
  2746  001216                     l2129:
  2747  001216  FFFF               	dw	65535	; assembler added errata NOP
  2748  001218  5027               	movf	___fldiv@aexp^0,w,c
  2749  00121A  B4D8               	btfsc	status,2,c
  2750  00121C  EF12  F009         	goto	u1451
  2751  001220  EF15  F009         	goto	u1450
  2752  001224                     u1451:
  2753  001224  FFFF               	dw	65535	; assembler added errata NOP
  2754  001226  EF30  F009         	goto	l2137
  2755  00122A                     u1450:
  2756  00122A  FFFF               	dw	65535	; assembler added errata NOP
  2757  00122C  90D8               	bcf	status,0,c
  2758  00122E  361B               	rlcf	___fldiv@rem^0,f,c
  2759  001230  361C               	rlcf	(___fldiv@rem+1)^0,f,c
  2760  001232  361D               	rlcf	(___fldiv@rem+2)^0,f,c
  2761  001234  361E               	rlcf	(___fldiv@rem+3)^0,f,c
  2762  001236  90D8               	bcf	status,0,c
  2763  001238  360F               	rlcf	___fldiv@b^0,f,c
  2764  00123A  3610               	rlcf	(___fldiv@b+1)^0,f,c
  2765  00123C  3611               	rlcf	(___fldiv@b+2)^0,f,c
  2766  00123E  3612               	rlcf	(___fldiv@b+3)^0,f,c
  2767  001240  AE25               	btfss	(___fldiv@grs+3)^0,7,c
  2768  001242  EF25  F009         	goto	u1461
  2769  001246  EF28  F009         	goto	u1460
  2770  00124A                     u1461:
  2771  00124A  FFFF               	dw	65535	; assembler added errata NOP
  2772  00124C  EF2A  F009         	goto	l885
  2773  001250                     u1460:
  2774  001250  FFFF               	dw	65535	; assembler added errata NOP
  2775  001252  800F               	bsf	___fldiv@b^0,0,c
  2776  001254                     l885:
  2777  001254  FFFF               	dw	65535	; assembler added errata NOP
  2778  001256  90D8               	bcf	status,0,c
  2779  001258  3622               	rlcf	___fldiv@grs^0,f,c
  2780  00125A  3623               	rlcf	(___fldiv@grs+1)^0,f,c
  2781  00125C  3624               	rlcf	(___fldiv@grs+2)^0,f,c
  2782  00125E  3625               	rlcf	(___fldiv@grs+3)^0,f,c
  2783  001260                     l2137:
  2784  001260  FFFF               	dw	65535	; assembler added errata NOP
  2785  001262  5013               	movf	___fldiv@a^0,w,c
  2786  001264  5C1B               	subwf	___fldiv@rem^0,w,c
  2787  001266  5014               	movf	(___fldiv@a+1)^0,w,c
  2788  001268  581C               	subwfb	(___fldiv@rem+1)^0,w,c
  2789  00126A  5015               	movf	(___fldiv@a+2)^0,w,c
  2790  00126C  581D               	subwfb	(___fldiv@rem+2)^0,w,c
  2791  00126E  5016               	movf	(___fldiv@a+3)^0,w,c
  2792  001270  581E               	subwfb	(___fldiv@rem+3)^0,w,c
  2793  001272  A0D8               	btfss	status,0,c
  2794  001274  EF3E  F009         	goto	u1471
  2795  001278  EF41  F009         	goto	u1470
  2796  00127C                     u1471:
  2797  00127C  FFFF               	dw	65535	; assembler added errata NOP
  2798  00127E  EF4B  F009         	goto	l2143
  2799  001282                     u1470:
  2800  001282  FFFF               	dw	65535	; assembler added errata NOP
  2801  001284  8C25               	bsf	(___fldiv@grs+3)^0,6,c
  2802  001286  5013               	movf	___fldiv@a^0,w,c
  2803  001288  5E1B               	subwf	___fldiv@rem^0,f,c
  2804  00128A  5014               	movf	(___fldiv@a+1)^0,w,c
  2805  00128C  5A1C               	subwfb	(___fldiv@rem+1)^0,f,c
  2806  00128E  5015               	movf	(___fldiv@a+2)^0,w,c
  2807  001290  5A1D               	subwfb	(___fldiv@rem+2)^0,f,c
  2808  001292  5016               	movf	(___fldiv@a+3)^0,w,c
  2809  001294  5A1E               	subwfb	(___fldiv@rem+3)^0,f,c
  2810  001296                     l2143:
  2811  001296  FFFF               	dw	65535	; assembler added errata NOP
  2812  001298  2A27               	incf	___fldiv@aexp^0,f,c
  2813  00129A                     l882:
  2814  00129A  FFFF               	dw	65535	; assembler added errata NOP
  2815  00129C  0E19               	movlw	25
  2816  00129E  6427               	cpfsgt	___fldiv@aexp^0,c
  2817  0012A0  EF54  F009         	goto	u1481
  2818  0012A4  EF57  F009         	goto	u1480
  2819  0012A8                     u1481:
  2820  0012A8  FFFF               	dw	65535	; assembler added errata NOP
  2821  0012AA  EF0B  F009         	goto	l2129
  2822  0012AE                     u1480:
  2823  0012AE  FFFF               	dw	65535	; assembler added errata NOP
  2824  0012B0  501B               	movf	___fldiv@rem^0,w,c
  2825  0012B2  101C               	iorwf	(___fldiv@rem+1)^0,w,c
  2826  0012B4  101D               	iorwf	(___fldiv@rem+2)^0,w,c
  2827  0012B6  101E               	iorwf	(___fldiv@rem+3)^0,w,c
  2828  0012B8  B4D8               	btfsc	status,2,c
  2829  0012BA  EF61  F009         	goto	u1491
  2830  0012BE  EF64  F009         	goto	u1490
  2831  0012C2                     u1491:
  2832  0012C2  FFFF               	dw	65535	; assembler added errata NOP
  2833  0012C4  EF81  F009         	goto	l2155
  2834  0012C8                     u1490:
  2835  0012C8  FFFF               	dw	65535	; assembler added errata NOP
  2836  0012CA  8022               	bsf	___fldiv@grs^0,0,c
  2837  0012CC  EF81  F009         	goto	l2155
  2838  0012D0                     l2149:
  2839  0012D0  FFFF               	dw	65535	; assembler added errata NOP
  2840  0012D2  90D8               	bcf	status,0,c
  2841  0012D4  360F               	rlcf	___fldiv@b^0,f,c
  2842  0012D6  3610               	rlcf	(___fldiv@b+1)^0,f,c
  2843  0012D8  3611               	rlcf	(___fldiv@b+2)^0,f,c
  2844  0012DA  3612               	rlcf	(___fldiv@b+3)^0,f,c
  2845  0012DC  AE25               	btfss	(___fldiv@grs+3)^0,7,c
  2846  0012DE  EF73  F009         	goto	u1501
  2847  0012E2  EF76  F009         	goto	u1500
  2848  0012E6                     u1501:
  2849  0012E6  FFFF               	dw	65535	; assembler added errata NOP
  2850  0012E8  EF78  F009         	goto	l891
  2851  0012EC                     u1500:
  2852  0012EC  FFFF               	dw	65535	; assembler added errata NOP
  2853  0012EE  800F               	bsf	___fldiv@b^0,0,c
  2854  0012F0                     l891:
  2855  0012F0  FFFF               	dw	65535	; assembler added errata NOP
  2856  0012F2  90D8               	bcf	status,0,c
  2857  0012F4  3622               	rlcf	___fldiv@grs^0,f,c
  2858  0012F6  3623               	rlcf	(___fldiv@grs+1)^0,f,c
  2859  0012F8  3624               	rlcf	(___fldiv@grs+2)^0,f,c
  2860  0012FA  3625               	rlcf	(___fldiv@grs+3)^0,f,c
  2861  0012FC  0620               	decf	___fldiv@new_exp^0,f,c
  2862  0012FE  A0D8               	btfss	status,0,c
  2863  001300  0621               	decf	(___fldiv@new_exp+1)^0,f,c
  2864  001302                     l2155:
  2865  001302  FFFF               	dw	65535	; assembler added errata NOP
  2866  001304  AE11               	btfss	(___fldiv@b+2)^0,7,c
  2867  001306  EF87  F009         	goto	u1511
  2868  00130A  EF8A  F009         	goto	u1510
  2869  00130E                     u1511:
  2870  00130E  FFFF               	dw	65535	; assembler added errata NOP
  2871  001310  EF68  F009         	goto	l2149
  2872  001314                     u1510:
  2873  001314  FFFF               	dw	65535	; assembler added errata NOP
  2874  001316  0E00               	movlw	0
  2875  001318  6E27               	movwf	___fldiv@aexp^0,c
  2876  00131A  AE25               	btfss	(___fldiv@grs+3)^0,7,c
  2877  00131C  EF92  F009         	goto	u1521
  2878  001320  EF95  F009         	goto	u1520
  2879  001324                     u1521:
  2880  001324  FFFF               	dw	65535	; assembler added errata NOP
  2881  001326  EFC0  F009         	goto	l893
  2882  00132A                     u1520:
  2883  00132A  FFFF               	dw	65535	; assembler added errata NOP
  2884  00132C  0EFF               	movlw	255
  2885  00132E  1422               	andwf	___fldiv@grs^0,w,c
  2886  001330  6E17               	movwf	??___fldiv^0,c
  2887  001332  0EFF               	movlw	255
  2888  001334  1423               	andwf	(___fldiv@grs+1)^0,w,c
  2889  001336  6E18               	movwf	(??___fldiv+1)^0,c
  2890  001338  0EFF               	movlw	255
  2891  00133A  1424               	andwf	(___fldiv@grs+2)^0,w,c
  2892  00133C  6E19               	movwf	(??___fldiv+2)^0,c
  2893  00133E  0E7F               	movlw	127
  2894  001340  1425               	andwf	(___fldiv@grs+3)^0,w,c
  2895  001342  6E1A               	movwf	(??___fldiv+3)^0,c
  2896  001344  5017               	movf	??___fldiv^0,w,c
  2897  001346  1018               	iorwf	(??___fldiv+1)^0,w,c
  2898  001348  1019               	iorwf	(??___fldiv+2)^0,w,c
  2899  00134A  101A               	iorwf	(??___fldiv+3)^0,w,c
  2900  00134C  B4D8               	btfsc	status,2,c
  2901  00134E  EFAB  F009         	goto	u1531
  2902  001352  EFAE  F009         	goto	u1530
  2903  001356                     u1531:
  2904  001356  FFFF               	dw	65535	; assembler added errata NOP
  2905  001358  EFB4  F009         	goto	l894
  2906  00135C                     u1530:
  2907  00135C  FFFF               	dw	65535	; assembler added errata NOP
  2908  00135E                     l2163:
  2909  00135E  FFFF               	dw	65535	; assembler added errata NOP
  2910  001360  0E01               	movlw	1
  2911  001362  6E27               	movwf	___fldiv@aexp^0,c
  2912  001364  EFC0  F009         	goto	l893
  2913  001368                     l894:
  2914  001368  FFFF               	dw	65535	; assembler added errata NOP
  2915  00136A  A00F               	btfss	___fldiv@b^0,0,c
  2916  00136C  EFBA  F009         	goto	u1541
  2917  001370  EFBD  F009         	goto	u1540
  2918  001374                     u1541:
  2919  001374  FFFF               	dw	65535	; assembler added errata NOP
  2920  001376  EFC0  F009         	goto	l893
  2921  00137A                     u1540:
  2922  00137A  FFFF               	dw	65535	; assembler added errata NOP
  2923  00137C  EFAF  F009         	goto	l2163
  2924  001380                     l893:
  2925  001380  FFFF               	dw	65535	; assembler added errata NOP
  2926  001382  5027               	movf	___fldiv@aexp^0,w,c
  2927  001384  B4D8               	btfsc	status,2,c
  2928  001386  EFC7  F009         	goto	u1551
  2929  00138A  EFCA  F009         	goto	u1550
  2930  00138E                     u1551:
  2931  00138E  FFFF               	dw	65535	; assembler added errata NOP
  2932  001390  EFF1  F009         	goto	l2175
  2933  001394                     u1550:
  2934  001394  FFFF               	dw	65535	; assembler added errata NOP
  2935  001396  0E01               	movlw	1
  2936  001398  260F               	addwf	___fldiv@b^0,f,c
  2937  00139A  0E00               	movlw	0
  2938  00139C  2210               	addwfc	(___fldiv@b+1)^0,f,c
  2939  00139E  2211               	addwfc	(___fldiv@b+2)^0,f,c
  2940  0013A0  2212               	addwfc	(___fldiv@b+3)^0,f,c
  2941  0013A2  A012               	btfss	(___fldiv@b+3)^0,0,c
  2942  0013A4  EFD6  F009         	goto	u1561
  2943  0013A8  EFD9  F009         	goto	u1560
  2944  0013AC                     u1561:
  2945  0013AC  FFFF               	dw	65535	; assembler added errata NOP
  2946  0013AE  EFF1  F009         	goto	l2175
  2947  0013B2                     u1560:
  2948  0013B2  FFFF               	dw	65535	; assembler added errata NOP
  2949  0013B4  C00F  F017         	movff	___fldiv@b,??___fldiv
  2950  0013B8  C010  F018         	movff	___fldiv@b+1,??___fldiv+1
  2951  0013BC  C011  F019         	movff	___fldiv@b+2,??___fldiv+2
  2952  0013C0  C012  F01A         	movff	___fldiv@b+3,??___fldiv+3
  2953  0013C4  341A               	rlcf	(??___fldiv+3)^0,w,c
  2954  0013C6  321A               	rrcf	(??___fldiv+3)^0,f,c
  2955  0013C8  3219               	rrcf	(??___fldiv+2)^0,f,c
  2956  0013CA  3218               	rrcf	(??___fldiv+1)^0,f,c
  2957  0013CC  3217               	rrcf	??___fldiv^0,f,c
  2958  0013CE  C017  F00F         	movff	??___fldiv,___fldiv@b
  2959  0013D2  C018  F010         	movff	??___fldiv+1,___fldiv@b+1
  2960  0013D6  C019  F011         	movff	??___fldiv+2,___fldiv@b+2
  2961  0013DA  C01A  F012         	movff	??___fldiv+3,___fldiv@b+3
  2962  0013DE  4A20               	infsnz	___fldiv@new_exp^0,f,c
  2963  0013E0  2A21               	incf	(___fldiv@new_exp+1)^0,f,c
  2964  0013E2                     l2175:
  2965  0013E2  FFFF               	dw	65535	; assembler added errata NOP
  2966  0013E4  BE21               	btfsc	(___fldiv@new_exp+1)^0,7,c
  2967  0013E6  EFFD  F009         	goto	u1571
  2968  0013EA  5021               	movf	(___fldiv@new_exp+1)^0,w,c
  2969  0013EC  E109               	bnz	u1570
  2970  0013EE  2820               	incf	___fldiv@new_exp^0,w,c
  2971  0013F0  A0D8               	btfss	status,0,c
  2972  0013F2  EFFD  F009         	goto	u1571
  2973  0013F6  EF00  F00A         	goto	u1570
  2974  0013FA                     u1571:
  2975  0013FA  FFFF               	dw	65535	; assembler added errata NOP
  2976  0013FC  EF0C  F00A         	goto	l2179
  2977  001400                     u1570:
  2978  001400  FFFF               	dw	65535	; assembler added errata NOP
  2979  001402  0E00               	movlw	0
  2980  001404  6E21               	movwf	(___fldiv@new_exp+1)^0,c
  2981  001406  6820               	setf	___fldiv@new_exp^0,c
  2982  001408  0E00               	movlw	0
  2983  00140A  6E0F               	movwf	___fldiv@b^0,c
  2984  00140C  0E00               	movlw	0
  2985  00140E  6E10               	movwf	(___fldiv@b+1)^0,c
  2986  001410  0E00               	movlw	0
  2987  001412  6E11               	movwf	(___fldiv@b+2)^0,c
  2988  001414  0E00               	movlw	0
  2989  001416  6E12               	movwf	(___fldiv@b+3)^0,c
  2990  001418                     l2179:
  2991  001418  FFFF               	dw	65535	; assembler added errata NOP
  2992  00141A  BE21               	btfsc	(___fldiv@new_exp+1)^0,7,c
  2993  00141C  EF1B  F00A         	goto	u1580
  2994  001420  5021               	movf	(___fldiv@new_exp+1)^0,w,c
  2995  001422  E106               	bnz	u1581
  2996  001424  0420               	decf	___fldiv@new_exp^0,w,c
  2997  001426  B0D8               	btfsc	status,0,c
  2998  001428  EF18  F00A         	goto	u1581
  2999  00142C  EF1B  F00A         	goto	u1580
  3000  001430                     u1581:
  3001  001430  FFFF               	dw	65535	; assembler added errata NOP
  3002  001432  EF2A  F00A         	goto	l2183
  3003  001436                     u1580:
  3004  001436  FFFF               	dw	65535	; assembler added errata NOP
  3005  001438  0E00               	movlw	0
  3006  00143A  6E21               	movwf	(___fldiv@new_exp+1)^0,c
  3007  00143C  0E00               	movlw	0
  3008  00143E  6E20               	movwf	___fldiv@new_exp^0,c
  3009  001440  0E00               	movlw	0
  3010  001442  6E0F               	movwf	___fldiv@b^0,c
  3011  001444  0E00               	movlw	0
  3012  001446  6E10               	movwf	(___fldiv@b+1)^0,c
  3013  001448  0E00               	movlw	0
  3014  00144A  6E11               	movwf	(___fldiv@b+2)^0,c
  3015  00144C  0E00               	movlw	0
  3016  00144E  6E12               	movwf	(___fldiv@b+3)^0,c
  3017  001450  0E00               	movlw	0
  3018  001452  6E1F               	movwf	___fldiv@sign^0,c
  3019  001454                     l2183:
  3020  001454  FFFF               	dw	65535	; assembler added errata NOP
  3021  001456  C020  F026         	movff	___fldiv@new_exp,___fldiv@bexp
  3022  00145A  A026               	btfss	___fldiv@bexp^0,0,c
  3023  00145C  EF32  F00A         	goto	u1591
  3024  001460  EF35  F00A         	goto	u1590
  3025  001464                     u1591:
  3026  001464  FFFF               	dw	65535	; assembler added errata NOP
  3027  001466  EF39  F00A         	goto	l2189
  3028  00146A                     u1590:
  3029  00146A  FFFF               	dw	65535	; assembler added errata NOP
  3030  00146C  8E11               	bsf	(___fldiv@b+2)^0,7,c
  3031  00146E  EF3B  F00A         	goto	l2191
  3032  001472                     l2189:
  3033  001472  FFFF               	dw	65535	; assembler added errata NOP
  3034  001474  9E11               	bcf	(___fldiv@b+2)^0,7,c
  3035  001476                     l2191:
  3036  001476  FFFF               	dw	65535	; assembler added errata NOP
  3037  001478  90D8               	bcf	status,0,c
  3038  00147A  3026               	rrcf	___fldiv@bexp^0,w,c
  3039  00147C  6E12               	movwf	(___fldiv@b+3)^0,c
  3040  00147E  EFBF  F008         	goto	l2105
  3041  001482                     l880:
  3042  001482  FFFF               	dw	65535	; assembler added errata NOP
  3043  001484  0012               	return		;funcret
  3044  001486  FFFF               	dw	65535	; errata NOP
  3045  001488                     __end_of___fldiv:
  3046                           	callstack 0
  3047                           
  3048 ;; *************** function ___fladd *****************
  3049 ;; Defined at:
  3050 ;;		line 10 in file "/opt/microchip/xc8/v2.36/pic/sources/c99/common/sprcadd.c"
  3051 ;; Parameters:    Size  Location     Type
  3052 ;;  b               4   64[COMRAM] unsigned char 
  3053 ;;  a               4   68[COMRAM] unsigned char 
  3054 ;; Auto vars:     Size  Location     Type
  3055 ;;  grs             1   79[COMRAM] unsigned char 
  3056 ;;  bexp            1   78[COMRAM] unsigned char 
  3057 ;;  aexp            1   77[COMRAM] unsigned char 
  3058 ;;  signs           1   76[COMRAM] unsigned char 
  3059 ;; Return value:  Size  Location     Type
  3060 ;;                  4   64[COMRAM] unsigned char 
  3061 ;; Registers used:
  3062 ;;		wreg, status,2, status,0
  3063 ;; Tracked objects:
  3064 ;;		On entry : 0/0
  3065 ;;		On exit  : 0/0
  3066 ;;		Unchanged: 0/0
  3067 ;; Data sizes:     COMRAM   BANK0   BANK1   BANK2   BANK3   BANK4   BANK5
  3068 ;;      Params:         8       0       0       0       0       0       0
  3069 ;;      Locals:         4       0       0       0       0       0       0
  3070 ;;      Temps:          4       0       0       0       0       0       0
  3071 ;;      Totals:        16       0       0       0       0       0       0
  3072 ;;Total ram usage:       16 bytes
  3073 ;; Hardware stack levels used: 1
  3074 ;; Hardware stack levels required when called: 2
  3075 ;; This function calls:
  3076 ;;		Nothing
  3077 ;; This function is called by:
  3078 ;;		_globalPWM
  3079 ;; This function uses a non-reentrant model
  3080 ;;
  3081                           
  3082                           	psect	text13
  3083  00060A                     __ptext13:
  3084                           	callstack 0
  3085  00060A                     ___fladd:
  3086                           	callstack 0
  3087  00060A  FFFF               	dw	65535	; assembler added errata NOP
  3088  00060C  5044               	movf	(___fladd@b+3)^0,w,c
  3089  00060E  0B80               	andlw	128
  3090  000610  6E4D               	movwf	___fladd@signs^0,c
  3091  000612  5044               	movf	(___fladd@b+3)^0,w,c
  3092  000614  2444               	addwf	(___fladd@b+3)^0,w,c
  3093  000616  6E4F               	movwf	___fladd@bexp^0,c
  3094  000618  AE43               	btfss	(___fladd@b+2)^0,7,c
  3095  00061A  EF11  F003         	goto	u981
  3096  00061E  EF14  F003         	goto	u980
  3097  000622                     u981:
  3098  000622  FFFF               	dw	65535	; assembler added errata NOP
  3099  000624  EF16  F003         	goto	l1865
  3100  000628                     u980:
  3101  000628  FFFF               	dw	65535	; assembler added errata NOP
  3102  00062A  804F               	bsf	___fladd@bexp^0,0,c
  3103  00062C                     l1865:
  3104  00062C  FFFF               	dw	65535	; assembler added errata NOP
  3105  00062E  504F               	movf	___fladd@bexp^0,w,c
  3106  000630  B4D8               	btfsc	status,2,c
  3107  000632  EF1D  F003         	goto	u991
  3108  000636  EF20  F003         	goto	u990
  3109  00063A                     u991:
  3110  00063A  FFFF               	dw	65535	; assembler added errata NOP
  3111  00063C  EF39  F003         	goto	l1875
  3112  000640                     u990:
  3113  000640  FFFF               	dw	65535	; assembler added errata NOP
  3114  000642  284F               	incf	___fladd@bexp^0,w,c
  3115  000644  A4D8               	btfss	status,2,c
  3116  000646  EF27  F003         	goto	u1001
  3117  00064A  EF2A  F003         	goto	u1000
  3118  00064E                     u1001:
  3119  00064E  FFFF               	dw	65535	; assembler added errata NOP
  3120  000650  EF33  F003         	goto	l1871
  3121  000654                     u1000:
  3122  000654  FFFF               	dw	65535	; assembler added errata NOP
  3123  000656  0E00               	movlw	0
  3124  000658  6E41               	movwf	___fladd@b^0,c
  3125  00065A  0E00               	movlw	0
  3126  00065C  6E42               	movwf	(___fladd@b+1)^0,c
  3127  00065E  0E00               	movlw	0
  3128  000660  6E43               	movwf	(___fladd@b+2)^0,c
  3129  000662  0E00               	movlw	0
  3130  000664  6E44               	movwf	(___fladd@b+3)^0,c
  3131  000666                     l1871:
  3132  000666  FFFF               	dw	65535	; assembler added errata NOP
  3133  000668  8E43               	bsf	(___fladd@b+2)^0,7,c
  3134  00066A  0E00               	movlw	0
  3135  00066C  6E44               	movwf	(___fladd@b+3)^0,c
  3136  00066E  EF42  F003         	goto	l1877
  3137  000672                     l1875:
  3138  000672  FFFF               	dw	65535	; assembler added errata NOP
  3139  000674  0E00               	movlw	0
  3140  000676  6E41               	movwf	___fladd@b^0,c
  3141  000678  0E00               	movlw	0
  3142  00067A  6E42               	movwf	(___fladd@b+1)^0,c
  3143  00067C  0E00               	movlw	0
  3144  00067E  6E43               	movwf	(___fladd@b+2)^0,c
  3145  000680  0E00               	movlw	0
  3146  000682  6E44               	movwf	(___fladd@b+3)^0,c
  3147  000684                     l1877:
  3148  000684  FFFF               	dw	65535	; assembler added errata NOP
  3149  000686  5048               	movf	(___fladd@a+3)^0,w,c
  3150  000688  0B80               	andlw	128
  3151  00068A  6E4E               	movwf	___fladd@aexp^0,c
  3152  00068C  504D               	movf	___fladd@signs^0,w,c
  3153  00068E  184E               	xorwf	___fladd@aexp^0,w,c
  3154  000690  B4D8               	btfsc	status,2,c
  3155  000692  EF4D  F003         	goto	u1011
  3156  000696  EF50  F003         	goto	u1010
  3157  00069A                     u1011:
  3158  00069A  FFFF               	dw	65535	; assembler added errata NOP
  3159  00069C  EF52  F003         	goto	l1883
  3160  0006A0                     u1010:
  3161  0006A0  FFFF               	dw	65535	; assembler added errata NOP
  3162  0006A2  8C4D               	bsf	___fladd@signs^0,6,c
  3163  0006A4                     l1883:
  3164  0006A4  FFFF               	dw	65535	; assembler added errata NOP
  3165  0006A6  5048               	movf	(___fladd@a+3)^0,w,c
  3166  0006A8  2448               	addwf	(___fladd@a+3)^0,w,c
  3167  0006AA  6E4E               	movwf	___fladd@aexp^0,c
  3168  0006AC  AE47               	btfss	(___fladd@a+2)^0,7,c
  3169  0006AE  EF5B  F003         	goto	u1021
  3170  0006B2  EF5E  F003         	goto	u1020
  3171  0006B6                     u1021:
  3172  0006B6  FFFF               	dw	65535	; assembler added errata NOP
  3173  0006B8  EF60  F003         	goto	l1889
  3174  0006BC                     u1020:
  3175  0006BC  FFFF               	dw	65535	; assembler added errata NOP
  3176  0006BE  804E               	bsf	___fladd@aexp^0,0,c
  3177  0006C0                     l1889:
  3178  0006C0  FFFF               	dw	65535	; assembler added errata NOP
  3179  0006C2  504E               	movf	___fladd@aexp^0,w,c
  3180  0006C4  B4D8               	btfsc	status,2,c
  3181  0006C6  EF67  F003         	goto	u1031
  3182  0006CA  EF6A  F003         	goto	u1030
  3183  0006CE                     u1031:
  3184  0006CE  FFFF               	dw	65535	; assembler added errata NOP
  3185  0006D0  EF83  F003         	goto	l1899
  3186  0006D4                     u1030:
  3187  0006D4  FFFF               	dw	65535	; assembler added errata NOP
  3188  0006D6  284E               	incf	___fladd@aexp^0,w,c
  3189  0006D8  A4D8               	btfss	status,2,c
  3190  0006DA  EF71  F003         	goto	u1041
  3191  0006DE  EF74  F003         	goto	u1040
  3192  0006E2                     u1041:
  3193  0006E2  FFFF               	dw	65535	; assembler added errata NOP
  3194  0006E4  EF7D  F003         	goto	l1895
  3195  0006E8                     u1040:
  3196  0006E8  FFFF               	dw	65535	; assembler added errata NOP
  3197  0006EA  0E00               	movlw	0
  3198  0006EC  6E45               	movwf	___fladd@a^0,c
  3199  0006EE  0E00               	movlw	0
  3200  0006F0  6E46               	movwf	(___fladd@a+1)^0,c
  3201  0006F2  0E00               	movlw	0
  3202  0006F4  6E47               	movwf	(___fladd@a+2)^0,c
  3203  0006F6  0E00               	movlw	0
  3204  0006F8  6E48               	movwf	(___fladd@a+3)^0,c
  3205  0006FA                     l1895:
  3206  0006FA  FFFF               	dw	65535	; assembler added errata NOP
  3207  0006FC  8E47               	bsf	(___fladd@a+2)^0,7,c
  3208  0006FE  0E00               	movlw	0
  3209  000700  6E48               	movwf	(___fladd@a+3)^0,c
  3210  000702  EF8C  F003         	goto	l1901
  3211  000706                     l1899:
  3212  000706  FFFF               	dw	65535	; assembler added errata NOP
  3213  000708  0E00               	movlw	0
  3214  00070A  6E45               	movwf	___fladd@a^0,c
  3215  00070C  0E00               	movlw	0
  3216  00070E  6E46               	movwf	(___fladd@a+1)^0,c
  3217  000710  0E00               	movlw	0
  3218  000712  6E47               	movwf	(___fladd@a+2)^0,c
  3219  000714  0E00               	movlw	0
  3220  000716  6E48               	movwf	(___fladd@a+3)^0,c
  3221  000718                     l1901:
  3222  000718  FFFF               	dw	65535	; assembler added errata NOP
  3223  00071A  504F               	movf	___fladd@bexp^0,w,c
  3224  00071C  5C4E               	subwf	___fladd@aexp^0,w,c
  3225  00071E  B0D8               	btfsc	status,0,c
  3226  000720  EF94  F003         	goto	u1051
  3227  000724  EF97  F003         	goto	u1050
  3228  000728                     u1051:
  3229  000728  FFFF               	dw	65535	; assembler added errata NOP
  3230  00072A  EFC2  F003         	goto	l1937
  3231  00072E                     u1050:
  3232  00072E  FFFF               	dw	65535	; assembler added errata NOP
  3233  000730  AC4D               	btfss	___fladd@signs^0,6,c
  3234  000732  EF9D  F003         	goto	u1061
  3235  000736  EFA0  F003         	goto	u1060
  3236  00073A                     u1061:
  3237  00073A  FFFF               	dw	65535	; assembler added errata NOP
  3238  00073C  EFA3  F003         	goto	l1907
  3239  000740                     u1060:
  3240  000740  FFFF               	dw	65535	; assembler added errata NOP
  3241  000742  0E80               	movlw	128
  3242  000744  1A4D               	xorwf	___fladd@signs^0,f,c
  3243  000746                     l1907:
  3244  000746  FFFF               	dw	65535	; assembler added errata NOP
  3245  000748  C04F  F050         	movff	___fladd@bexp,___fladd@grs
  3246  00074C  C04E  F04F         	movff	___fladd@aexp,___fladd@bexp
  3247  000750  C050  F04E         	movff	___fladd@grs,___fladd@aexp
  3248  000754  C041  F050         	movff	___fladd@b,___fladd@grs
  3249  000758  C045  F041         	movff	___fladd@a,___fladd@b
  3250  00075C  C050  F045         	movff	___fladd@grs,___fladd@a
  3251  000760  C042  F050         	movff	___fladd@b+1,___fladd@grs
  3252  000764  C046  F042         	movff	___fladd@a+1,___fladd@b+1
  3253  000768  C050  F046         	movff	___fladd@grs,___fladd@a+1
  3254  00076C  C043  F050         	movff	___fladd@b+2,___fladd@grs
  3255  000770  C047  F043         	movff	___fladd@a+2,___fladd@b+2
  3256  000774  C050  F047         	movff	___fladd@grs,___fladd@a+2
  3257  000778  C044  F050         	movff	___fladd@b+3,___fladd@grs
  3258  00077C  C048  F044         	movff	___fladd@a+3,___fladd@b+3
  3259  000780  C050  F048         	movff	___fladd@grs,___fladd@a+3
  3260  000784                     l1937:
  3261  000784  FFFF               	dw	65535	; assembler added errata NOP
  3262  000786  0E00               	movlw	0
  3263  000788  6E50               	movwf	___fladd@grs^0,c
  3264  00078A  504F               	movf	___fladd@bexp^0,w,c
  3265  00078C  C04E  F049         	movff	___fladd@aexp,??___fladd
  3266  000790  6A4A               	clrf	(??___fladd+1)^0,c
  3267  000792  5E49               	subwf	??___fladd^0,f,c
  3268  000794  0E00               	movlw	0
  3269  000796  5A4A               	subwfb	(??___fladd+1)^0,f,c
  3270  000798  BE4A               	btfsc	(??___fladd+1)^0,7,c
  3271  00079A  EFD8  F003         	goto	u1071
  3272  00079E  504A               	movf	(??___fladd+1)^0,w,c
  3273  0007A0  E10A               	bnz	u1070
  3274  0007A2  0E1A               	movlw	26
  3275  0007A4  5C49               	subwf	??___fladd^0,w,c
  3276  0007A6  A0D8               	btfss	status,0,c
  3277  0007A8  EFD8  F003         	goto	u1071
  3278  0007AC  EFDB  F003         	goto	u1070
  3279  0007B0                     u1071:
  3280  0007B0  FFFF               	dw	65535	; assembler added errata NOP
  3281  0007B2  EF1E  F004         	goto	l827
  3282  0007B6                     u1070:
  3283  0007B6  FFFF               	dw	65535	; assembler added errata NOP
  3284  0007B8  5041               	movf	___fladd@b^0,w,c
  3285  0007BA  1042               	iorwf	(___fladd@b+1)^0,w,c
  3286  0007BC  1043               	iorwf	(___fladd@b+2)^0,w,c
  3287  0007BE  1044               	iorwf	(___fladd@b+3)^0,w,c
  3288  0007C0  A4D8               	btfss	status,2,c
  3289  0007C2  EFE5  F003         	goto	u1081
  3290  0007C6  EFE9  F003         	goto	u1080
  3291  0007CA                     u1081:
  3292  0007CA  FFFF               	dw	65535	; assembler added errata NOP
  3293  0007CC  0E01               	movlw	1
  3294  0007CE  EFEB  F003         	goto	u1090
  3295  0007D2                     u1080:
  3296  0007D2  FFFF               	dw	65535	; assembler added errata NOP
  3297  0007D4  0E00               	movlw	0
  3298  0007D6                     u1090:
  3299  0007D6  FFFF               	dw	65535	; assembler added errata NOP
  3300  0007D8  6E50               	movwf	___fladd@grs^0,c
  3301  0007DA  0E00               	movlw	0
  3302  0007DC  6E41               	movwf	___fladd@b^0,c
  3303  0007DE  0E00               	movlw	0
  3304  0007E0  6E42               	movwf	(___fladd@b+1)^0,c
  3305  0007E2  0E00               	movlw	0
  3306  0007E4  6E43               	movwf	(___fladd@b+2)^0,c
  3307  0007E6  0E00               	movlw	0
  3308  0007E8  6E44               	movwf	(___fladd@b+3)^0,c
  3309  0007EA  C04E  F04F         	movff	___fladd@aexp,___fladd@bexp
  3310  0007EE  EF29  F004         	goto	l826
  3311  0007F2                     l828:
  3312  0007F2  FFFF               	dw	65535	; assembler added errata NOP
  3313  0007F4  A050               	btfss	___fladd@grs^0,0,c
  3314  0007F6  EFFF  F003         	goto	u1101
  3315  0007FA  EF02  F004         	goto	u1100
  3316  0007FE                     u1101:
  3317  0007FE  FFFF               	dw	65535	; assembler added errata NOP
  3318  000800  EF09  F004         	goto	l1949
  3319  000804                     u1100:
  3320  000804  FFFF               	dw	65535	; assembler added errata NOP
  3321  000806  90D8               	bcf	status,0,c
  3322  000808  3050               	rrcf	___fladd@grs^0,w,c
  3323  00080A  0901               	iorlw	1
  3324  00080C  6E50               	movwf	___fladd@grs^0,c
  3325  00080E  EF0C  F004         	goto	l1951
  3326  000812                     l1949:
  3327  000812  FFFF               	dw	65535	; assembler added errata NOP
  3328  000814  90D8               	bcf	status,0,c
  3329  000816  3250               	rrcf	___fladd@grs^0,f,c
  3330  000818                     l1951:
  3331  000818  FFFF               	dw	65535	; assembler added errata NOP
  3332  00081A  A041               	btfss	___fladd@b^0,0,c
  3333  00081C  EF12  F004         	goto	u1111
  3334  000820  EF15  F004         	goto	u1110
  3335  000824                     u1111:
  3336  000824  FFFF               	dw	65535	; assembler added errata NOP
  3337  000826  EF17  F004         	goto	l1955
  3338  00082A                     u1110:
  3339  00082A  FFFF               	dw	65535	; assembler added errata NOP
  3340  00082C  8E50               	bsf	___fladd@grs^0,7,c
  3341  00082E                     l1955:
  3342  00082E  FFFF               	dw	65535	; assembler added errata NOP
  3343  000830  3444               	rlcf	(___fladd@b+3)^0,w,c
  3344  000832  3244               	rrcf	(___fladd@b+3)^0,f,c
  3345  000834  3243               	rrcf	(___fladd@b+2)^0,f,c
  3346  000836  3242               	rrcf	(___fladd@b+1)^0,f,c
  3347  000838  3241               	rrcf	___fladd@b^0,f,c
  3348  00083A  2A4F               	incf	___fladd@bexp^0,f,c
  3349  00083C                     l827:
  3350  00083C  FFFF               	dw	65535	; assembler added errata NOP
  3351  00083E  504E               	movf	___fladd@aexp^0,w,c
  3352  000840  5C4F               	subwf	___fladd@bexp^0,w,c
  3353  000842  A0D8               	btfss	status,0,c
  3354  000844  EF26  F004         	goto	u1121
  3355  000848  EF29  F004         	goto	u1120
  3356  00084C                     u1121:
  3357  00084C  FFFF               	dw	65535	; assembler added errata NOP
  3358  00084E  EFF9  F003         	goto	l828
  3359  000852                     u1120:
  3360  000852                     l826:
  3361  000852  FFFF               	dw	65535	; assembler added errata NOP
  3362  000854  BC4D               	btfsc	___fladd@signs^0,6,c
  3363  000856  EF2F  F004         	goto	u1131
  3364  00085A  EF32  F004         	goto	u1130
  3365  00085E                     u1131:
  3366  00085E  FFFF               	dw	65535	; assembler added errata NOP
  3367  000860  EF7F  F004         	goto	l1983
  3368  000864                     u1130:
  3369  000864  FFFF               	dw	65535	; assembler added errata NOP
  3370  000866  504F               	movf	___fladd@bexp^0,w,c
  3371  000868  A4D8               	btfss	status,2,c
  3372  00086A  EF39  F004         	goto	u1141
  3373  00086E  EF3C  F004         	goto	u1140
  3374  000872                     u1141:
  3375  000872  FFFF               	dw	65535	; assembler added errata NOP
  3376  000874  EF47  F004         	goto	l1965
  3377  000878                     u1140:
  3378  000878  FFFF               	dw	65535	; assembler added errata NOP
  3379  00087A  0E00               	movlw	0
  3380  00087C  6E41               	movwf	?___fladd^0,c
  3381  00087E  0E00               	movlw	0
  3382  000880  6E42               	movwf	(?___fladd+1)^0,c
  3383  000882  0E00               	movlw	0
  3384  000884  6E43               	movwf	(?___fladd+2)^0,c
  3385  000886  0E00               	movlw	0
  3386  000888  6E44               	movwf	(?___fladd+3)^0,c
  3387  00088A  EFD6  F005         	goto	l835
  3388  00088E                     l1965:
  3389  00088E  FFFF               	dw	65535	; assembler added errata NOP
  3390  000890  5045               	movf	___fladd@a^0,w,c
  3391  000892  2641               	addwf	___fladd@b^0,f,c
  3392  000894  5046               	movf	(___fladd@a+1)^0,w,c
  3393  000896  2242               	addwfc	(___fladd@b+1)^0,f,c
  3394  000898  5047               	movf	(___fladd@a+2)^0,w,c
  3395  00089A  2243               	addwfc	(___fladd@b+2)^0,f,c
  3396  00089C  5048               	movf	(___fladd@a+3)^0,w,c
  3397  00089E  2244               	addwfc	(___fladd@b+3)^0,f,c
  3398  0008A0  A044               	btfss	(___fladd@b+3)^0,0,c
  3399  0008A2  EF55  F004         	goto	u1151
  3400  0008A6  EF58  F004         	goto	u1150
  3401  0008AA                     u1151:
  3402  0008AA  FFFF               	dw	65535	; assembler added errata NOP
  3403  0008AC  EF23  F005         	goto	l2019
  3404  0008B0                     u1150:
  3405  0008B0  FFFF               	dw	65535	; assembler added errata NOP
  3406  0008B2  A050               	btfss	___fladd@grs^0,0,c
  3407  0008B4  EF5E  F004         	goto	u1161
  3408  0008B8  EF61  F004         	goto	u1160
  3409  0008BC                     u1161:
  3410  0008BC  FFFF               	dw	65535	; assembler added errata NOP
  3411  0008BE  EF68  F004         	goto	l1973
  3412  0008C2                     u1160:
  3413  0008C2  FFFF               	dw	65535	; assembler added errata NOP
  3414  0008C4  90D8               	bcf	status,0,c
  3415  0008C6  3050               	rrcf	___fladd@grs^0,w,c
  3416  0008C8  0901               	iorlw	1
  3417  0008CA  6E50               	movwf	___fladd@grs^0,c
  3418  0008CC  EF6B  F004         	goto	l1975
  3419  0008D0                     l1973:
  3420  0008D0  FFFF               	dw	65535	; assembler added errata NOP
  3421  0008D2  90D8               	bcf	status,0,c
  3422  0008D4  3250               	rrcf	___fladd@grs^0,f,c
  3423  0008D6                     l1975:
  3424  0008D6  FFFF               	dw	65535	; assembler added errata NOP
  3425  0008D8  A041               	btfss	___fladd@b^0,0,c
  3426  0008DA  EF71  F004         	goto	u1171
  3427  0008DE  EF74  F004         	goto	u1170
  3428  0008E2                     u1171:
  3429  0008E2  FFFF               	dw	65535	; assembler added errata NOP
  3430  0008E4  EF76  F004         	goto	l1979
  3431  0008E8                     u1170:
  3432  0008E8  FFFF               	dw	65535	; assembler added errata NOP
  3433  0008EA  8E50               	bsf	___fladd@grs^0,7,c
  3434  0008EC                     l1979:
  3435  0008EC  FFFF               	dw	65535	; assembler added errata NOP
  3436  0008EE  3444               	rlcf	(___fladd@b+3)^0,w,c
  3437  0008F0  3244               	rrcf	(___fladd@b+3)^0,f,c
  3438  0008F2  3243               	rrcf	(___fladd@b+2)^0,f,c
  3439  0008F4  3242               	rrcf	(___fladd@b+1)^0,f,c
  3440  0008F6  3241               	rrcf	___fladd@b^0,f,c
  3441  0008F8  2A4F               	incf	___fladd@bexp^0,f,c
  3442  0008FA  EF23  F005         	goto	l2019
  3443  0008FE                     l1983:
  3444  0008FE  FFFF               	dw	65535	; assembler added errata NOP
  3445  000900  5045               	movf	___fladd@a^0,w,c
  3446  000902  5C41               	subwf	___fladd@b^0,w,c
  3447  000904  5046               	movf	(___fladd@a+1)^0,w,c
  3448  000906  5842               	subwfb	(___fladd@b+1)^0,w,c
  3449  000908  5047               	movf	(___fladd@a+2)^0,w,c
  3450  00090A  5843               	subwfb	(___fladd@b+2)^0,w,c
  3451  00090C  5044               	movf	(___fladd@b+3)^0,w,c
  3452  00090E  0A80               	xorlw	128
  3453  000910  6E49               	movwf	??___fladd^0,c
  3454  000912  5048               	movf	(___fladd@a+3)^0,w,c
  3455  000914  0A80               	xorlw	128
  3456  000916  5849               	subwfb	??___fladd^0,w,c
  3457  000918  B0D8               	btfsc	status,0,c
  3458  00091A  EF91  F004         	goto	u1181
  3459  00091E  EF94  F004         	goto	u1180
  3460  000922                     u1181:
  3461  000922  FFFF               	dw	65535	; assembler added errata NOP
  3462  000924  EFC2  F004         	goto	l1993
  3463  000928                     u1180:
  3464  000928  FFFF               	dw	65535	; assembler added errata NOP
  3465  00092A  5041               	movf	___fladd@b^0,w,c
  3466  00092C  5C45               	subwf	___fladd@a^0,w,c
  3467  00092E  6E49               	movwf	??___fladd^0,c
  3468  000930  5042               	movf	(___fladd@b+1)^0,w,c
  3469  000932  5846               	subwfb	(___fladd@a+1)^0,w,c
  3470  000934  6E4A               	movwf	(??___fladd+1)^0,c
  3471  000936  5043               	movf	(___fladd@b+2)^0,w,c
  3472  000938  5847               	subwfb	(___fladd@a+2)^0,w,c
  3473  00093A  6E4B               	movwf	(??___fladd+2)^0,c
  3474  00093C  5044               	movf	(___fladd@b+3)^0,w,c
  3475  00093E  5848               	subwfb	(___fladd@a+3)^0,w,c
  3476  000940  6E4C               	movwf	(??___fladd+3)^0,c
  3477  000942  0EFF               	movlw	255
  3478  000944  2449               	addwf	??___fladd^0,w,c
  3479  000946  6E41               	movwf	___fladd@b^0,c
  3480  000948  0EFF               	movlw	255
  3481  00094A  204A               	addwfc	(??___fladd+1)^0,w,c
  3482  00094C  6E42               	movwf	(___fladd@b+1)^0,c
  3483  00094E  0EFF               	movlw	255
  3484  000950  204B               	addwfc	(??___fladd+2)^0,w,c
  3485  000952  6E43               	movwf	(___fladd@b+2)^0,c
  3486  000954  0EFF               	movlw	255
  3487  000956  204C               	addwfc	(??___fladd+3)^0,w,c
  3488  000958  6E44               	movwf	(___fladd@b+3)^0,c
  3489  00095A  0E80               	movlw	128
  3490  00095C  1A4D               	xorwf	___fladd@signs^0,f,c
  3491  00095E  6C50               	negf	___fladd@grs^0,c
  3492  000960  5050               	movf	___fladd@grs^0,w,c
  3493  000962  A4D8               	btfss	status,2,c
  3494  000964  EFB6  F004         	goto	u1191
  3495  000968  EFB9  F004         	goto	u1190
  3496  00096C                     u1191:
  3497  00096C  FFFF               	dw	65535	; assembler added errata NOP
  3498  00096E  EFCB  F004         	goto	l843
  3499  000972                     u1190:
  3500  000972  FFFF               	dw	65535	; assembler added errata NOP
  3501  000974  0E01               	movlw	1
  3502  000976  2641               	addwf	___fladd@b^0,f,c
  3503  000978  0E00               	movlw	0
  3504  00097A  2242               	addwfc	(___fladd@b+1)^0,f,c
  3505  00097C  2243               	addwfc	(___fladd@b+2)^0,f,c
  3506  00097E  2244               	addwfc	(___fladd@b+3)^0,f,c
  3507  000980  EFCB  F004         	goto	l843
  3508  000984                     l1993:
  3509  000984  FFFF               	dw	65535	; assembler added errata NOP
  3510  000986  5045               	movf	___fladd@a^0,w,c
  3511  000988  5E41               	subwf	___fladd@b^0,f,c
  3512  00098A  5046               	movf	(___fladd@a+1)^0,w,c
  3513  00098C  5A42               	subwfb	(___fladd@b+1)^0,f,c
  3514  00098E  5047               	movf	(___fladd@a+2)^0,w,c
  3515  000990  5A43               	subwfb	(___fladd@b+2)^0,f,c
  3516  000992  5048               	movf	(___fladd@a+3)^0,w,c
  3517  000994  5A44               	subwfb	(___fladd@b+3)^0,f,c
  3518  000996                     l843:
  3519  000996  FFFF               	dw	65535	; assembler added errata NOP
  3520  000998  5041               	movf	___fladd@b^0,w,c
  3521  00099A  1042               	iorwf	(___fladd@b+1)^0,w,c
  3522  00099C  1043               	iorwf	(___fladd@b+2)^0,w,c
  3523  00099E  1044               	iorwf	(___fladd@b+3)^0,w,c
  3524  0009A0  A4D8               	btfss	status,2,c
  3525  0009A2  EFD5  F004         	goto	u1201
  3526  0009A6  EFD8  F004         	goto	u1200
  3527  0009AA                     u1201:
  3528  0009AA  FFFF               	dw	65535	; assembler added errata NOP
  3529  0009AC  EF1A  F005         	goto	l2017
  3530  0009B0                     u1200:
  3531  0009B0  FFFF               	dw	65535	; assembler added errata NOP
  3532  0009B2  5050               	movf	___fladd@grs^0,w,c
  3533  0009B4  A4D8               	btfss	status,2,c
  3534  0009B6  EFDF  F004         	goto	u1211
  3535  0009BA  EFE2  F004         	goto	u1210
  3536  0009BE                     u1211:
  3537  0009BE  FFFF               	dw	65535	; assembler added errata NOP
  3538  0009C0  EF1A  F005         	goto	l2017
  3539  0009C4                     u1210:
  3540  0009C4  FFFF               	dw	65535	; assembler added errata NOP
  3541  0009C6  0E00               	movlw	0
  3542  0009C8  6E41               	movwf	?___fladd^0,c
  3543  0009CA  0E00               	movlw	0
  3544  0009CC  6E42               	movwf	(?___fladd+1)^0,c
  3545  0009CE  0E00               	movlw	0
  3546  0009D0  6E43               	movwf	(?___fladd+2)^0,c
  3547  0009D2  0E00               	movlw	0
  3548  0009D4  6E44               	movwf	(?___fladd+3)^0,c
  3549  0009D6  EFD6  F005         	goto	l835
  3550  0009DA                     l2001:
  3551  0009DA  FFFF               	dw	65535	; assembler added errata NOP
  3552  0009DC  90D8               	bcf	status,0,c
  3553  0009DE  3641               	rlcf	___fladd@b^0,f,c
  3554  0009E0  3642               	rlcf	(___fladd@b+1)^0,f,c
  3555  0009E2  3643               	rlcf	(___fladd@b+2)^0,f,c
  3556  0009E4  3644               	rlcf	(___fladd@b+3)^0,f,c
  3557  0009E6  AE50               	btfss	___fladd@grs^0,7,c
  3558  0009E8  EFF8  F004         	goto	u1221
  3559  0009EC  EFFB  F004         	goto	u1220
  3560  0009F0                     u1221:
  3561  0009F0  FFFF               	dw	65535	; assembler added errata NOP
  3562  0009F2  EFFD  F004         	goto	l2007
  3563  0009F6                     u1220:
  3564  0009F6  FFFF               	dw	65535	; assembler added errata NOP
  3565  0009F8  8041               	bsf	___fladd@b^0,0,c
  3566  0009FA                     l2007:
  3567  0009FA  FFFF               	dw	65535	; assembler added errata NOP
  3568  0009FC  A050               	btfss	___fladd@grs^0,0,c
  3569  0009FE  EF03  F005         	goto	u1231
  3570  000A02  EF06  F005         	goto	u1230
  3571  000A06                     u1231:
  3572  000A06  FFFF               	dw	65535	; assembler added errata NOP
  3573  000A08  EF0B  F005         	goto	l2011
  3574  000A0C                     u1230:
  3575  000A0C  FFFF               	dw	65535	; assembler added errata NOP
  3576  000A0E  80D8               	bsf	status,0,c
  3577  000A10  3650               	rlcf	___fladd@grs^0,f,c
  3578  000A12  EF0E  F005         	goto	l2013
  3579  000A16                     l2011:
  3580  000A16  FFFF               	dw	65535	; assembler added errata NOP
  3581  000A18  90D8               	bcf	status,0,c
  3582  000A1A  3650               	rlcf	___fladd@grs^0,f,c
  3583  000A1C                     l2013:
  3584  000A1C  FFFF               	dw	65535	; assembler added errata NOP
  3585  000A1E  504F               	movf	___fladd@bexp^0,w,c
  3586  000A20  B4D8               	btfsc	status,2,c
  3587  000A22  EF15  F005         	goto	u1241
  3588  000A26  EF18  F005         	goto	u1240
  3589  000A2A                     u1241:
  3590  000A2A  FFFF               	dw	65535	; assembler added errata NOP
  3591  000A2C  EF1A  F005         	goto	l2017
  3592  000A30                     u1240:
  3593  000A30  FFFF               	dw	65535	; assembler added errata NOP
  3594  000A32  064F               	decf	___fladd@bexp^0,f,c
  3595  000A34                     l2017:
  3596  000A34  FFFF               	dw	65535	; assembler added errata NOP
  3597  000A36  AE43               	btfss	(___fladd@b+2)^0,7,c
  3598  000A38  EF20  F005         	goto	u1251
  3599  000A3C  EF23  F005         	goto	u1250
  3600  000A40                     u1251:
  3601  000A40  FFFF               	dw	65535	; assembler added errata NOP
  3602  000A42  EFED  F004         	goto	l2001
  3603  000A46                     u1250:
  3604  000A46                     l2019:
  3605  000A46  FFFF               	dw	65535	; assembler added errata NOP
  3606  000A48  0E00               	movlw	0
  3607  000A4A  6E4E               	movwf	___fladd@aexp^0,c
  3608  000A4C  AE50               	btfss	___fladd@grs^0,7,c
  3609  000A4E  EF2B  F005         	goto	u1261
  3610  000A52  EF2E  F005         	goto	u1260
  3611  000A56                     u1261:
  3612  000A56  FFFF               	dw	65535	; assembler added errata NOP
  3613  000A58  EF4D  F005         	goto	l852
  3614  000A5C                     u1260:
  3615  000A5C  FFFF               	dw	65535	; assembler added errata NOP
  3616  000A5E  C050  F049         	movff	___fladd@grs,??___fladd
  3617  000A62  0E7F               	movlw	127
  3618  000A64  1649               	andwf	??___fladd^0,f,c
  3619  000A66  B4D8               	btfsc	status,2,c
  3620  000A68  EF38  F005         	goto	u1271
  3621  000A6C  EF3B  F005         	goto	u1270
  3622  000A70                     u1271:
  3623  000A70  FFFF               	dw	65535	; assembler added errata NOP
  3624  000A72  EF41  F005         	goto	l853
  3625  000A76                     u1270:
  3626  000A76  FFFF               	dw	65535	; assembler added errata NOP
  3627  000A78                     l2025:
  3628  000A78  FFFF               	dw	65535	; assembler added errata NOP
  3629  000A7A  0E01               	movlw	1
  3630  000A7C  6E4E               	movwf	___fladd@aexp^0,c
  3631  000A7E  EF4D  F005         	goto	l852
  3632  000A82                     l853:
  3633  000A82  FFFF               	dw	65535	; assembler added errata NOP
  3634  000A84  A041               	btfss	___fladd@b^0,0,c
  3635  000A86  EF47  F005         	goto	u1281
  3636  000A8A  EF4A  F005         	goto	u1280
  3637  000A8E                     u1281:
  3638  000A8E  FFFF               	dw	65535	; assembler added errata NOP
  3639  000A90  EF4D  F005         	goto	l852
  3640  000A94                     u1280:
  3641  000A94  FFFF               	dw	65535	; assembler added errata NOP
  3642  000A96  EF3C  F005         	goto	l2025
  3643  000A9A                     l852:
  3644  000A9A  FFFF               	dw	65535	; assembler added errata NOP
  3645  000A9C  504E               	movf	___fladd@aexp^0,w,c
  3646  000A9E  B4D8               	btfsc	status,2,c
  3647  000AA0  EF54  F005         	goto	u1291
  3648  000AA4  EF57  F005         	goto	u1290
  3649  000AA8                     u1291:
  3650  000AA8  FFFF               	dw	65535	; assembler added errata NOP
  3651  000AAA  EF87  F005         	goto	l2037
  3652  000AAE                     u1290:
  3653  000AAE  FFFF               	dw	65535	; assembler added errata NOP
  3654  000AB0  0E01               	movlw	1
  3655  000AB2  2641               	addwf	___fladd@b^0,f,c
  3656  000AB4  0E00               	movlw	0
  3657  000AB6  2242               	addwfc	(___fladd@b+1)^0,f,c
  3658  000AB8  2243               	addwfc	(___fladd@b+2)^0,f,c
  3659  000ABA  2244               	addwfc	(___fladd@b+3)^0,f,c
  3660  000ABC  A044               	btfss	(___fladd@b+3)^0,0,c
  3661  000ABE  EF63  F005         	goto	u1301
